:100000000C94D9120C940A130C940A130C940A132E
:100010000C940A130C940A130C940A130C940A13EC
:100020000C940A130C940A130C940A130C940A13DC
:100030000C940A130C947B730C940A130C940A13FB
:100040000C940A130C94FA430C940A130C940A139C
:100050000C940A130C940A130C94BD7B0C9457B4A3
:100060000C940A130C94E8420C940A130C940A138F
:100070000C940A130C940A130C940A130C940A138C
:100080000C940A130C940A130C940A130C940A137C
:100090000C940A130C940A130C940A130C940A136C
:1000A0000C940A130C940A130C940A130C940A135C
:1000B0000C940A130C940A130C940A130C940A134C
:1000C0000C940A130C940A130C940A130C940A133C
:1000D0000C940A130C940A130C9487430C94484311
:1000E0000C940A13912CAE2CDF2CFC2C112D3A2DE4
:1000F000A72D0D2EB62E40324E3247326E3272325E
:100100008C329536A132ED321F3346336F33C43310
:10011000D533E633F733083419349536A0359536A0
:10012000AB351B362136413670B073B062B066B065
:100130006CB0AAB077B07BB081B085B089B08FB019
:1001400093B097B0AAB09DB0A1B0A5B073B378B387
:100150007DB387B391B30AB49BB3A3B3ABB3B5B3C9
:10016000BFB3C9B3D8B3E2B30AB4ECB3F6B300B4C7
:10017000084AD73B3BCE016E84BCBFFDC12F3D6C0E
:1001800074319ABD56833DDA3D00C77F11BED9E474
:10019000BB4C3E916BAAAABE000000803F05A84C54
:1001A000CDB2D44EB93836A9020C50B99186880820
:1001B0003CA6AAAA2ABE000000803F004E414E493C
:1001C0004E495459494E46CDCCCC3D0AD7233C1715
:1001D000B7D13877CC2B329595E6241FB14F0A0062
:1001E0000020410000C84200401C4620BCBE4CCA52
:1001F0001B0E5AAEC59D74434F4D4D554E4943415C
:1002000054494F4E0044525952554E004552524F98
:10021000525300494E464F004543484F0047322F46
:1002200047332062616420706172616D657465722C
:10023000730A00206F6620004D424C20473239205F
:10024000706F696E74200059206F7574206F66207E
:1002500072616E67652028312D35292E0A005820DD
:100260006F7574206F662072616E67652028312D6E
:1002700035292E0A004D6573682070726F62696EB1
:100280006720646F6E652E0A005374617274206D6E
:100290006573682070726F62696E67207769746831
:1002A0002022473239205331222066697273742E1E
:1002B0000A004732380A47323920533200537461FA
:1002C00074653A20004D65736820626564206C6532
:1002D00076656C696E6720686173206E6F2064615B
:1002E00074612E0A0053206F7574206F662072614E
:1002F0006E67652028302D35292E0A004D657368FC
:1003000020706F696E742063616E6E6F7420626519
:10031000207265736F6C7665640A00456E642066B2
:10032000696C65206C6973740A00426567696E20A8
:1003300066696C65206C6973740A00286E6F2066AC
:10034000696C6529005344207072696E74696E6728
:10035000206279746520004E6F74205344207072BF
:10036000696E74696E670A0043757272656E7420F7
:1003700066696C653A200046696C652064656C6549
:100380007465643A0044656C6574696F6E206661DB
:10039000696C65642C2046696C653A200025697398
:1003A0000025696D20256973002569682025696D20
:1003B0002025697300256964202569682025696DF9
:1003C00020256973002569792025696420256968DD
:1003D0002025696D20256973005072696E74207440
:1003E000696D653A2000180213020C020502F7013C
:1003F0006F66660044454255473A004B494C4C45B0
:10040000442E20004D3131332053006F6B002C20DF
:10041000002C2000544845524D414C5F50524F54DF
:10042000454354494F4E004155544F5245504F5249
:10043000545F53445F53544154555300454D455206
:1004400047454E43595F5041525345520043415333
:10045000455F4C494748545F4252494748544E45CE
:10046000535300544F47474C455F4C4947485453FA
:1004700000534F4654574152455F504F5745520025
:100480004255494C445F50455243454E54004C45FB
:1004900056454C494E475F44415441005A5F5052C3
:1004A0004F4245004155544F4C4556454C00505223
:1004B000494E545F4A4F420050524F4752455353A2
:1004C000004155544F5245504F52545F54454D5082
:1004D00000564F4C554D45545249430045455052E6
:1004E0004F4D0053455249414C5F584F4E5F584F56
:1004F0004646004649524D574152455F4E414D4593
:100500003A4D61726C696E20312E312E39202847A8
:1005100069746875622920534F555243455F434FB4
:1005200044455F55524C3A68747470733A2F2F6784
:1005300069746875622E636F6D2F4D61726C696EA0
:100540004669726D776172652F4D61726C696E20BC
:1005500050524F544F434F4C5F56455253494F4EA4
:100560003A312E30204D414348494E455F54595051
:10057000453A3344205072696E7465722045585470
:1005800052554445525F434F554E543A31205555CC
:1005900049443A63656465326132662D34316132B3
:1005A0002D343734382D396231322D633535633689
:1005B000326633363766660A002F2F20002054003B
:1005C000205200416363656C65726174696F6E3AB5
:1005D0002050005741524E494E4721204C6F772002
:1005E0005A204A65726B206D6179206C65616420C8
:1005F000746F20756E77616E7465642070617573B9
:1006000065732E0A0020466C6F773A200000013691
:100610003726032BFFFFFF3C3D382AFFFFFFFF2E4D
:10062000303E12FFFFFFFFFFFFFF0809FF2C071AF4
:100630001C18FFFFFF08440A2C4324221E20643AA2
:100640000020693A0020703A00496E76616C696456
:100650002065787472756465720A0043290A006126
:10066000626C656420286D696E2074656D70200071
:10067000436F6C6420657874727564657320617271
:1006800065200020643A0020693A0020703A004E4C
:100690006F2063617365206C696768740A00454563
:1006A00050524F4D204F4B0A00205A004475616C48
:1006B00020456E6473746F702041646A7573746D45
:1006C000656E7420286D6D293A20003F4B207661BD
:1006D0006C7565206F7574206F662072616E67653A
:1006E0002028302D3130292E0A00416476616E6356
:1006F00065204B3D004163746976652045787472CE
:10070000756465723A2000496E76616C6964206593
:10071000787472756465720A0043616E6E6F74203E
:10072000656E746572207375626469723A20004761
:100730003239205332005370656369616C204D6516
:100740006E753A204E657874204D65736820506F41
:10075000696E740A00473239205331005370656363
:1007600069616C204D656E753A2053746172742016
:100770004D657368204C6576656C696E670A004D3F
:1007800031343020533630005370656369616C201A
:100790004D656E753A2050726568656174204265DA
:1007A000640A004D353031005370656369616C2017
:1007B0004D656E753A205265616420454550524F33
:1007C0004D0A004D353030005370656369616C200F
:1007D0004D656E753A205361766520454550524F00
:1007E0004D0A004D33303320452D31205336302013
:1007F0004338205531005370656369616C204D6545
:100800006E753A204175746F2054756E6520486F7F
:1008100074626564205069640A004D3330332045AA
:10082000302053323030204338205531005370652A
:100830006369616C204D656E753A204175746F2057
:1008400054756E6520486F74656E64205049440A83
:10085000003C5370656369616C5F4D656E753E0069
:100860003C5370656369616C5F4D656E753E002F2A
:10087000002F002F002F2E2E0A002F2E2E002F2E9D
:100880002E003C5370656369616C5F4D656E753E0B
:100890000A003C5370656369616C204D656E753E5E
:1008A000003C5370656369616C204D656E753E0058
:1008B0003C5361766520454550524F4D3E003C53B8
:1008C00061766520454550524F4D3E003C4E65785F
:1008D00074204D65736820506F696E743E003C4E05
:1008E000657874204D65736820506F696E743E00A2
:1008F0003C5374617274204D657368204C65766555
:100900006C696E673E003C5374617274204D657370
:1009100068204C6576656C696E673E003C50726578
:1009200068656174206265643E003C50726568656C
:100930006174206265643E003C52656164204545F7
:1009400050524F4D3E003C52656164204545505227
:100950004F4D3E003C4175746F2054756E652048C4
:100960006F74626564205049443E003C4175746F69
:100970002054756E6520486F746265642050494448
:100980003E003C4175746F2054756E6520486F744D
:10099000656E64205049443E003C4175746F20549C
:1009A000756E6520486F74656E64205049443E0042
:1009B0003C457869743E003C457869743E00563188
:1009C0003136004A333320004D3530300A4D343251
:1009D000302053310A4731205A31302046323430EA
:1009E0000A47312058302059302046363030300008
:1009F0004A3232004A3232004731205A35204632DC
:100A000034300A47312058313930205932302046AD
:100A1000363030300A4731205A30204632343000E8
:100A20004731205A3520463234300A473120583178
:100A3000393020593139302046363030300A47318C
:100A4000205A302046323430004731205A35204673
:100A50003234300A47312058313930205932302071
:100A600046363030300A4731205A30204632343052
:100A7000004739310A4731205A313020463234306C
:100A80000A4739300A4732380A4732390A47312093
:100A9000583230205932302046363030300A473113
:100AA000205A302046323430004A3032004A313247
:100AB000004731205A3130004F4B004731205A3126
:100AC0003000473930004731204525694635303000
:100AD00000473120452D302E314625690047312011
:100AE00045302E31462569004731205A2569462573
:100AF00069004731205A2D302E3146256900473193
:100B0000205A302E31462569004731205925694643
:100B1000256900473120592D302E3146256900477F
:100B2000312059302E31462569004731205825693A
:100B300046256900473120582D302E314625690061
:100B400047312058302E314625690047393100475A
:100B5000323800473238205A00473238205900478F
:100B600032382058004132305620004731205A3167
:100B700030004A3034004A3231004A3230004B49AA
:100B80004C4C45442E20004A303400454E4400462B
:100B90004E20004A3032003939393A393939004D5E
:100BA0000048004137562000413656202D2D2D009B
:100BB0004A30320041365620005A3A2000593A2035
:100BC00000583A2000413556004134562000413348
:100BD0005620004132562000413156200041305607
:100BE00020004D3834004A3136004A313800473948
:100BF000310A4731205A313020463234300A4739E1
:100C000030004A3134004A3030004A3031004A3135
:100C10003000656E7175657565696E672022004BE1
:100C2000494C4C45442E20005072696E7465722008
:100C300073746F707065642064756520746F2065CF
:100C400072726F72732E2046697820746865206511
:100C500072726F7220616E6420757365204D393930
:100C60003920746F20726573746172742E20285459
:100C7000656D706572617475726520697320726547
:100C80007365742E205365742069742061667465E1
:100C9000722072657374617274696E67290A004EFE
:100CA0006F20436865636B73756D20776974682086
:100CB0006C696E65206E756D6265722C204C617377
:100CC00074204C696E653A20004E6F20436865635E
:100CD0006B73756D2077697468206C696E65206E22
:100CE000756D6265722C204C617374204C696E6561
:100CF0003A2000636865636B73756D206D69736D71
:100D0000617463682C204C617374204C696E653A81
:100D100020004C696E65204E756D626572206973A6
:100D2000206E6F74204C617374204C696E65204E88
:100D3000756D6265722B312C204C617374204C6987
:100D40006E653A20004D313130004D33310053444F
:100D50002072656164206572726F720A00446F6E62
:100D600065207072696E74696E672066696C650AC9
:100D70000024F4D43050C38E20C2A24017828B705E
:100D800011127A910D816CD90AA861E108C75866E1
:100D900007615143061E4B5D05C145A7041A411169
:100DA00004093D9803713931034036DB0265339104
:100DB00002D4305402802E1D02632CEE01752AC528
:100DC00001B028A001102781018F2564012B244B3D
:100DD00001E0223401AC211F018D200D01801FFC98
:100DE00000841EED00971DDF00B81CD200E61BC674
:100DF00000201BBC00641AB200B219A8000A19A096
:100E0000006A189900D117910040178B00B516841D
:100E10000031167E00B31579003A157300C7146FC0
:100E20000058146A00EE1366008813630025135EF1
:100E300000C7125B006C12570015125400C111510B
:100E40000070114F0021114B00D61049008D104742
:100E5000004610440002104200C00F4000800F3EC8
:100E600000420F3C00060F3B00CB0E3800930E37BC
:100E7000005C0E3500270E3400F30D3200C10D3139
:100E800000900D3000600D2E00320D2D00050D2C50
:100E900000D90C2B00AE0C2900850C29005C0C2716
:100EA00000350C27000E0C2600E80B2400C40B2490
:100EB00000A00B23007D0B23005A0B2100390B21CE
:100EC00000180B2000F80A1F00D90A1E00BB0A1EDA
:100ED000009D0A1D00800A1D00630A1C00470A1BB2
:100EE000002C0A1B00110A1A00F7091A00DD091963
:100EF00000C4091900AB091900920917007B0918F1
:100F000000630917004C091600360916002009165F
:100F1000000A091500F5081500E0081400CC0814B3
:100F200000B8081400A4081400900813007D0812EB
:100F3000006B08130058081200460812003408110C
:100F400000230811001208110001081100F0071019
:100F500000E0071000D0071000C0071000B0070F16
:100F600000A107100091070E0083070F0074070F00
:100F70000065070E0057070E0049070E003B070DDE
:100F8000002E070E0020070D0013070D0006070DA9
:100F900000F9060C00ED060D00E0060C00D4060C6E
:100FA00000C8060C00BC060C00B0060C00A4060B22
:100FB0000099060C008D060B0082060B0077060BCD
:100FC000006C060B0061060A0057060B004C060A6F
:100FD0000042060A0038060A002E060A0024060A05
:100FE000001A060A001006090007060A00FD050996
:100FF00000F4050900EB050900E2050900D905091F
:1010000000D0050900C7050900BE050900B505089F
:1010100000AD050800A50509009C05080094050819
:10102000008C050800840508007C0508007405088C
:10103000006C050700650508005D050700560508FA
:10104000004E050700470507004005080038050762
:1010500000310507002A050700230507001C0506C7
:1010600000160507000F0507000805060002050722
:1010700000FB040600F5040700EE040600E8040681
:1010800000E2040700DB040600D5040600CF0406D6
:1010900000C9040600C3040600BD040600B7040628
:1010A00000B1040500AC040600A6040600A0040577
:1010B000009B04060095040500900406008A0405C0
:1010C0000085040500800406007A04050075040507
:1010D00000700405006B040500660405006104054A
:1010E000005C04050057040500520405004D04058A
:1010F0000048040500430405003E0404003A0405CA
:101100000035040500300404002C04050027040405
:1011100000230405001E0404001A0404001604053C
:1011200000110404000D0404000904050004040473
:101130000000040400FC030400F8030400F40304AA
:1011400000F0030400EC030400E8030400E40304DB
:1011500000E0030400DC030400D8030400D403040B
:1011600000D0030400CC030400C8030300C503033C
:101170000024F404D9201BC40C5C0E9804C4095F3D
:101180000265077101F405F900FB04B30048048708
:1011900000C10369005803550003034500BE023A2D
:1011A000008402310053022A002902250004022093
:1011B00000E4011C00C8011900AF011700980114D8
:1011C0000084011300710110006101100051010E33
:1011D0000043010D0036010B002B010B0020010B19
:1011E00000150109000C01090003010800FB0008BB
:1011F00000F3000800EB000700E4000600DE000634
:1012000000D8000600D2000600CC000500C700058B
:1012100000C2000500BD000400B9000400B50004D0
:1012200000B1000400AD000400A9000400A5000303
:1012300000A20003009F0004009B0003009800032D
:10124000009500020093000300900003008D00024F
:10125000008B000300880002008600020084000367
:1012600000810002007F0002007D0002007B00027E
:10127000007900020077000100760002007400028D
:101280000072000100710002006F0002006D000199
:10129000006C0002006A00010069000200670001A2
:1012A00000660001006500010064000200620001A8
:1012B0000061000100600001005F0002005D0001AC
:1012C000005C0001005B0001005A000100590001B0
:1012D00000580001005700010056000100550001B0
:1012E00000540001005300000053000100520001AF
:1012F0000051000100500001004F0001004E0000AD
:10130000004E0001004D0001004C0001004B0000A8
:10131000004B0001004A00010049000100480000A4
:10132000004800010047000100460000004600019F
:10133000004500000045000100440001004300009A
:101340000043000100420000004200010041000093
:101350000041000100400001003F0000003F00018B
:10136000003E0000003E0001003D0000003D000185
:10137000003C0000003C0000003C0001003B00007D
:10138000003B0001003A0000003A00010039000073
:10139000003900010038000000380000003800016A
:1013A0000037000000370001003600000036000062
:1013B0000036000100350000003500000035000156
:1013C000003400000034000000340001003300004D
:1013D0000033000000330001003200000032000042
:1013E0000032000100310000003100000031000136
:1013F000003000000030000000300001002F00002D
:10140000002F0000002F0000002F0001002E000020
:10141000002E0000002E0001002D0000002D000015
:10142000002D0000002D0001002C0000002C000009
:10143000002C0000002C0001002B0000002B0000FD
:10144000002B0000002B0001002A0000002A0000F1
:10145000002A0000002A00010029000000290000E5
:1014600000290000002900000029000100280000D8
:1014700000280000002800000028000000280001CB
:1014800000270000002700000027000000270000C0
:1014900000270001002600000026000000260000B2
:1014A00000260000002600010025000000250000A5
:1014B0000025000000250000002500000025000197
:1014C000002400000024000000240000002400008C
:1014D000002400010023000000230000002300007E
:1014E000002300000023000000230000002300016F
:1014F0000022000000220000002200000022000064
:101500000022000000220001002100000021000054
:101510000021000000210000002100000021000047
:101520000021000100200000002000000020000039
:10153000002000000020000000200000002000002B
:1015400000200001001F0000001F0000001F00001D
:10155000001F0000001F0000001F0000001F00010E
:10156000001E0000001E0000001E0000001E000003
:1015700000C23100001C260000F4190000D80F0042
:1015800000EB080000C004000075020000400100EC
:1015900000526573656E643A20006F6B0020746FB3
:1015A0006F206C6F6E6720657874727573696F6EEB
:1015B0002070726576656E7465640A0020636F6CD6
:1015C0006420657874727573696F6E2070726576C9
:1015D000656E7465640A00627573793A207061758E
:1015E00073656420666F7220696E7075740A00629C
:1015F0007573793A2070617573656420666F722027
:10160000757365720A00627573793A2070726F6340
:10161000657373696E670A004A3135004B494C4C5B
:1016200045442E20004B494C4C2063617573656422
:10163000206279204B494C4C20627574746F6E2F78
:1016400070696E0A004B494C4C45442E20004B49B2
:101650004C4C2063617573656420627920746F6FF0
:10166000206D75636820696E6163746976652074A6
:10167000696D65202D2063757272656E7420636FCD
:101680006D6D616E643A20004A3131005072696EAE
:101690007465722068616C7465642E206B696C6C73
:1016A00028292063616C6C6564210A000000A0C0D9
:1016B00000000000000000005761726E696E673A1A
:1016C00020486F6D696E672042756D7020446976A1
:1016D00069736F72203C20310A000202040000A0EE
:1016E000400000A0400000004000005C43000057A4
:1016F0004300004E43FFFFFF20746F6F206C6F6E3E
:101700006720657874727573696F6E207072657684
:10171000656E7465640A0020636F6C64206578747C
:10172000727573696F6E2070726576656E7465642C
:101730000A00454550524F4D206461746173697AC7
:1017400065206572726F722E0A00290A0020627984
:101750007465733B20637263200053657474696E13
:1017600067732053746F726564202800290A002073
:1017700062797465733B2063726320002073746F19
:101780007265642073657474696E67732072657422
:10179000726965766564202800202863616C637532
:1017A0006C6174656429210A0020213D20004545B3
:1017B00050524F4D20435243206D69736D617463E5
:1017C00068202D202873746F7265642920002053CF
:1017D000697A653A2000496E6465783A2000204DA8
:1017E00061726C696E3D563535290A0028454550B1
:1017F000524F4D3D00454550524F4D207665727316
:10180000696F6E206D69736D617463682000024AB0
:101810003135004A3132004A3137002020506C61A6
:101820006E6E657242756666657242797465733A6A
:1018300020002046726565204D656D6F72793A20F3
:1018400000436F6D70696C65643A204E6F7620318D
:101850003720323031380A00207C20417574686F9F
:10186000723A2028646176696472616D69726F2CC6
:1018700020666F7220416E796375626963206933F7
:10188000204D656761290A00323031392D31312D03
:10189000313500204C617374205570646174656447
:1018A0003A2000312E312E390A004D61726C696E7A
:1018B0000020536F6674776172652052657365749A
:1018C0000A00205761746368646F6720526573650E
:1018D000740A002042726F776E206F757420526513
:1018E0007365740A002045787465726E616C2052CD
:1018F000657365740A00506F77657255700A0073DE
:10190000746172740A004D3234004D3233202573F5
:10191000006175746F25692E67006572726F7220A1
:1019200077726974696E6720746F2066696C650AE6
:1019300000205A3A0020593A0020583A00656E6457
:1019400073746F7073206869743A2000446F6E6519
:1019500020736176696E672066696C652E0A004D9A
:101960003239006F70656E206661696C65642C2089
:1019700046696C653A200043616E6E6F74206F702B
:10198000656E2073756264697220004A3035004AC2
:101990003233004739310A4731205A2D3130204641
:1019A0003234300A47393000534420636172642076
:1019B0006F6B0A006F70656E526F6F74206661699D
:1019C0006C65640A00766F6C756D652E696E69745E
:1019D000206661696C65640A004572726F723A0034
:1019E000534420696E6974206661696C0A006563FE
:1019F000686F3A001000C90210012C014001220159
:101A000070011801B0010E01F00104015002FA004A
:101A1000B002F0003003E600D003DC009004D200F6
:101A20007005C800A006BE000008B400B009AA00F6
:101A3000D00BA000600E960060118C000015820093
:101A400020197800C01D6E00A0226400B0275A0043
:101A5000902C500000314600E0343C001038320039
:101A6000903A2800603C1E00A03D1400803E0A0011
:101A7000203F00002CFFFFFFFFFF000101010101DB
:101A80006265640A002C2073797374656D20737429
:101A90006F7070656421204865617465725F4944A8
:101AA0003A20004265642068656174696E6720664B
:101AB00061696C65640048656174696E6720666180
:101AC000696C65640045312048656174696E672002
:101AD0006661696C65640048656174696E6720665B
:101AE00061696C65640070012C0190012701B001EF
:101AF0002201C0011D01F001180110021301300282
:101B00000E016002090190020401C002FF000003FF
:101B1000FA004003F5008003F000D003EB0020043E
:101B2000E6007004E100E004DC004005D700C005D9
:101B3000D2004006CD00D006C8008007C3003008A0
:101B4000BE00F008B900C009B400B00AAF00B00B85
:101B5000AA00D00CA500000EA000500F9B00C010E2
:101B600096005012910000148C00C0158700B01729
:101B70008200B0197D00D01B7800001E7300402049
:101B80006E0090226900F024640040275F009029D5
:101B90005A00E02B5500102E500020304B00103220
:101BA0004600E033410090353C0010373700703874
:101BB0003200A0392D00B03A2800A03B2300603C41
:101BC0001E00103D1900903D1400103E0F00703EA5
:101BD0000A00C03E0500003F0000403FFBFF803F81
:101BE000F6FFC03FF1FF453120544845524D414C6E
:101BF0002052554E415741590042454420544845D2
:101C0000524D414C2052554E415741590054686540
:101C1000726D616C2052756E61776179004531207B
:101C20004572723A204D415854454D5000457272EC
:101C30003A204D415854454D5020424544004D41B5
:101C40005854454D50207472696767657265640029
:101C50004531204572723A204D494E54454D500051
:101C60004572723A204D494E54454D5020424544EC
:101C7000004D494E54454D50207472696767657236
:101C80006564004D383420582059205A20450020E2
:101C90002F002042403A0020403A003A0043617051
:101CA0003A00205A00205900580020204D61783A0F
:101CB0002000205A00205900580020204D696E3A1B
:101CC00020004F6E20004F666600536F66742065DB
:101CD0006E6473746F70733A20004B642000236449
:101CE0006566696E652044454641554C545F004B1E
:101CF00069200023646566696E6520444546415548
:101D00004C545F004B70200023646566696E65204B
:101D100044454641554C545F005049442041757438
:101D20006F74756E652066696E69736865642120DD
:101D300050757420746865206C617374204B702C2E
:101D4000204B6920616E64204B6420636F6E737456
:101D5000616E74732066726F6D2062656C6F7720A0
:101D6000696E746F20436F6E66696775726174691E
:101D70006F6E2E680A00504944204175746F747567
:101D80006E65206661696C6564212074696D656F9C
:101D900075740A00453120544845524D414C20523B
:101DA000554E415741590042454420544845524DF3
:101DB000414C2052554E4157415900546865726D4F
:101DC000616C2052756E61776179004531204865FC
:101DD0006174696E67206661696C65640042656460
:101DE0002068656174696E67206661696C6564006E
:101DF00048656174696E67206661696C656400504E
:101E00004944204175746F74756E65206661696C14
:101E10006564212054656D7065726174757265200A
:101E2000746F6F20686967680A00204B643A20006D
:101E3000204B693A2000204B703A20000A20436C66
:101E4000617373696320504944200A002054753A35
:101E50002000204B753A2000206D61783A20002048
:101E60006D696E3A200020643A2000206269617337
:101E70003A2000504944204175746F74756E652096
:101E80006661696C656421204261642065787472C2
:101E900075646572206E756D6265720A0050494402
:101EA000204175746F74756E652073746172740A65
:101EB000004F66660A004661646520486569676888
:101EC000742000426564204C6576656C696E6720FD
:101ED000004661696C656420746F20656E61626C98
:101EE0006520426564204C6576656C696E670A0002
:101EF0004D65736820426564204C6576656C20648E
:101F00006174613A0A004D65736820706F696E7480
:101F10002063616E6E6F74206265207265736F6CF2
:101F20007665640A004D34323120696E636F7272D7
:101F300065637420706172616D657465722075737C
:101F40006167650A002066697273740A005A005955
:101F5000005800486F6D652000546F6F20666172F5
:101F60002066726F6D207265666572656E636520AE
:101F7000706F696E740A007C3C3E5E2B3D3F2F5BA8
:101F80005D3B2C2A225C0020496E76616C696420DE
:101F9000657874727564657220000000A0C000004E
:101FA00000000000000000005743000057430000FD
:101FB0004E43486F6D696E67206661696C656400A9
:101FC000206E6F7420656E74657265642E0A005011
:101FD000726F7465637465642050696E0A004A30DC
:101FE00036004A3034004A30370020573A004A3031
:101FF00038004A30390020573A00205A3A00205918
:102000003A0020436F756E7420583A0020453A001C
:10201000205A3A0020593A00583A004861726463E5
:102020006F6465642044656661756C7420536574E3
:1020300074696E6773204C6F616465640A00B80B45
:102040000000B80B00003C0000001027000000005A
:10205000FA430000FA430000C04000007042000054
:10206000A0420000A0420000C843E17AD2422028EA
:102070006D6D290020204D393030204B004C696EA9
:1020800065617220416476616E63653A0A0020449E
:102090000020490020204D333034205000204400DF
:1020A00020490020204D3330312050005049442039
:1020B00073657474696E67733A0A00205A002020B1
:1020C0004D36363600456E6473746F702061646AF5
:1020D0007573746D656E743A0A00205A00205900B9
:1020E0002020473239205333205800205A00202026
:1020F0004D3432302053004D6573682042656420B2
:102100004C6576656C696E673A0A00205A00205962
:102110000020204D323036205800486F6D65206F0A
:1021200066667365743A0A00204500205A002059FB
:102130000020580020540020530020204D3230351C
:1021400020510020453C6D61785F655F6A65726B68
:102150003E0020583C6D61785F785F6A65726B3E27
:1021600020593C6D61785F795F6A65726B3E205AD9
:102170003C6D61785F7A5F6A65726B3E00416476A0
:10218000616E6365643A20513C6D696E5F7365678B
:102190006D656E745F74696D655F75733E20533C49
:1021A0006D696E5F66656564726174653E20543C5E
:1021B0006D696E5F74726176656C5F666565647289
:1021C0006174653E0020540020520020204D3230C2
:1021D00034205000416363656C65726174696F6E91
:1021E0002028756E6974732F7332293A20503C7021
:1021F00072696E745F616363656C3E20523C726508
:1022000074726163745F616363656C3E20543C74F7
:10221000726176656C5F616363656C3E0A002045A0
:1022200000205A0020590020204D32303120580023
:102230004D6178696D756D20416363656C65726190
:1022400074696F6E2028756E6974732F7332293A22
:102250000A00204500205A0020590020204D32302D
:10226000332058004D6178696D756D206665656431
:1022700072617465732028756E6974732F73293ABF
:102280000A00204500205A0020590020204D3932F4
:1022900020580053746570732070657220756E69E4
:1022A000743A0A0020204D3230302044300A002099
:1022B000204D3230302044002044697361626C65E7
:1022C000640A0046696C616D656E74207365747490
:1022D000696E67733A002020473231202020203B6E
:1022E00000545249474745524544006F70656E009F
:1022F0003A20007A325F6D696E007A5F6D696E0018
:10230000795F6D696E00785F6D696E005265706F00
:102310007274696E6720656E6473746F7020737475
:10232000617475730A000A4D656173757265642086
:10233000706F696E74733A0A005A206F666673652F
:10234000743A20004E756D20582C593A20352C35A2
:102350000A004572726F722077726974696E672025
:10236000746F20454550524F4D210A000000210056
:10237000240027002A002D00300033000101000056
:10238000040107010A0100002200250028002B009B
:102390002E003100340002010000050108010B018C
:1023A000000020002300260029002C002F0032000E
:1023B00000010000030106010901050505050705E7
:1023C00008080808020202020A0A080804040404B1
:1023D00001010101010101010303030303030303DD
:1023E000040707070C0C0C0C0C0C0C0C020202026C
:1023F00006060606060606060B0B0B0B0B0B0B0B55
:102400000102102020080810204010204080020106
:1024100002010804020101020408102040808040EB
:1024200020100804020180040201804020100804EA
:102430000201080402010102040810204080010288
:1024400004081020408000000A0B02090C0D0E0841
:10245000070304010000000000000000000000006D
:10246000000000000000000000000000000000006C
:102470000000121110000000000000000000000029
:10248000000000000000000000000000556E6B6EB0
:102490006F776E20636F6D6D616E643A202200006D
:1024A0000048420000484200008040000000005701
:1024B000726974696E6720746F2066696C653A2072
:1024C000006F70656E206661696C65642C204669DA
:1024D0006C653A20006F70656E206661696C65649A
:1024E0002C2046696C653A200046696C652073654E
:1024F0006C65637465640A002053697A653A20004C
:1025000046696C65206F70656E65643A20002066D0
:10251000696C653A2000646F696E67006672657366
:1025200068004E6F772000454E4420535542524F6D
:102530005554494E450A002220706F7300222070C6
:102540006172656E743A2200535542524F55544998
:102550004E452043414C4C207461726765743A22A9
:10256000004B494C4C45442E2000747279696E67CB
:1025700020746F2063616C6C207375622D67636FCC
:1025800064652066696C6573207769746820746F70
:102590006F206D616E79206C6576656C732E204DB1
:1025A0004158206C6576656C2069733A0000DDC087
:1025B0001DBB11241FBECFEFD1E2DEBFCDBF00E0B7
:1025C0000CBF13E0A0E0B2E0EEE4FDE901E00BBFD8
:1025D00002C007900D92AA3DB107D9F726E1AAEDF6
:1025E000B3E001C01D92A93FB207E1F712E1C8EDC7
:1025F000D2E100E006C021970109802FFE010E9470
:10260000FFCDC73DD10780E00807A9F70E943EBB78
:102610000C9496CE0C9400002F923F924F925F92B2
:102620006F927F928F929F92AF92BF92CF92DF92E2
:10263000EF92FF920F931F93CF93DF93CDB7DEB747
:10264000CB56D1090FB6F894DEBF0FBECDBF91E0D7
:102650009093F90A8091AE168D3411F40C94D01C2D
:10266000843511F40C94B729873411F00C94032AA3
:102670002090AC163090AD162CE12216310409F4EE
:102680003EC6A4F444E0241631044CF452E025166E
:1026900031040CF046C037FE3DC00C94CC1C64E005
:1026A0002616310409F4ECC50C94CC1C7AE52716E7
:1026B000310411F40C94051C6CF49DE129163104CD
:1026C00009F422C6AAE22A16310411F40C947A1BEA
:1026D0000C94CC1CBBE52B16310411F40C94091C92
:1026E000ECE52E16310411F00C94CC1C9FE4292E3D
:1026F00092E0392E27E0E22E2BE0F22E67EF73E016
:1027000079AF68AF3AEDC32E33E0D32E00E010E08E
:102710000C94481C8091410281110C940A2A0C945B
:10272000052A80914102882311F40C94052A0E9405
:10273000439982E50E94BA3E882309F450C10E9461
:102740003A3E4B015C0120E030E0A9010E94BDC689
:10275000882309F474C12091F7033091F803409164
:10276000F9035091FA0328AF39AF4AAF5BAF4091FC
:10277000FB035091FC036091FD037091FE034CAF8D
:102780005DAF6EAF7FAF6091140B7091150B8091B0
:10279000160B9091170B2C966CAF7DAF8EAF9FAF41
:1027A0002C978091180B9091190BA0911A0BB09156
:1027B0001B0B28968CAF9DAFAEAFBFAF28972C9662
:1027C0002CAD3DAD4EAD5FAD2C9768AD79AD8AAD0A
:1027D0009BAD0E94BDC681110FC028962CAD3DADAA
:1027E0004EAD5FAD28976CAD7DAD8EAD9FAD0E94B7
:1027F000BDC6882309F423C111E092E029163104F3
:1028000009F010E020E030E0A901C501B4010E9408
:10281000BDC6881F8827881F181759F020E030E0B0
:1028200040E85FEB64962CAF3DAF4EAF5FAF64976F
:102830000AC040E050E060E87FE364964CAF5DAFD3
:102840006EAF7FAF649728AD39AD4AAD5BAD2C96C6
:102850006CAD7DAD8EAD9FAD2C970E94E6CA6096A3
:102860006CAF7DAF8EAF9FAF60972CAD3DAD4EADE1
:102870005FAD28966CAD7DAD8EAD9FAD28970E9463
:10288000E6CA6B017C0160962CAD3DAD4EAD5FADEF
:102890006097CA01B9010E9422C72B013C01A70120
:1028A0009601C701B6010E9422C79B01AC01C3017A
:1028B000B2010E94E7CA0E9452CD24966CAF7DAF50
:1028C0008EAF9FAF249720E030E040E05FE30E94AE
:1028D00022C72B013C01A5019401C501B4010E944E
:1028E00022C74B015C01A3019201C301B2010E9406
:1028F00022C79B01AC01C501B4010E94E6CA0E9437
:1029000052CD64962CAD3DAD4EAD5FAD64970E9447
:1029100022C74B015C01C701B601905824962CAD2B
:102920003DAD4EAD5FAD24970E94C3CBA501940190
:102930000E9422C76B017C012C962CAD3DAD4EADA3
:102940005FAD2C9768AD79AD8AAD9BAD0E94E7CAAB
:1029500020E030E040E05FE30E9422C79B01AC0131
:10296000C701B6010E94E7CA28AD39AD4AAD5BADDB
:102970000E94E6CA6B017C0128962CAD3DAD4EADA0
:102980005FAD28976CAD7DAD8EAD9FAD0E94E7CA5F
:1029900020E030E040E05FE30E9422C72B013C01D1
:1029A00024962CAD3DAD4EAD5FAD249760966CADD9
:1029B0007DAD8EAD9FAD60970E94C3CBA501940104
:1029C0000E9422C79B01AC01C301B2010E94E7CA69
:1029D0002CAD3DAD4EAD5FAD0E94E6CA14C089E49A
:1029E0000E94BA3E882329F00E943A3E6B017C0186
:1029F00003C0C12CD12C76018AE40E94BA3E882300
:102A000009F10E943A3E2C966CAF7DAF8EAF9FAF1E
:102A10002C9720E030E0A901C701B6010E94BDC695
:102A200081111FC020E030E0A9012C966CAD7DAD76
:102A30008EAD9FAD2C970E94BDC6811112C0E9EDED
:102A4000F9E10AC420E030E0A901C701B6010E9403
:102A5000BDC68823A1F32C961CAE1DAE1EAE1FAEC4
:102A60002C97C701B601905868AF79AF8AAF9BAF7A
:102A70002C968CAD9DADAEADBFAD2C97B0588CAF44
:102A80009DAFAEAFBFAF28AD39AD4AAD5BADCA01AA
:102A9000B9010E9422C74B015C012CAD3DAD4EAD8A
:102AA0005FADCA01B9010E9422C79B01AC01C501FB
:102AB000B4010E94E7CA0E9452CDA0966CAF7DAFD0
:102AC0008EAF9FAFA0972091F7033091F80340910C
:102AD000F9035091FA0328962CAF3DAF4EAF5FAF8C
:102AE0002897A701960128966CAD7DAD8EAD9FAD60
:102AF00028970E94E7CA64966CAF7DAF8EAF9FAFF8
:102B000064974091FB035091FC036091FD03709129
:102B1000FE0360964CAF5DAF6EAF7FAF60972C96B3
:102B20002CAD3DAD4EAD5FAD2C9760966CAD7DADDF
:102B30008EAD9FAD60970E94E7CAA4966CAF7DAF43
:102B40008EAF9FAFA4976091140B7091150B80917D
:102B5000160B9091170B68966CAF7DAF8EAF9FAF41
:102B6000689764962CAD3DAD4EAD5FAD64970E9405
:102B7000E6CA6B017C018091180B9091190BA09112
:102B80001A0BB0911B0B6C968CAF9DAFAEAFBFAF65
:102B90006C97A4962CAD3DAD4EAD5FADA497BC0136
:102BA000CD010E94E6CA4B015C012091FF033091E8
:102BB00000044091010450910204A8962CAF3DAF4F
:102BC0004EAF5FAFA89760911C0B70911D0B809169
:102BD0001E0B90911F0B0E94E6CA24966CAF7DAF2E
:102BE0008EAF9FAF2497A701960168AD79AD8AADEE
:102BF0009BAD0E9422C72B013C01A50194016CAD45
:102C00007DAD8EAD9FAD0E9422C79B01AC01C3017B
:102C1000B2010E94E7CA2B013C01A501940168ADF5
:102C200079AD8AAD9BAD0E9422C74B015C01A70123
:102C300096016CAD7DAD8EAD9FAD0E9422C79B010C
:102C4000AC01C501B4010E94E6CAA30192010E9431
:102C50005ACB6B017C0120E030E0A9010E94BDC687
:102C600087FF0AC02BED3FE049EC50E4C701B601F5
:102C70000E94E7CA6B017C0132E02316310451F453
:102C80002BED3FE049EC50E4C701B6010E94E6CAD3
:102C90006B017C0120E030E0A901C701B6010E9470
:102CA000BDC6811128C068962CAD3DAD4EAD5FAD5F
:102CB000689728966CAD7DAD8EAD9FAD28970E942C
:102CC000BDC6811118C06C962CAD3DAD4EAD5FAD4B
:102CD0006C9760966CAD7DAD8EAD9FAD60970E9498
:102CE000BDC6811108C01BEDC12E1FE0D12E19EC0D
:102CF000E12E10E4F12EA7019601A0966CAD7DADFA
:102D00008EAD9FADA0970E9422C74B015C0120E0D1
:102D100030E0A90124966CAD7DAD8EAD9FAD2497BA
:102D20000E94BDC68823E9F0A5019401C501B40144
:102D30000E9422C74B015C0124962CAD3DAD4EADE7
:102D40005FAD2497CA01B9010E9422C79B01AC0163
:102D5000C501B4010E94E7CA0E9452CD4B015C013B
:102D60000DC020E030E0A901C501B4010E940DCDE5
:102D700087FF04C0B7FAB094B7F8B0942FE632E1F9
:102D800043E85AE3C501B4010E94BDC687FF02C0F3
:102D90000C94052AC501B4010E945CCC0E9430CC81
:102DA0002E967FAF6EAF2E97672B31F441E050E047
:102DB0002E965FAF4EAF2E974090030450900404C0
:102DC00060900504709006042E96AEADBFAD2E97B0
:102DD000BD0180E090E00E94C1C64B015C019B01F7
:102DE000AC01C701B6010E94C3CB28966CAF7DAF82
:102DF0008EAF9FAF2897A501940124966CAD7DAD51
:102E00008EAD9FAD24970E94C3CBA0966CAF7DAFD3
:102E10008EAF9FAFA097A30192016091200B70919C
:102E2000210B8091220B9091230B0E94E6CAA501F1
:102E300094010E94C3CBAC966CAF7DAF8EAF9FAFB9
:102E4000AC9728962CAD3DAD4EAD5FAD2897CA012D
:102E5000B9010E9422C720E030E040E05FE30E9419
:102E600022C79B01AC0160E070E080E89FE30E9414
:102E7000E6CA68966CAF7DAF8EAF9FAF6897A89695
:102E80002CAD3DAD4EAD5FADA89729873A874B87F6
:102E90005C874D865E866F86788A609102027091AB
:102EA0000302072E000C880B990B0E94C3C62091C9
:102EB0004B0230914C0240914D0250914E020E94C3
:102EC00022C72AE037ED43E25CE30E9422C76CABE5
:102ED0007DAB8EAB9FAB0E944BB49B01AC012853E2
:102EE0003F4F4F4F5F4F6C962CAF3DAF4EAF5FAF34
:102EF0006C9748AC59AC6AAC7BAC22242394312C3F
:102F000039E121963FAF21972E964EAD5FAD2E97BA
:102F10004215530509F44DC10E94F8800E944BB43C
:102F2000DC01CB016C962CAD3DAD4EAD5FAD6C9729
:102F3000821B930BA40BB50BB7FD10C00E944BB4C2
:102F40009B01AC0128533F4F4F4F5F4F6C962CAF06
:102F50003DAF4EAF5FAF6C970E94175021963FADCB
:102F60002197315021963FAF2197332309F445C073
:102F70002CAD3DAD4EAD5FAD68966CAD7DAD8EAD0B
:102F80009FAD68970E9422C76B017C019201A3014B
:102F900028966CAD7DAD8EAD9FAD28970E9422C75F
:102FA000A70196010E94E7CA7B018C019201A3014F
:102FB00068966CAD7DAD8EAD9FAD68970E9422C7BF
:102FC0004B015C012CAD3DAD4EAD5FAD28966CADB7
:102FD0007DAD8EAD9FAD28970E9422C79B01AC01AD
:102FE000C501B4010E94E6CA2B013C01C701D8010A
:102FF0008CAF9DAFAEAFBFAF55C0B10180E090E0E8
:103000000E94C1C628962CAD3DAD4EAD5FAD289750
:103010000E9422C74B015C010E94C0CB6B017C0166
:10302000C501B4010E9448CD4B015C01A701960186
:1030300068AD79AD8AAD9BAD0E9422C72B013C01E2
:103040002C962CAD3DAD4EAD5FAD2C97C501B401B6
:103050000E9422C7A30192010E94E7CA2B013C01F2
:10306000A501940168AD79AD8AAD9BAD0E9422C7E0
:103070004B015C012C962CAD3DAD4EAD5FAD2C9758
:10308000C701B6010E9422C79B01AC01C501B40172
:103090000E94E6CA6CAF7DAF8EAF9FAF49E121962B
:1030A0004FAF21979201A30164966CAD7DAD8EADBB
:1030B0009FAD64970E94E7CA69837A838B839C8360
:1030C0002CAD3DAD4EAD5FADA4966CAD7DAD8EAD7E
:1030D0009FADA4970E94E7CA6D837E838F839887F4
:1030E000A0962CAD3DAD4EAD5FADA09769857A85BC
:1030F0008B859C850E94E7CA69877A878B879C8726
:10310000AC962CAD3DAD4EAD5FADAC976D857E857B
:103110008F8598890E94E7CA6D877E878F87988BF5
:1031200080912102882321F0CE0101960E94E24D78
:10313000E090F80A1CA61DA61EA61FA689819A81EA
:10314000AB81BC8188A399A3AAA3BBA38D819E81D7
:10315000AF81B8858CA39DA3AEA3BFA389859A85B3
:10316000AB85BC8588A799A7AAA7BBA7AE01485D78
:103170005F4FBE016C5D7F4FCE0180960E941DA9FE
:10318000BE01645D7F4F6B018E010C5C1F4F9E0181
:10319000235F3F4FAE01485D5F4F68507109CE011C
:1031A00080960E941358882321F07FEF271A370A50
:1031B000ABCEE090F80A18AA19AA1AAA1BAA809105
:1031C000140B9091150BA091160BB091170B88A3BF
:1031D00099A3AAA3BBA38091180B9091190BA0915E
:1031E0001A0BB0911B0B8CA39DA3AEA3BFA3809120
:1031F0001C0B90911D0BA0911E0BB0911F0B88A76B
:1032000099A7AAA7BBA7AE01485D5F4FBE016C5D41
:103210007F4FCE0180960E941DA9CE01C0966C0101
:103220008E010C5C1F4F20E23BE0AE01485D5F4F1A
:10323000BE016C5D7F4F40970E94135880E1E4E12E
:10324000FBE0A7EFB3E001900D928A95E1F70C94B3
:10325000052A0E94D63EF80184918F010F5F1F4F0F
:103260008111F7CFEDE1F2E084918F010F5F1F4FE5
:10327000882311F40C94052A0E94D63EF801F4CF5D
:1032800080E50E94BA3E882379F08091E603909110
:10329000E703009749F04AE050E060E070E00E94E8
:1032A0003CC56B017C0103C0C12CD12C760183E5A8
:1032B0000E94BA3E882361F00E943A3E20E030E04E
:1032C0004AE754E40E9422C70E9430CC6B017C0183
:1032D0000E9436680E944BB4C60ED71EE81EF91E27
:1032E0000E944BB4DC01CB018C199D09AE09BF09CA
:1032F000B7FD02C00C94052A0E941750F1CF80E060
:103300000E94E39A0C94052A83E50E94BA3E882322
:1033100021F10E941A3E182F863070F0E5EEF2E09F
:1033200084918F010F5F1F4F882311F40C94052A9D
:103330000E94D63EF801F4CF833009F44AC130F43C
:10334000813091F1823009F43FC008C0843009F423
:103350009FC1853009F4ACC101C010E00E94969A6B
:10336000811103C0E5ECF2E013C08091751688234B
:1033700019F06BE073E002C06FE073E08DEB92E058
:103380000E94604D8AE00E94D63E0E9457A996C1D5
:1033900084917F019FEFE91AF90A882309F48EC10D
:1033A0000E94D63EF701F4CF0E940AAA10920102B1
:1033B0001092000282EB92E09093360D8093350DCF
:1033C0000E94023F0C94052A809100029091010214
:1033D00097FF0EC0E9E8F2E084918F010F5F1F4F65
:1033E000882311F40C94052A0E94D63EF801F4CFEC
:1033F0000097A1F4809121028093ED0319821A8233
:103400001B821C8218A219A21AA21BA2BE016F5F06
:103410007F4FCE0180960E94B6B127C0815065E0F3
:103420000E94AFCD80FF03C024E0291B922FA5E0AE
:103430009A02F0011124E80FF11D87FDFA95EE0FB5
:10344000FF1FEE0FFF1FE350FA4E8091FF03909194
:103450000004A0910104B091020480839183A283AF
:10346000B3838091ED0380932102809100029091BB
:103470000102893191050CF067C0109221029C0174
:103480002F5F3F4F309301022093000265E00E94BE
:10349000AFCD80FF03C024E0291B922F4091FF0392
:1034A00050910004609101047091020448A359A353
:1034B0006AA37BA319821A821B821C82B4E08B024E
:1034C00090011124F901E558F04F4F01208131811D
:1034D00042815381F4E09F02C0011124BC01615775
:1034E000704F5B01DB016D917D918D919C91FE018F
:1034F00031966F01E12CF12C00EA10E40E94E6B055
:1035000019821A821B821C82B601CE0180960E940B
:10351000B6B1F50180819181A281B3818093F703D7
:103520009093F803A093F903B093FA03F401808118
:103530009181A281B3818093FB039093FC03A093BC
:10354000FD03B093FE03BCC080E090E0A0EAB0E4CD
:103550008093FF0390930004A0930104B0930204AE
:103560000E94D09B0E9436688FEF9FEF90930102DC
:1035700080930002E5E7F2E084918F010F5F1F4F17
:10358000882321F00E94D63EF801F6CF83E992E02D
:103590009A83898304E610E019A308A3BE016F5F34
:1035A0007F4FCE0180960E9469B28AEB92E09A83A7
:1035B000898319A308A3BE016F5F7F4FCE01809658
:1035C0000E9469B281E00E94E39A81E00E94C39A5E
:1035D00077C088E50E94BA3E8823A1F00E940A3E87
:1035E0001FEF160F1530A8F0EEE5F2E084918F0181
:1035F0000F5F1F4F882311F40C94052A0E94D63EBA
:10360000F801F4CF88E50E94D63E0E94AEC20C9429
:10361000052A89E50E94BA3E8823A1F00E940A3E4D
:103620000FEF060F0530A8F0E7E4F2E084918F0178
:103630000F5F1F4F882311F40C94052A0E94D63E79
:10364000F801F4CF89E50E94D63E0E94AEC20C94E8
:10365000052A8AE50E94BA3E882399F00E943A3EE4
:1036600025E0129FF0011124E00FF11DEE0FFF1F66
:10367000EE0FFF1FE350FA4E6083718382839383C2
:1036800035C08AE50E94D63E0E94AEC20C94052A3F
:103690008AE50E94BA3E8823A1F30E943A3E6093D5
:1036A000F9157093FA158093FB159093FC151EC0C5
:1036B00080E00E94C39A0E940AAA18C01230B1F496
:1036C00060910002709101026931710514F069E1A5
:1036D00070E088E392E00E94474D69E170E083E387
:1036E00092E00E94474D8AE00E94D63E0E949E963C
:1036F0000C94052A80914102882311F40C94052A28
:1037000089E40E94BA3EE82E882321F00E940A3EF6
:10371000062F01C000E08AE40E94BA3EF82E8823FA
:1037200021F00E940A3E162F01C010E0EE2011F099
:10373000053020F4FF2081F0153070F0ECEFF2E05E
:1037400084918F010F5F1F4F882311F40C94052A79
:103750000E94D63EF801F4CF0E94CC3EEE2091F0BC
:1037600034E00302F0011124E157F04F8081918190
:10377000A281B3818093140B9093150BA093160B29
:10378000B093170BFF2091F044E01402F0011124D4
:10379000E558F04F80819181A281B3818093180B0D
:1037A0009093190BA0931A0BB0931B0B80E50E940A
:1037B000BA3E882319F00E942B3E03C080E50E9488
:1037C000713E86E40E94BA3E8823D9F00E943A3EB8
:1037D0006B017C0120E030E0A9010E940DCD18169C
:1037E00084F420E030E040E752E4C701B6010E94D3
:1037F000C3CB60934B0270934C0280934D02909325
:103800004E020E94D7530C94052A1092EC030C949C
:10381000052A9093EC030C94052A0E943A3E2B0152
:103820003C01133049F0F6012081318142815381FE
:103830000E94E6CA2B013C01A8ADB9AD2D913D9186
:103840004D915C91C301B2010E94E6CA4B015C013B
:103850002DEB37E346E855EB0E940DCD87FD20C0E8
:103860002DEB37E346E855E3C501B4010E94BDC620
:103870001816B4F01F5FB4E0EB0EF11CE8ADF9AD23
:103880003496F9AFE8AFF4E0CF0ED11C143039F123
:10389000D1018D911D010E94BA3E882359F3BDCFFD
:1038A000133051F4409203045092040460920504D2
:1038B0007092060401E0DECFA5019401F70160815A
:1038C0007181828193810E94E7CAD7016D937D93B4
:1038D0008D939C931397812F0E94279CCBCF00231D
:1038E00009F404CFC0900304D0900404E0900504D0
:1038F000F090060420E030E0A901C701B6010E9463
:10390000E7CA2091EF163091F0164091F1165091D0
:10391000F2160E9422C70E9418CD6093770F709311
:10392000780F8093790F90937A0FC092670FD0929F
:10393000680FE092690FF0926A0F9091450F8091A5
:10394000460F981719F00E94D867D0CE0E943668AB
:1039500080916F00982F927081FF05C080916F0059
:103960008D7F80936F004091770F5091780F609119
:10397000790F70917A0F40936B1550936C1560938B
:103980006D1570936E15992309F4B0CE80916F0078
:10399000826080936F00AACE0E949DB20C94052A8B
:1039A0008091AC169091AD168637910509F4AAC79F
:1039B0000CF0CEC08D34910509F4D1C40CF05AC07E
:1039C0008A31910509F43DC264F58531910509F408
:1039D000F6C1C4F48231910509F432C684319105EF
:1039E00009F4ADC1419711F00C94B4295F988A98FD
:1039F000479880910801817080930601479812983A
:103A00000C94052A8731910509F4E3C10CF4DBC15C
:103A10008831910509F4F3C1499709F4FBC10C946D
:103A2000B4298F31910509F49AC384F48C3191053E
:103A300009F4ADC20CF413C28D31910511F40C944C
:103A4000052A4E9709F4ADC20C94B4298A32910527
:103A500009F438C42CF4809709F435C30C94B429C4
:103A60008B34910509F462C48C34910509F462C465
:103A70000C94B4298B36910509F4B4C50CF042C0FE
:103A80008535910509F40BC6FCF48235910509F4DE
:103A9000D0C584F48135910511F00C94B4290E94AD
:103AA000387E0E94C8A4109208041092070400E017
:103AB00010E0A8C58335910509F4BEC5843591058C
:103AC00009F4BEC50C94B4298836910509F44BC499
:103AD0007CF48C35910511F00C94B429FFE4CF2EC1
:103AE000F2E0DF2EA3EEEA2EA6E1FA2E10E0F0C5FA
:103AF0008936910509F4FAC48A36910509F456C548
:103B00000C94B4298037910509F4BFC484F48D3630
:103B1000910509F42BC50CF4B5C48E36910509F452
:103B20004BC48F36910509F45AC40C94B4298237DA
:103B3000910509F44DC60CF4AFC48337910509F41F
:103B4000FBC08537910511F40C94052A0C94B42917
:103B50008E3221E0920711F40C94F0270CF06EC025
:103B60008B3C910509F48CC7ACF58C38910509F4B0
:103B700000C58CF48837910509F413C70CF40EC7FF
:103B80008937910511F00C94B4291092A20B109270
:103B9000A10B0C94052A8E3B910509F404C534F45D
:103BA0008B39910509F4BDC40C94B429883C910566
:103BB00009F4FDC6893C910511F00C94B4297FE409
:103BC000E72E72E0F72E03EC16E1E3EDCE2EE6E1F0
:103BD000DE2E3DC78C3D910511F40C948426A4F48F
:103BE0008D3C910509F4DDC70CF466C78E3C910548
:103BF00011F40C945E26833D910511F00C94B429C8
:103C00000E94048E0C94052A823E910511F40C94B6
:103C1000FE263CF48D3D910511F40C9491260C94F4
:103C2000B4298C3241E0940711F40C9427278D328B
:103C3000914011F40C9450270C94B429853F61E015
:103C4000960711F40C94DD28E4F58A39A1E09A076F
:103C500009F41FC4BCF48033E1E09E0711F40C9416
:103C6000472814F40C944428833621E0920709F481
:103C70005FC08039914011F00C94B4290E943668DD
:103C80000C94052A853A41E0940711F40C94DA2843
:103C90004CF4843A914011F00C94B4290E94C886E7
:103CA0000C94052A8C3A71E0970711F40C94812644
:103CB000843F914011F00C94B4290E947D6E0C94C5
:103CC000052A8A39B2E09B0711F40C941C29B4F43C
:103CD000873FF1E09F0711F40C94E32814F40C944F
:103CE000E028883F31E0930711F40C94EF288C30E2
:103CF000924011F40C9413290C94B4298B3853E09E
:103D0000950711F40C94052A3CF48438934011F47F
:103D10000C9449290C94B429803AA3E09A0709F439
:103D200011C2873E934011F40C94A1290C94B4293C
:103D3000E9EDF9E10C94C728E3EFF4E088C5EAE285
:103D4000F3E084918F010F5F1F4F882321F00E94C1
:103D5000D63EF801F6CF1092411284EF9FE00E9408
:103D60007B918BE1E4EFFFE0DE01159601900D926F
:103D70008A95E1F78091F20F9091F30F9C838B83EA
:103D800085EE92E09A83898340E050E0BE016F5F48
:103D90007F4F80E090E00E94B277CE0101960E94B2
:103DA000AD4FEBE1F3E084918F010F5F1F4F88234C
:103DB00011F40C94052A0E94D63EF801F4CF0E941B
:103DC00081750C94052A1092C30F1092C40F0C94A5
:103DD000052AE091AA16F091AB168081882329F07C
:103DE000803209F410823196F8CF40E061E0809192
:103DF000AA169091AB160E94B3B40C94052A809138
:103E0000C40F882319F081E08093C30F0E94017EC4
:103E10000C94052A1092C30F80917315813011F014
:103E20000C94052A82E0809373150E944BB4609332
:103E30006F157093701580937115909372150C9493
:103E4000052A8091C40F882311F40C94052A83E578
:103E50000E94BA3E81110C940F2A0C94052A83E427
:103E60000E94713E882309F450C0E8E6F3E0849193
:103E70008F010F5F1F4F882321F00E94D63EF8016B
:103E8000F6CF80918F11811103C0EBE3F3E012C0F4
:103E9000BE016F5F7F4F8CE891E10E9443908E01DD
:103EA0000F5F1F4FF80181918F01882349F10E9414
:103EB000D63EF8CF84918F010F5F1F4F882301F109
:103EC0000E94D63EF801F6CFB6EECB2EB3E0DB2E45
:103ED000E12CF12C20E080918B0B90E00E2C02C0A5
:103EE000959587950A94E2F780FDA9C29FEFE91A9C
:103EF000F90AA2E0CA0ED11CB5E0EB16F10459F79D
:103F00008AE00E94D63E0C94052A8091C40F882333
:103F100039F08091C30F882319F0E5E4F3E003C082
:103F2000E7E5F3E028C084918F010F5F1F4F8823DE
:103F300021F00E94D63EF801F6CF60913D127091BB
:103F40003E1280913F12909140124AE00E94F2414D
:103F50008FE20E94D63E6091391270913A128091A0
:103F60003B1290913C124AE00E94F2418AE00E948A
:103F7000D63E0C94052A84918F010F5F1F4F882332
:103F800011F40C94052A0E94D63EF801F4CF40E0CB
:103F900060E08091AA169091AB160E94B3B40C9485
:103FA000052A8091C40F882311F40C94052A8CE80B
:103FB00091E10E9494AE8CE891E10E941E901092D3
:103FC000C20F1092C10F8091C40F882311F40C947A
:103FD000052A0091AA161091AB160E94A577B80188
:103FE000CE0180960E94B9798C01892B11F40C9432
:103FF000052A68A179A16115710511F06C5F7F4FE9
:1040000019821C8222E0A801CE0101960E94B1957E
:10401000811102C0F12C14C0CE0101960E941377C9
:104020008823C1F361E0CE0101960E94279000979A
:1040300089F325EEDC012C931C820E943DACF82E06
:10404000CE0101960E94C63EF11003C0E5E8F3E000
:1040500022C0E7E7F3E084917F01BFEFEB1AFB0A90
:10406000882321F00E94D63EF701F5CFF801819117
:104070008F01882319F00E94D63EF8CF8AE00E9473
:10408000D63E10923D1210923E1210923F121092A4
:1040900040120C94052A84917F012FEFE21AF20A54
:1040A000882321F00E94D63EF701F5CFD8018D91EB
:1040B0008D01882319F00E94D63EF8CF8EE20E942F
:1040C000D63E0C94052A8091C30F81110E94366858
:1040D0008091C40F882311F40C94052A80E50E9476
:1040E000BA3E882319F00E942B3E03C080E50E944F
:1040F000713E182F482F61E08091AA169091AB165F
:104100000E94B3B483E50E94BA3E882381F00E94E6
:104110000A3EAB01BC0140933D1250933E126093A6
:104120003F12709340128CE891E10E94348F80918D
:10413000C40F882319F081E08093C30F11110C94F0
:10414000052A64CE8091AA169091AB1621E02093A7
:10415000C20F40E060E00E94B3B40C94052A0E94B4
:10416000B27D7B018C0120E831E541E050E00E9406
:10417000ABCAC9016DE671E00E94BCCD4B015C0188
:10418000C801B70120E13EE040E050E00E94ABCA28
:10419000CA01B90128E130E040E050E00E94ABCA1A
:1041A000762E672EC62ED72E8CE3282E312C412C4E
:1041B000512CC801B701A20191010E94ABCAF62E91
:1041C000E72ECA01B901A20191010E94ABCACB013D
:1041D0008E010F5F1F4F81149104D1F0EF92FF9277
:1041E0007F936F936F927F92BF92AF929F928F92C5
:1041F00085EC93E09F938F931F930F930E948FC63C
:104200000FB6F894DEBF0FBECDBFEEEEF9E145C0AC
:10421000A114B10489F0EF92FF927F936F936F9294
:104220007F92BF92AF9285EB93E09F938F931F9302
:104230000F930E948FC6E4CFCD2879F0EF92FF92C2
:104240007F936F936F927F9289EA93E09F938F930E
:104250001F930F930E948FC6D3CF892B69F0EF92E3
:10426000FF927F936F9381EA93E09F938F931F93C5
:104270000F930E948FC6C4CFEF92FF928DE993E017
:104280009F938F931F930F930E948FC60F900F9051
:104290000F900F900F900F90B8CF84917F017FEF18
:1042A000E71AF70A882321F00E94D63EF701F5CFDE
:1042B000B80189ED93E00E94604D8AE00E94D63EED
:1042C0000C94052A83E50E94BA3E882311F40C94CD
:1042D000052A0E941A3EE82E80E50E94BA3E8823F5
:1042E00039F00E941A3E182F87FF03C00C94052A4C
:1042F0001DE089E40E94BA3E882341F00E942B3ED3
:1043000081110C947D2AEDE0F6E00BC089E40E9457
:10431000713EF6CF319686E0ED33F80711F40C9438
:104320007D2A84911813F6CF0C94522A0E94017EA4
:104330000C94052A80917315813011F00C94052A94
:1043400082E0809373150E944BB460936F15709355
:10435000701580937115909372150C94052A0E9424
:10436000237E0C94052A88E690E00E94679C8111C8
:104370000C94052A80918B0B83FF02C00C94052AB4
:1043800083E50E94BA3E882399F00E943A3E0E943B
:104390002BCCCB010E941A740E943A3E20E030E000
:1043A00044EB52E40E94BDC6181614F00E94237E0E
:1043B0000E94AB4D0C94052A8EE40E94BA3E8823DD
:1043C00011F40C94052A0E940A3E6093881670939B
:1043D000891680938A1690938B160C94052A83E590
:1043E0000E94713E882359F083E50E94BA3E8823DB
:1043F00019F00E941A3E01C080E080938B0BEEEE14
:10440000F9E184918F010F5F1F4F811103C0E4EF29
:10441000F3E004C00E94D63EF801F3CF84918F01EF
:104420000F5F1F4F882321F00E94D63EF801F6CF80
:1044300080918B0B811148CDE0EFF3E018C0BB24D5
:10444000B394B20E222319F08CE20E94D63EF601FC
:1044500085919491FC0184918F010F5F1F4F8823F8
:1044600021F00E94D63EF801F6CF2B2D3FCD84914E
:104470008F010F5F1F4F882309F442CD0E94D63E63
:10448000F801F5CF10924002C0C78BEF93E00E9475
:10449000D04F0E948F88B9C783E50E94BA3E811130
:1044A00003C0EEEEF9E10BC00E941A3E8D3318F402
:1044B00080932202AAC78CE380932202A6C784912C
:1044C0008F010F5F1F4F882321F00E94D63EF80115
:1044D000F6CF4091220250E060E070E084E094E08A
:1044E0000E940D4D8AE00E94D63E8FC789E690E07B
:1044F0000E94679C811111C0EBE0F4E084918F0170
:104500000F5F1F4F882321F00E94D63EF801F6CF9F
:104510000E943A7B8AE00E94D63E1092F90A0C94DF
:10452000922A83E50E94BA3E882309F46EC70E944E
:104530001A3E182F8D3308F01CE31093060B0E94CF
:104540004BB46B017C01212F30E0A8EEB3E00E9458
:10455000D7CAC60ED71EE81EF91EC092020BD09213
:10456000030BE092040BF092050B4FC70E94A99C2D
:104570004CC780918B0B83FD48C783E50E94BA3EF0
:10458000882309F442C70E943A3E0E942BCC6E3623
:10459000710514F06EE670E070930A0460930904EC
:1045A0000E94F47B32C70E9468972FC780E50E9463
:1045B000BA3E811106C083E50E94BA3E882359F0B5
:1045C00005C00E941A3E811120C7F5CF0E940A3E05
:1045D0006F3F710510F06FEF70E070930804609307
:1045E000070413C780E50E94BA3E811105C01092EE
:1045F00008041092070409C70E940A3E672B09F0BD
:1046000004C7F5CF62E370E080E090E00E9413B44D
:104610000E94F8800F5F1F4F0331110599F762E385
:1046200070E080E090E00E9413B40E94F88094D77C
:10463000ECC61092EB03E9C681E08093EB03E5C67C
:1046400083E50E94BA3E882399F00E943A3E20E01A
:1046500030E04AE754E40E9422C70E9430CC6093C5
:104660002302709324028093250290932602CDC6E4
:1046700088E50E94713E8111E3C689E50E94713E82
:104680008111DEC68AE50E94713E8111D9C685E49A
:104690000E94713E8111D4C60E94C8A4B6C683E5AB
:1046A0000E94713E882309F4B0C60E943A3E20E081
:1046B00030E04AE754E40E9422C70E9430CC609365
:1046C000FE0A7093FF0A8093000B9093010B9DC626
:1046D000F60181916F010E94713E882309F46EC03A
:1046E000133009F063C00E943A3E4B015C0120E0A8
:1046F00030E040EA51E40E94BDC687FF4EC0A501EC
:1047000094016091EF167091F0168091F1169091DE
:10471000F2160E94C3CB2B013C019B01AC016091BE
:104720005A0B70915B0B80915C0B90915D0B0E941A
:1047300022C760935A0B70935B0B80935C0B909332
:104740005D0BA301920160917A0B70917B0B8091BC
:104750007C0B90917D0B0E9422C760937A0B709323
:104760007B0B80937C0B90937D0B6091BF167091B7
:10477000C0168091C1169091C2160E94C1C6A301B5
:1047800092010E9422C70E9430CC6093BF167093A2
:10479000C0168093C1169093C2168092EF16909225
:1047A000F016A092F116B092F21608C00E943A3E9E
:1047B000D7016D937D938D939C9313971F5FB4E006
:1047C000EB0EF11C143009F083CF0E94ACBA1DC669
:1047D0000E94366883E50E94BA3E882311F40C9447
:1047E000761B0E940A3E6230710511F00C94761B14
:1047F0000E94B3578BE50E94D63E6091EC0A7091FF
:10480000ED0A8091EE0A9091EF0A42E00E94774211
:104810004091F00A5091F10A6091F20A7091F30A06
:1048200081E194E00E942A4D4091F40A5091F50AEA
:104830006091F60A7091F70A8EE094E00E942A4D8A
:104840008DE50E94D63E8AE00E94D63EDEC5849168
:104850008F010F5F1F4F882321F00E94D63EF80181
:10486000F6CF60E083EE94E00E94E28E61E08CED92
:1048700094E00E94E28E61E081ED94E00E94E28E7D
:1048800061E081EC94E00E94E28E60E088EB94E0CD
:104890000E94E28E61E08EEA94E00E94E28E60E087
:1048A00084EA94E00E94E28E60E08CE994E00E9449
:1048B000E28E61E08EE894E00E94E28E60E080E8A3
:1048C00094E00E94E28E60E081E794E00E94E28E34
:1048D00060E083E694E00E94E28E60E08DE494E084
:1048E0000E94E28E60E08CE394E00E94E28E60E041
:1048F00087E294E00E94E28E61E084E194E00E940D
:10490000E28E83C50091AA161091AB1683E0D12CDC
:1049100040E08150E1F0F8019081292F2B7F213474
:10492000C1F721812133A9F7913421F0953421F485
:1049300041E002C0DD24D39498012E5F3F4F8901EE
:104940002F5F3F4FD8019C919032C9F3E2CF4423AF
:1049500069F0EEEEF9E184917F01BFEFEB1AFB0AFB
:10496000882321F00E94D63EF701F5CFDD2069F0C3
:10497000E9EBF5E084917F012FEFE21AF20A882338
:1049800021F00E94D63EF701F5CFD8018D918D011F
:10499000882309F4B5CA0E94D63EF7CF0E94A2AA86
:1049A00034C581E08093A20B8093A10B2EC588ECC7
:1049B00090E00E94679C811128C584E40E94713EAA
:1049C000882309F441C00E943A3E6B017C0111E04A
:1049D00020E030E0A9010E94BDC6811101C010E0B5
:1049E0001093611620E030E0A901C701B6010E94D2
:1049F000BDC6882349F10E943A3EE0919615B4E085
:104A0000EB9FF0011124EA59F94E60837183828390
:104A1000938320E030E0A9016091661670916716DB
:104A200080916816909169160E94BDC681110CC0D4
:104A300080E090E0A0EEBFE3809366169093671647
:104A4000A0936816B09369160E9406A5DEC4F7010C
:104A500081917F010E94713E882351F00E943A3E6D
:104A60000E9430CCD8016D937D938D939C931397C6
:104A70000C5F1F4FC016D10651F70E943BB9C5C449
:104A80006FE4E62E62E0F62E0EE61BE0F701819160
:104A90007F010E94713E882341F00E943A3ED80176
:104AA0006D937D938D939C9313970C5F1F4FBBE089
:104AB0000E371B0759F7A9C483E50E94BA3E882325
:104AC000A1F00E943A3E6093660B7093670B80934F
:104AD000680B9093690B6093620B7093630B8093E8
:104AE000640B9093650B10E001C011E080E50E941B
:104AF000BA3E882359F00E943A3E6093660B709349
:104B0000670B8093680B9093690B10E082E50E941D
:104B1000BA3E882359F00E943A3E60936A0B709324
:104B20006B0B80936C0B90936D0B10E084E50E94EF
:104B3000BA3E882359F00E943A3E6093620B70930C
:104B4000630B8093640B9093650B5FC4112309F48E
:104B50005CC44091660B5091670B6091680B70913B
:104B6000690B83EC95E00E942A4D40916A0B5091AD
:104B70006B0B60916C0B70916D0B80EC95E00E945B
:104B80002A4D4091620B5091630B6091640B7091C0
:104B9000650B8DEB95E00E942A4D8AE00E94D63E7F
:104BA00034C481E50E94713E8823C1F08091E60300
:104BB0009091E703009739F04AE050E060E070E040
:104BC0000E943CC503C060E070E0CB0160937E0BA7
:104BD00070937F0B8093800B9093810B83E50E94F1
:104BE000713E882351F00E943A3E6093860B709389
:104BF000870B8093880B9093890B84E50E94713E0C
:104C0000882351F00E943A3E6093820B7093830B8D
:104C10008093840B9093850B88E50E94713E8823D6
:104C200051F00E943A3E60934E0B70934F0B80936D
:104C3000500B9093510B89E50E94713E882351F0EF
:104C40000E943A3E6093520B7093530B8093540B27
:104C50009093550B8AE50E94713E8823F1F00E94E3
:104C60003A3E6093560B7093570B8093580B90937A
:104C7000590B2DEC3CEC4CEC5DE30E94BDC61816C4
:104C800064F0E3EDF5E084918F010F5F1F4F8823FF
:104C900021F00E94D63EF801F6CF85E40E94713ED5
:104CA000882309F4B2C30E943A3E60935A0B709372
:104CB0005B0B80935C0B90935D0BA7C34FE4C42EFA
:104CC00042E0D42E53EAE52E5BE0F52E10E0F6012B
:104CD00081916F010E94713E882359F00E943A3EF3
:104CE000D7016D937D938D939C931397812F0E9491
:104CF000279C1F5FB4E0EB0EF11C133041F70C94BE
:104D0000761B0E94848481C383E50E94BA3E882377
:104D100009F47BC30E940A3E70930302609302026F
:104D200074C38DED90E00E94679C81116EC383E592
:104D30000E94BA3E811103C0EEEEF9E139C0009144
:104D4000961510E00E940A3E000F111FF801E75B64
:104D5000FD4F718360838091961590E07C01EE0C8D
:104D6000FF1CEE0CFF1C87010D5C1D4F880F991F67
:104D7000FC01E75BFD4F60817181072E000C880B01
:104D8000990B0E94C3C62AE037ED43E25CE30E9420
:104D900022C7F701EE59F94E2081318142815381BA
:104DA0000E9422C7F80160837183828393832DC39D
:104DB00084918F010F5F1F4F882321F00E94D63E00
:104DC000F801F6CF85E40E94D63E80919615805D6D
:104DD0000E94D63EE0919615F0E0EE0FFF1FE75BD4
:104DE000FD4F6081718185E096E00E94474D85E22C
:104DF0000E94D63E8AE00E94D63E07C380E50E940C
:104E0000713E882309F401C30E940A3E6B017C01B4
:104E100083E50E94BA3E882321F00E940A3E8B015E
:104E200002C00FEF1FEFC8010196039708F0EDC213
:104E3000D7FCEBC28C2DEDE0F6E09491891709F4D4
:104E400031C3319626E0ED33F207B9F72EC383E57F
:104E50000E94BA3E882319F00E940A3E02C064E014
:104E600071E079A368A380E50E94BA3E882339F0F7
:104E70000E940A3E693833E1730730F402C068EEDD
:104E800073E07A83698304C088E893E19A83898315
:104E9000BE01605E7F4FCE0101960E9469B2B5C22D
:104EA00085E40E94BA3E811110C080E50E94713EE7
:104EB000882391F00E943A3E609384157093851583
:104EC000809386159093871507C00E941A3E882309
:104ED00061F3E9EDF9E171C089E40E94713E882334
:104EE00081F00E943A3E2CEA35EC47E25EE30E94F4
:104EF00022C76093801570938115809382159093DB
:104F0000831584E40E94713E882381F00E943A3E1A
:104F10002CEA35EC47E25EE30E94C3CB6093881530
:104F20007093891580938A1590938B15EEEEF9E1B5
:104F300084918F010F5F1F4F882321F00E94D63E7E
:104F4000F801F6CF40918415509185156091861532
:104F50007091871585E496E00E942A4D2CEA35EC85
:104F600047E25EE360918015709181158091821512
:104F7000909183150E94C3CBAB01BC0181E496E004
:104F80000E942A4D2CEA35EC47E25EE360918815D9
:104F90007091891580918A1590918B150E9422C776
:104FA000AB01BC018DE396E00E942A4D8AE00E948D
:104FB000D63E2BC20E94D63EF80184918F010F5F2E
:104FC0001F4F8111F7CFE9E4F6E084918F010F5F65
:104FD0001F4F882309F419C20E94D63EF801F5CF6D
:104FE00083E50E94713E182F882371F00E943A3E9B
:104FF0000E942BCC709338026093370221E0672B1C
:1050000009F020E020938A0B80E50E94713E8823FE
:1050100059F02091370230913802232B11F00E9471
:105020002B3E80938A0BF1C11111EFC1EEEEF9E135
:1050300084918F010F5F1F4F882321F00E94D63E7D
:10504000F801F6CF80918A0B882319F063E173E0B1
:1050500002C066E173E080E796E00E94604D6091D7
:105060003702709138028FE596E00E94474DEBE5DC
:10507000F6E084918F010F5F1F4F882309F4C5C1AB
:105080000E94D63EF801F5CF0E94CC88BEC180E5D3
:105090000E94713E882351F00E943A3E60937C1535
:1050A00070937D1580937E1590937F1589E40E94FF
:1050B000713E882381F00E943A3E2CEA35EC47E2AB
:1050C0005EE30E9422C760937815709379158093F0
:1050D0007A1590937B1584E40E94713E882381F0B9
:1050E0000E943A3E2CEA35EC47E25EE30E94C3CBD5
:1050F000609374157093751580937615909377155A
:10510000EEEEF9E184918F010F5F1F4F882321F0AC
:105110000E94D63EF801F6CF40917C1550917D1546
:1051200060917E1570917F158BE896E00E942A4D64
:105130002CEA35EC47E25EE36091781570917915C1
:1051400080917A1590917B150E94C3CBAB01BC0175
:1051500087E896E00E942A4D2CEA35EC47E25EE3B0
:1051600060917415709175158091761590917715F1
:105170000E9422C7AB01BC0183E896E00E942A4D41
:105180008AE00E94D63E41C10E94D63EF801849139
:105190008F010F5F1F4F8111F7CFEFE8F6E0849189
:1051A0008F010F5F1F4F882309F42FC10E94D63E45
:1051B000F801F5CF0E94DD8528C10E94716E25C1DE
:1051C0000E943AA322C183E50E94713E882321F008
:1051D0000E942B3E91E089270E94A69E16C181E085
:1051E0008093920B0E9467681092920B882309F4B7
:1051F0000CC1EEEEF9E184918F010F5F1F4F811119
:1052000003C0EEE9F6E004C00E94D63EF801F3CFF9
:1052100084918F010F5F1F4F882309F4F6C00E940D
:10522000D63EF801F5CF8091C30F882309F4EDC075
:1052300081E08093C60FE9C08AE50E94BA3E8111E1
:1052400003C0ECEAF6E00BC00E943A3E6093F5150D
:105250007093F6158093F7159093F815D6C0849146
:105260008F010F5F1F4F882321F00E94D63EF80167
:10527000F6CF4091F5155091F6156091F7157091A4
:10528000F81589EA96E00E942A4D8AE00E94D63EEF
:10529000BCC08BE40E94BA3E811103C0EEEEF9E17E
:1052A00036C08BE40E94BA3E8823C1F00E943A3E89
:1052B0006B017C0120E030E0A9010E940DCD87FD4B
:1052C0000AC020E030E040E251E4C701B6010E948C
:1052D000BDC6181634F4EBECF6E00EC0C12CD12C90
:1052E00076010E943668C0925E0BD0925F0BE0920E
:1052F000600BF092610B89C084918F010F5F1F4F8B
:10530000882309F482C00E94D63EF801F5CF84912B
:105310008F010F5F1F4F882321F00E94D63EF801B6
:10532000F6CF40915E0B50915F0B6091600B7091D6
:10533000610B8AEE96E00E942A4D8AE00E94D63EDA
:1053400064C081E08093410283E50E94BA3E8823D5
:1053500039F00E942B3E811158C00E94EC5755C075
:1053600083E50E94713EF7CF0E949DB24EC0F0903F
:10537000AC160E9436681091751680E00E94C39AA0
:10538000FF2029F1EEEEF9E184918F010F5F1F4FAD
:10539000882321F00E94D63EF801F6CF84E50E94D2
:1053A000D63E6F2D70E080E090E04AE00E94F2412E
:1053B00080E20E94D63EE7E0F7E084918F010F5F24
:1053C0001F4F882311F10E94D63EF801F6CF1092AC
:1053D000F80A812F0E94C39AEEEEF9E184918F01C1
:1053E0000F5F1F4F882321F00E94D63EF801F6CFB1
:1053F0006091F80A70E085EF96E00E94474D8AE0E0
:105400000E94D63E02C00E949DB21092F90A0E94EC
:10541000CF5788C00E9443990E94D753F6CF0E946D
:105420000A3EAB01BC0140933D1250933E12609383
:105430003F12709340128CE891E10E94348FE5CFC7
:105440000E94366888E50E94713E882331F05F9A99
:105450008091F6038E7F8093F60389E50E94713E6A
:10546000882339F08A9A479A8091F6038D7F80933A
:10547000F6038AE50E94713E882361F0809108015D
:105480008095817080930601479A8091F6038B7F07
:105490008093F60385E40E94713E882309F4B5CF1A
:1054A000129AB3CF0E9493C2B0CF0E943668BC2C30
:1054B00060E08C2D0E9410B30F3F4FEF140759F49A
:1054C0008C2D0E94BAB231E020E0892B09F030E047
:1054D000032F122F05C00130110561F401E010E027
:1054E0008B2D0E94BAB28017910709F48ECF0E94CB
:1054F0001750F6CF00E010E0F3CF61E0812F0E945B
:1055000010B36E2D812F0E94E2B2F12CB701812FD2
:105510000E944CB3193009F078CFF0920804E09261
:10552000070473CFC559DF4F0FB6F894DEBF0FBE27
:10553000CDBFDF91CF911F910F91FF90EF90DF9042
:10554000CF90BF90AF909F908F907F906F905F9023
:105550004F903F902F9008952F923F924F925F92DD
:105560006F927F928F929F92AF92BF92CF92DF9273
:10557000EF92FF920F931F93CF93DF93CDB7DEB7D8
:105580006F970FB6F894DEBF0FBECDBFC090110469
:10559000D0901204E0901304F090140420E030E066
:1055A00040EA50E4C701B6010E94BDC687FD19C19B
:1055B00020E030E041E953E4C701B6010E940DCD7F
:1055C00018160CF40EC11092E0131092DF138091A4
:1055D00009014091DE13042E000C550B817021E06F
:1055E000822790E04817590709F433C080910901D8
:1055F000817028272093DE1381111BC00E948175C2
:10560000E6E0FCE084918F01882351F0082E000C25
:10561000990B0E947C750F5F1F4FF8018491F4CFA6
:105620008DE090E00E947C758AE090E00E947C759D
:1056300010C0EAE0FCE084918F01882389F3082EF2
:10564000000C990B0E947C750F5F1F4FF80184912D
:10565000F4CF8091D113833009F44CC02CF488230B
:1056600051F08130D9F072C0843009F43EC08530E9
:1056700009F44DC06BC08091C30F882309F466C044
:1056800081E08093D1130E944BB46093D513709343
:10569000D6138093D7139093D81358C08091C30F1B
:1056A000811154C080918F11882321F082E0809372
:1056B000D1134CC01092D113E2E0FCE084918F0131
:1056C000882351F0082E000C990B0E947C750F5F07
:1056D0001F4FF8018491F4CF8DE090E00E947C751B
:1056E0008AE090E00E947C7531C080911E1488236E
:1056F000E9F22CC08091C30F811128C08091450F21
:105700009091460F891B8F7009F496C01FC080913D
:10571000C30F81111BC08091450F9091460F891BCB
:105720008F7009F4ABC012C08DE090E00E947C75D0
:105730008AE090E00E947C751092D11382EE9BE08B
:105740009093360D8093350D0E94023F8091C613D1
:105750009091C71303974CF57AE7272E78E0372E00
:10576000E0E68E2EEAEE9E2EA12CB12C8CE295E185
:105770000E94E33918161906C4F48091C61390915B
:10578000C713049794F48CE295E10E94A7398093A3
:10579000CC13E091CD13F091CE138A3019F08D30F7
:1057A00009F07DC0309709F083C08091C6139091B5
:1057B000C713009711F40C94183901979093C713ED
:1057C0008093C6138091C8139091C913019664E029
:1057D00070E00E94D0CD9093C9138093C8130C94AD
:1057E00018398091DF139091E0138136FAEE9F070C
:1057F000E8F01092E0131092DF13EEE0FCE08491E9
:105800008F01882351F0082E000C990B0E947C75A3
:105810000F5F1F4FF8018491F4CF8DE090E00E945C
:105820007C758AE090E00E947C75D1CE01969093C1
:10583000E0138093DF13CBCE8EEE9BE09093360D7A
:105840008093350D0E94023F80911E14882311F031
:1058500082E001C084E08093D113EAEEFBE0849102
:105860008F01882309F438CF082E000C990B0E9471
:105870007C750F5F1F4FF8018491F3CFE6EEFBE0DC
:1058800084918F01882309F44FCF082E000C990BC7
:105890000E947C750F5F1F4FF8018491F3CF8A330C
:1058A00009F480CFEF35F10514F40C94B1367ACFBA
:1058B0008091CA139091CB1320E6289F7001299FF5
:1058C000F00C112487010A5B1D4EE00FF11F1082BE
:1058D00061E470E0C8010E9453CE009711F40C946B
:1058E00095369093D0138093CF13801B910B8E0D20
:1058F0009F1D60E070E0895B9D4E0E94BEC20E94C9
:105900002BCCCB01770FAA0BBB0B8232910510F089
:105910000C949536FC018827EE58FF4F8F4F0C945E
:10592000FFCDEDEDFBE084918F01882351F0082E2F
:10593000000C990B0E947C750F5F1F4FF80184913A
:10594000F4CF20E030E040E05FE36091110470911B
:10595000120480911304909114041EC0E8EDFBE042
:1059600084918F01882351F0082E000C990B0E941E
:105970007C750F5F1F4FF8018491F4CF60910F0485
:1059800070911004072E000C880B990B0E94C3C65F
:1059900020E030E040E05FE30E94E7CA0E942BCCA9
:1059A000CB010E9412430E94EBB68DE090E00E9472
:1059B0007C758AE090E00E947C750C949536E3ED4E
:1059C000FBE084918F01882351F0082E000C990B85
:1059D0000E947C750F5F1F4FF8018491F4CF20E087
:1059E00030E040E05FE360910B0470910C04809123
:1059F0000D0490910E04D0CFEEECFBE084918F016A
:105A0000882351F0082E000C990B0E947C750F5FC3
:105A10001F4FF8018491F4CF6091090470910A043A
:105A2000B1CF209107043091080444E6429FC001A1
:105A3000439F900D11246FEF70E00E94D0CD8B0139
:105A40006536710510F004E610E0E9ECFBE08491A6
:105A50007F01882359F0082E000C990B0E947C7559
:105A6000FFEFEF1AFF0AF7018491F3CFB80180E04E
:105A700090E082C6E5ECFBE084918F01882351F031
:105A8000082E000C990B0E947C750F5F1F4FF801C8
:105A90008491F4CF80E290E00E947C75E1ECFBE021
:105AA00084918F01882351F0082E000C990B0E94DD
:105AB0007C750F5F1F4FF8018491F4CF6091F7035D
:105AC0007091F8038091F9039091FA030E94ECB66B
:105AD00080E290E00E947C75EDEBFBE084918F0109
:105AE000882351F0082E000C990B0E947C750F5FE3
:105AF0001F4FF8018491F4CF6091FB037091FC0378
:105B00008091FD039091FE030E94ECB680E290E04C
:105B10000E947C75E9EBFBE084918F01882351F0B2
:105B2000082E000C990B0E947C750F5F1F4FF80127
:105B30008491F4CF6091FF0370910004809101047F
:105B4000909102040E94ECB680E290E0E2C4809161
:105B5000C30F882309F450C0E4EBFBE084918F016C
:105B6000882351F0082E000C990B0E947C750F5F62
:105B70001F4FF8018491F4CF8091C40F882359F10D
:105B800080918F11882329F18091391290913A12D6
:105B9000A0913B12B0913C120097A105B105C1F054
:105BA000BC01CD016D597F4F8F4F9F4F24E630E0F0
:105BB00040E050E00E94ABCA60913D1270913E12ED
:105BC00080913F12909140120E94ABCA822F01C077
:105BD00080E090E0E6CEE0EBFBE084918F0188234B
:105BE00009F4E3CE082E000C990B0E947C750F5F20
:105BF0001F4FF8018491F3CFE8EAFBE084918F0115
:105C0000882309F4D2CE082E000C990B0E947C75D3
:105C10000F5F1F4FF8018491F3CFE3EAFBE084911B
:105C20008F01882351F0082E000C990B0E947C757F
:105C30000F5F1F4FF8018491F4CF8091D51390919D
:105C4000D613A091D713B091D813892B8A2B8B2B05
:105C500009F477C00E944BB4A50194010E94ABCA1D
:105C600069017A016091D5137091D6138091D71391
:105C70009091D813A50194010E94ABCA8601021B22
:105C8000130BC8016CE370E00E94BCCDCB019927D7
:105C9000EAE0F0E0BF010E94D0CD282FCB01BF0188
:105CA0000E94D0CD805D8093EE03205D2093EF03B2
:105CB0001092F0038EEE93E00E94EBB680E290E04B
:105CC0000E947C75E1EAFBE084917F01882359F012
:105CD000082E000C990B0E947C75FFEFEF1AFF0A4B
:105CE000F7018491F3CF80E290E00E947C75C801B7
:105CF0006CE370E00E94BCCD6AE070E00E94D0CD01
:105D0000605D6093EE03805D8093EF031092F0037B
:105D10008EEE93E00E94EBB680E290E00E947C75EC
:105D2000EFE9FBE084918F01882309F43ECE082E31
:105D3000000C990B0E947C750F5F1F4FF801849136
:105D4000F3CF80E290E00E947C75E7E9FBE084916C
:105D50008F01882309F429CE082E000C990B0E948C
:105D60007C750F5F1F4FF8018491F3CF1092FF13E2
:105D70008091090180FF11C0E3E9FBE084918F016C
:105D8000882309F412CE082E000C990B0E947C7512
:105D90000F5F1F4FF8018491F3CF83E50E9487B610
:105DA000882341F00E94A2B60E9430CC7093D41395
:105DB0006093D313EFE8FBE084918F01882351F0C7
:105DC000082E000C990B0E947C750F5F1F4FF80185
:105DD0008491F4CF8DE090E00E947C758AE090E0A1
:105DE0000E947C7580911D14882309F484C18091E0
:105DF000D3139091D413009741F0049709F02FC367
:105E0000EAE2F9E084918F01C1C0E7EBF9E0849107
:105E10008F01882351F0082E000C990B0E947C758D
:105E20000F5F1F4FF8018491F4CF8DE090E00E9446
:105E30007C758AE090E00E947C75E0EBF9E084914B
:105E40008F01882351F0082E000C990B0E947C755D
:105E50000F5F1F4FF8018491F4CF8DE090E00E9416
:105E60007C758AE090E00E947C75E9E9F9E0849114
:105E70008F01882351F0082E000C990B0E947C752D
:105E80000F5F1F4FF8018491F4CF8DE090E00E94E6
:105E90007C758AE090E00E947C75E2E8F9E08491EC
:105EA0008F01882351F0082E000C990B0E947C75FD
:105EB0000F5F1F4FF8018491F4CF8DE090E00E94B6
:105EC0007C758AE090E00E947C75EBE6F9E08491B5
:105ED0008F01882351F0082E000C990B0E947C75CD
:105EE0000F5F1F4FF8018491F4CF8DE090E00E9486
:105EF0007C758AE090E00E947C75E4E5F9E084918D
:105F00008F01882351F0082E000C990B0E947C759C
:105F10000F5F1F4FF8018491F4CF8DE090E00E9455
:105F20007C758AE090E00E947C75E6E4F9E084915B
:105F30008F01882351F0082E000C990B0E947C756C
:105F40000F5F1F4FF8018491F4CF8DE090E00E9425
:105F50007C758AE090E00E947C75E8E3F9E084912A
:105F60008F01882351F0082E000C990B0E947C753C
:105F70000F5F1F4FF8018491F4CF8DE090E00E94F5
:105F80007C758AE090E00E947C7569C2882351F09C
:105F9000082E000C990B0E947C750F5F1F4FF801B3
:105FA0008491F4CF8DE090E00E947C758AE090E0CF
:105FB0000E947C75ECE1F9E084918F01882351F017
:105FC000082E000C990B0E947C750F5F1F4FF80183
:105FD0008491F4CF8DE090E00E947C758AE090E09F
:105FE0000E947C75E6E0F9E084918F01882351F0EE
:105FF000082E000C990B0E947C750F5F1F4FF80153
:106000008491F4CF8DE090E00E947C758AE090E06E
:106010000E947C75E0EFF8E084918F01882351F0B5
:10602000082E000C990B0E947C750F5F1F4FF80122
:106030008491F4CF8DE090E00E947C758AE090E03E
:106040000E947C75EEEDF8E084918F01882351F079
:10605000082E000C990B0E947C750F5F1F4FF801F2
:106060008491F4CF8DE090E00E947C758AE090E00E
:106070000E947C75ECECF8E084918F01882351F04C
:10608000082E000C990B0E947C750F5F1F4FF801C2
:106090008491F4CF8DE090E00E947C758AE090E0DE
:1060A0000E947C75EEEBF8E084918F01882351F01B
:1060B000082E000C990B0E947C750F5F1F4FF80192
:1060C0008491F4CF8DE090E00E947C758AE090E0AE
:1060D0000E947C75E0EBF8E084918F01882309F43D
:1060E0004CCF082E000C990B0E947C750F5F1F4F40
:1060F000F8018491F3CF8091C40F882309F486C1FD
:1061000081E080934112109243121092421283E177
:1061100090E10E947B918BE1E3E1F0E1DE011596D5
:1061200001900D928A95E1F78091111090911210D3
:106130009C838B8385EE92E09A83898340E050E0D4
:10614000BE016F5F7F4F80E090E00E94B277CE018A
:1061500001960E94AD4FC0904212D0904312009120
:10616000D3131091D413C601801B910B049720F018
:106170006801F3E0CF0ED11C51EA452E58E0552EB0
:1061800062E9662E68E0762EC016D10608F467C173
:106190000115110509F0A1C067EC7FE083E190E1F2
:1061A0000E9443906AE173E087EC9FE00E945ECE1C
:1061B000892B09F04AC0F201849141EAE42E48E0BB
:1061C000F42E882359F0082E000C990B0E947C7540
:1061D000FFEFEF1AFF0AF7018491F3CF8DE090E013
:1061E0000E947C758AE090E00E947C75F3018491A6
:1061F00032E9E32E38E0F32E882359F0082E000C04
:10620000990B0E947C75FFEFEF1AFF0AF70184914A
:10621000F3CF8DE090E00E947C758AE090E00E94D0
:106220007C754AE060E070E0CB010E94F241E2E858
:10623000F8E084917F012FEFE21AF20A882309F433
:10624000E2C00E94D63EF701F4CFEEE7F8E0849179
:106250007F01882359F0082E000C990B0E947C7551
:10626000FFEFEF1AFF0AF7018491F3CF8DE090E082
:106270000E947C758AE090E00E947C75F101849117
:106280002AE7E22E28E0F22E882359F0082E000C8F
:10629000990B0E947C75FFEFEF1AFF0AF7018491BA
:1062A000F3CF8DE090E00E947C758AE090E00E9440
:1062B0007C754AE060E070E0CB010E94F241E5E7C6
:1062C000F8E084917F012FEFE21AF20A882309F4A3
:1062D0009AC00E94D63EF701F4CF60E070E0C8019A
:1062E00001970E9478798091C50F882309F45FC0D7
:1062F000E3E7F8E084917F01882359F0082E000C31
:10630000990B0E947C75FFEFEF1AFF0AF701849149
:10631000F3CF87EC9FE00E94EBB68DE090E00E9407
:106320007C758AE090E00E947C75E1E7F8E084915A
:106330007F01882359F0082E000C990B0E947C7570
:10634000FFEFEF1AFF0AF7018491F3CF84ED9FE08E
:106350000E94EBB68DE090E00E947C758AE090E0B0
:106360000E947C75C801A0E0B0E04AE0BC01CD010C
:106370000E94F241EFE6F8E084917F012FEFE21AEC
:10638000F20A882321F00E94D63EF701F5CF94ED62
:10639000E92E9FE0F92EF70181917F01882319F002
:1063A0000E94D63EF8CF8AE00E94D63E2CC087ECF1
:1063B0009FE00E94EBB68DE090E00E947C758AE041
:1063C00090E00E947C7584ED9FE00E94EBB68DE02A
:1063D00090E00E947C758AE090E00E947C75C80184
:1063E000A0E0B0E04AE0BC01CD010E94F24184EDA2
:1063F000E82E8FE0F82EF70181917F01882399F232
:106400000E94D63EF8CF0F5F1F4FBECEE0E6F8E009
:1064100084918F01882351F0082E000C990B0E9463
:106420007C750F5F1F4FF8018491F4CF8DE090E0F1
:106430000E947C758AE090E00E947C75E1E5F8E0BE
:1064400084918F01882309F498CD082E000C990BB4
:106450000E947C750F5F1F4FF8018491F3CFEBE82A
:10646000FBE084918F01882309F49FCA082E000C59
:10647000990B0E947C750F5F1F4FF8018491F3CF39
:106480008091C30F882339F00E94E4764EC4809136
:10649000C30F8823E9F00E94D0B047C48091D11384
:1064A000823019F0833609F040C40E94C376E7E8D1
:1064B000FBE084918F01882309F477CA082E000C31
:1064C000990B0E947C750F5F1F4FF8018491F3CFE9
:1064D0008091D113833609F028C4DDCF8EE79BE08D
:1064E0000E94D04F8091450F9091460F891B8F706D
:1064F00009F01BC48091D113823009F416C483368D
:1065000009F047C412C48DE090E00E947C758AE0D7
:1065100090E00E947C7549CA8091450F9091460F8A
:10652000891B8F7009F001C48091D113823009F466
:10653000FCC3833609F4F9C380918F1181117DC4A6
:10654000F4C383E50E9487B6811126C083E40E94CC
:1065500087B6882309F4E9C38091450F9091460FCF
:10656000891B8F7009F0E1C320E030E040E251E484
:106570006091FF03709100048091010490910204E6
:106580000E94BDC687FF08C08BE69BE09093360D46
:106590008093350D0E94023F0E94A2B620E030E0B9
:1065A000A9010E94BDC687FD10C00E94A2B620E0CE
:1065B00030E849E853E40E940DCD18164CF00E94D3
:1065C000A2B60E9430CCCB0105C080E090E002C0B2
:1065D00083E191E00E941A74A8C383E50E9487B604
:1065E000882309F4A2C30E94A2B620E030E0A901EA
:1065F0000E94BDC687FD11C00E94A2B620E030E017
:1066000046E153E40E940DCD18164CF00E94A2B64C
:106610000E9430CC362F272F04C030E001C036E96D
:1066200020E0832F922F8E36910514F08EE690E0B5
:1066300090930A04809309040E94F47B76C383E557
:106640000E9487B68823D9F00E94A2B620E030E0ED
:106650004FE753E40E9422C720E030E048EC52E4C8
:106660000E94C3CB0E9430CC6F3F710519F010F02F
:106670006FEF70E0709308046093070496C98FEF82
:1066800090E090930804809307048FC98091450F90
:106690009091460F891B8F7009F087C98091C30FB5
:1066A000811183C90E948F885F9A8091F6038E7F43
:1066B0008093F6038A9A479A8091F6038D7F8093A0
:1066C000F603809108018095817080930601479AB6
:1066D0008091F6038B7F8093F603129A66C983E557
:1066E0000E9487B6882319F10E94A2B620E030E00C
:1066F00040E252E40E94BDC687FD0FC00E94A2B6D0
:1067000020E030EC49E754E40E940DCD181644F027
:106710000E94A2B60E942BCC05C068E270E002C0C5
:1067200067EE73E07093030260930202FEC2E5E637
:10673000FBE084918F01882351F0082E000C990B07
:106740000E947C750F5F1F4FF8018491F4CFC090B9
:106750000202D09003020D2C000CEE08FF08F7FE99
:106760000DC06DE28CE295E1A5D566277727CB01B8
:106770006C197D098E099F094AE003C04AE0C701F0
:10678000B6010E94ABB611C98091450F9091460F9A
:10679000891B8F7009F0C9C28091D113823009F42E
:1067A000C4C2833609F08FC2C0C28091450F909158
:1067B000460F891B8F7009F0F8C88091D113823081
:1067C00009F4F3C8833609F05AC3EFC88091450F26
:1067D0009091460F891B8F7009F0A7C28091D11349
:1067E000823009F4A2C2833609F09CC49EC2809113
:1067F000450F9091460F891B8F7009F096C28091CA
:10680000D113823009F491C2833609F0C0C48DC21D
:106810008091450F9091460F891B8F7009F085C2BA
:106820008091D113823009F480C2833609F0E4C428
:106830007CC28091FF13811103C00E94817568C1E1
:106840008E3271F5809100148E3209F0EAC0809189
:106850006411882309F45CC18150809364118823FA
:1068600061F090E001974FE1489F9001499F300D02
:106870001124C901825D9F4E02C080EF9FE02BE191
:10688000FC013496A3E1B0E101900D922A95E1F765
:10689000FC0182819381909312108093111038C172
:1068A0008C3309F0BEC06CE173E08FEF93E10E947E
:1068B0005ECE892B21F481E080931D1429C16BE207
:1068C00073E08FEF93E10E945ECE892B79F4EDE2C5
:1068D000F8E084918F010F5F1F4F882321F00E9401
:1068E000D63EF801F6CF8AE198E088C062E473E012
:1068F0008FEF93E10E945ECE892B79F4E6EFF7E00B
:1069000084918F010F5F1F4F882321F00E94D63E94
:10691000F801F6CF83EE97E071C069E573E08FEF81
:1069200093E10E945ECE892B79F4E8ECF7E0849144
:106930008F010F5F1F4F882321F00E94D63EF80180
:10694000F6CF83EC97E05AC067E673E08FEF93E1F0
:106950000E945ECE892B79F4E8EAF7E084918F01FA
:106960000F5F1F4F882321F00E94D63EF801F6CF1B
:1069700083EA97E043C065E773E08FEF93E10E94FD
:106980005ECE892B79F4E8E8F7E084918F010F5F00
:106990001F4F882321F00E94D63EF801F6CF8FE7E3
:1069A00097E02CC063E873E08FEF93E10E945ECE26
:1069B000892B71F40CE517E0F8018491882329F004
:1069C0000F5F1F4F0E94D63EF7CF85E597E016C0B8
:1069D00069E973E08FEF93E10E945ECE892BA9F401
:1069E000E6E3F7E084918F010F5F1F4F882321F0CA
:1069F0000E94D63EF801F6CF8FE297E09093360DD5
:106A00008093350D0E94023F83C06BEA73E08FEFE5
:106A100093E10E945ECE892B09F07AC010921D147A
:106A200077C01D8218861C821B8285EE92E09A83B5
:106A3000898380911610811103C060EF7FE002C04E
:106A40006FE070E16115710519F06C5F7F4F02C056
:106A500060E070E021E04FEF53E1CE0105960E9427
:106A6000B195882361F18BE1FE013596A3E1B0E198
:106A700001900D928A95E1F72B813C8130931210A1
:106A800020931110809164118A3008F03DC091E08C
:106A9000980F90936411FFE18F9FC0011124DC01D6
:106AA000AE5CBF4E4BE1E3E1F0E101900D924A95FF
:106AB000E1F7FC01E25DFF4E3383228325C0EEEE59
:106AC000F9E184918F010F5F1F4F882321F00E940D
:106AD000D63EF801F6CFE9E1F7E084918F010F5F30
:106AE0001F4F882321F00E94D63EF801F6CF0FEF0A
:106AF00013E1F80181918F01882319F00E94D63E9D
:106B0000F8CF8AE00E94D63ECE0101960E94AD4F9A
:106B10001092FF138091090180FF07C1E9EAFAE0B2
:106B200084918F01882311F40C94D52C082E000C2D
:106B3000990B0E947C750F5F1F4FF8018491F2CF73
:106B40008FE40E9487B681110C94D52C83E40E94B7
:106B500087B60C94D52C83E50E9487B6811159C065
:106B60008FE40E9487B6882319F081E79AE007C076
:106B700084E50E9487B6882349F089E49AE09093DF
:106B8000360D8093350D0E94023F43C083E40E947E
:106B900087B6882319F080E29AE0F1CF81E50E9460
:106BA00087B6882319F088EF99E0E9CF88E40E943E
:106BB00087B68823C9F0E4EFF9E084918F01882338
:106BC00051F0082E000C990B0E947C750F5F1F4F2F
:106BD000F8018491F4CF8DE090E00E947C758AE00A
:106BE00090E00E947C7515C08CE40E9487B68823D3
:106BF00081F0E0EFF9E084918F01882361F3082EA2
:106C0000000C990B0E947C750F5F1F4FF801849157
:106C1000F4CFE8EBFAE084918F01882311F40C940F
:106C2000D52C082E000C990B0E947C750F5F1F4F0E
:106C3000F8018491F2CF8091450F8091460F0C941A
:106C4000D52C83E50E9487B6882309F46EC088ECB2
:106C500099E09093360D8093350D0E94023FE8EB4A
:106C6000FAE084918F01882311F40C94D52C082E1E
:106C7000000C990B0E947C750F5F1F4FF8018491E7
:106C8000F2CFE3ECF9E084918F01882351F0082ED4
:106C9000000C990B0E947C750F5F1F4FF8018491C7
:106CA000F4CFEEEBF9E084918F01882311F40C947A
:106CB000D52C082E000C990B0E947C750F5F1F4F7E
:106CC000F8018491F2CF88E50E9487B6811106C051
:106CD00089E50E9487B6882309F4C3C088E50E942D
:106CE00087B6882341F08FE59BE09093360D809323
:106CF000350D0E94023F89E50E9487B6882341F046
:106D000089E59BE09093360D8093350D0E94023FFC
:106D10008AE50E9487B6882341F083E59BE0909343
:106D2000360D8093350D0E94023F8091CA139091D9
:106D3000CB13019664E070E00E94D0CD9093CB130A
:106D40008093CA138091C6139091C71301969093B4
:106D5000C7138093C6131092CE131092CD130C94C8
:106D6000B62B4091CA135091CB139F012F5F3F4F19
:106D70003093CE132093CD1390E6949F9001959F6E
:106D8000300D11242A5B3D4EE20FF31F80830C94DB
:106D9000B62B0091CF131091D013780124E0E20EAE
:106DA000F11C6AE270E0C7010E9453CEF801248111
:106DB0002F3221F4B8016B5F7F4F03C02C3339F4BD
:106DC000B7018FEF93E10E9467CE0C94D52C1092FF
:106DD000FF13009719F0FC01319710828091CF13B7
:106DE0009091D01340E061E004960E94B3B480918A
:106DF0008F11882389F0EAE7FBE084918F018823D3
:106E000009F481CB082E000C990B0E947C750F5F52
:106E10001F4FF8018491F3CFE6E7FBE084918F01E7
:106E2000882309F470CB082E000C990B0E947C7506
:106E30000F5F1F4FF8018491F3CF0E94C376E2E702
:106E4000FBE084918F01882311F40C94D52C082E3B
:106E5000000C990B0E947C750F5F1F4FF801849105
:106E6000F2CF8AE50E9487B6811138CF83E40E9471
:106E700087B6882309F459CF8FE49BE050CF86E48E
:106E80000E9487B6882309F44AC10E94A2B60E94D4
:106E900030CC8B018BE49BE09093360D8093350DC5
:106EA000B1D788E50E9487B6882309F450C00E94B4
:106EB000A2B62B013C012DEC3CEC4CE45EE30E94BD
:106EC000BDC69E012F5F3F4F7901181674F020E078
:106ED00030E0A901C301B2010E940DCD18162CF4B7
:106EE0001F930F9380E49BE004C12DEC3CEC4CEC31
:106EF0005DEBC301B2010E94BDC618167CF020E014
:106F000030E040E85FEBC301B2010E940DCD1816DE
:106F10002CF41F930F9384E39BE0EBC01F930F931C
:106F2000C301B2010E942BCC7F936F938AE29BE056
:106F30009F938F93FF92EF920E948FC60FB6F894A3
:106F4000DEBF0FBECDBFCE01019637D7DFC089E5CA
:106F50000E9487B6882309F441C00E94A2B62B0183
:106F60003C012DEC3CEC4CE45EE30E94BDC6FE010E
:106F700031967F01181674F020E030E0A901C301BA
:106F8000B2010E940DCD18162CF41F930F938FE1C0
:106F90009BE0AFC02DEC3CEC4CEC5DEBC301B201CF
:106FA0000E94BDC618167CF020E030E040E85FEBA0
:106FB000C301B2010E940DCD18162CF41F930F933C
:106FC00083E19BE096C01F930F93C301B2010E941F
:106FD0002BCC7F936F9389E09BE0AACF8AE50E9438
:106FE00087B6882309F441C00E94A2B62B013C0158
:106FF0002DEC3CEC4CE45EE30E94BDC6FE013196F4
:107000007F01181674F020E030E0A901C301B2013D
:107010000E940DCD18162CF41F930F938EEF9AE05B
:1070200068C02DEC3CEC4CEC5DEBC301B2010E945E
:10703000BDC618167CF020E030E040E85FEBC301ED
:10704000B2010E940DCD18162CF41F930F9382EFFE
:107050009AE04FC01F930F93C301B2010E942BCC43
:107060007F936F9388EE9AE063CF85E40E9487B6A2
:10707000882309F44BC00E94A2B62B013C012DECE1
:107080003CEC4CE45EE30E94BDC6FE0131967F01FC
:10709000181674F020E030E0A901C301B2010E948B
:1070A0000DCD18162CF41F930F938DED9AE021C08F
:1070B0002DEC3CEC4CEC5DEBC301B2010E94BDC673
:1070C00018167CF020E030E040E85FEBC301B2012D
:1070D0000E940DCD18162CF41F930F9381ED9AE0AA
:1070E00008C0C301B2010E942BCC7F936F9386EC42
:1070F0009AE09F938F93FF92EF920E948FC60F901A
:107100000F900F900F900F900F901DCF82EC9AE090
:107110009093360D8093350D75D60C94D52C00E0E8
:1071200010E0B8CE20E030E040E251E46091FF038F
:107130007091000480910104909102040E94BDC6E8
:1071400087FF07C08BEB9AE09093360D8093350D47
:1071500059D682E390E090930A04809309040E9438
:10716000F47B88EC90E00E941A74E8EBFAE08491DA
:107170008F01882311F40C94D52C082E000C990B48
:107180000E947C750F5F1F4FF8018491F2CF20E0C1
:1071900030E040E251E46091FF037091000480917F
:1071A0000104909102040E94BDC687FF07C081EBD5
:1071B0009AE09093360D8093350D24D680E590E0CB
:1071C00090930A04809309040E94F47B80EF90E07E
:1071D0000E941A74E8EBFAE084918F01882311F47D
:1071E0000C94D52C082E000C990B0E947C750F5F17
:1071F0001F4FF8018491F2CF80E090E00E941A7452
:1072000010920A04109209040E94F47BEDEAFAE05D
:1072100084918F01882311F40C94D52C082E000C36
:10722000990B0E947C750F5F1F4FF8018491F2CF7C
:107230006F960FB6F894DEBF0FBECDBFDF91CF9132
:107240001F910F91FF90EF90DF90CF90BF90AF9084
:107250009F908F907F906F905F904F903F902F9076
:10726000089590917B16E92FF0E0E155F44F80836B
:107270009F5F943018F490937B1602C010927B1697
:1072800080917C168F5F80937C1608958091EA0A26
:107290009091EB0A981759F0E92FF0E0E659F54F75
:1072A00080819F5F9F779093EB0A90E008958FEF26
:1072B0009FEF08950F931F93CF93DF93FC01A68553
:1072C000B7858D0100581F4FE8018881998101968B
:1072D0008F779927AD014E575F4FEA012881398199
:1072E00028173907D1F3E80128813981A20FB31F8C
:1072F0006C93A685B785A058BF4F11969C938E932B
:10730000A689B7892C9181E090E0078C02C0880F94
:10731000991F0A94E2F7822B8C9381E081A3048861
:10732000F589E02D80818064808381E090E0DF91A9
:10733000CF911F910F910895FC0181A1882329F01D
:10734000A489B5898C9186FFFBCF11A20895FC0119
:10735000A485B585FD01E058FF4F2081318132962B
:10736000808191812817390779F080819181A80F58
:10737000B91F8C91208131812F5F3F4F2F773327A9
:107380003183208390E008958FEF9FEF0895DC0113
:107390001C96ED91FC911D97DF01A058BF4F2D91D8
:1073A0003C91119712968D919C911197281739074E
:1073B00039F08D919C91E80FF91F808190E008953C
:1073C0008FEF9FEF0895FC0124853585F901E05882
:1073D000FF4F8081918132962081318180589F4F6B
:1073E000821B930B60E870E00C94D0CD0895089553
:1073F00080E090E00895CF93FC0120812B33A1F031
:1074000020917C16243080F4C62FBC0180917B161D
:10741000F0E68F9FC00111248C54944F0E9467CED8
:107420008C2F1FDF81E001C080E0CF9108952F9263
:107430003F924F925F926F927F928F929F92AF9204
:10744000BF92CF92DF92EF92FF920F931F93CF9351
:10745000DF9300D000D0CDB7DEB79A8389830E9436
:107460004BB4E981FA81C680D780E084F184C114ED
:10747000D104E104F10409F0ACC22485222309F40B
:1074800069C332852150248721E0230F2287458557
:10749000241301C01286E981FA8124E0329FE00DB5
:1074A000F11D1124C684D784E088F188E981FA812E
:1074B000C282D382E482F582DC01CB018C0D9D1D5A
:1074C000A11DB11D86839783A087B1878481958193
:1074D000892B09F43FC3FFB7FD83F894E981FA8152
:1074E000228033802101612C712C048115818091CF
:1074F00039028F3121F08F3F09F068C205C0EEE0FC
:10750000F8E124912E83DAC08FE180933902EEE016
:10751000F8E184918E838F3F09F458C2823009F4D8
:1075200069C030F5882309F44CC0813009F0C6C029
:107530001092800010928100809181008860809379
:10754000810080918100816080938100E9EDF3E208
:10755000E491F0E0EE0FFF1FEA57FC4D8591949106
:10756000EFE1F4E2E491E0931804E1E0EE8330C14E
:107570009E81943009F482C008F460C0953009F00F
:107580009DC01092200110922101809121018860FC
:107590008093210180912101816080932101E9ED97
:1075A000F3E2E491F0E0EE0FFF1FEA57FC4D859106
:1075B0009491EFE1F4E2E491E093150495E09E8369
:1075C00007C114BC15BC84B5826084BD85B58160DB
:1075D00085BDE9EDF3E2E491F0E0EE0FFF1FEA571D
:1075E000FC4D85919491EFE1F4E2E491E09319046C
:1075F0001E82ABC21092B0001092B1008091B00018
:1076000082608093B0008091B10081608093B1006E
:10761000E9EDF3E2E491F0E0EE0FFF1FEA57FC4DD5
:10762000859194919093940B8093930BEFE1F4E206
:10763000E491E093950BF2E0FE8387C210929000F4
:1076400010929100809191008860809391008091C8
:107650009100816080939100E9EDF3E2E491F0E024
:10766000EE0FFF1FEA57FC4D85919491EFE1F4E294
:10767000E491E093170423E02E83AAC01092A000A7
:107680001092A1008091A10088608093A100809158
:10769000A10081608093A100E9EDF3E2E491F0E0C4
:1076A000EE0FFF1FEA57FC4D85919491EFE1F4E254
:1076B000E491E093160484E08E838AC0EE81E7FDB6
:1076C00085C161E08FE10E9410B38E818D7F09F04A
:1076D00083C04801A12CB12C60E072E18AE790E000
:1076E000A50194010E94E3CD29833A834B835C83F7
:1076F00069017A01F1E0CF1AD108E108F1082FEF12
:10770000C216D104E104F10409F008F44EC060E4AB
:1077100072E48FE090E0A50194010E94E3CD69013D
:107720007A0181E0C81AD108E108F1089E819230FF
:1077300009F5EFEFCE16D104E104F10409F008F4E5
:10774000CBC160E970ED83E090E0A50194010E9457
:10775000E3CD69017A01F1E0CF1AD108E108F1081F
:107760002FEFC216D104E104F10411F008F041C179
:1077700083E027C08FEFC816D104E104F104B9F00B
:10778000B0F068E478EE81E090E0A50194010E94F9
:10779000E3CD69017A0191E0C91AD108E108F10845
:1077A000EE81EE2309F49AC163C181E001C082E059
:1077B0009E81911106C095B5987F892B85BD7AC0B1
:1077C00085E09091B100987F892B8093B10072C0C1
:1077D00061E08FE10E9410B34801A12CB12C60E060
:1077E00072E18AE790E0A50194010E94E3CD69016E
:1077F0007A01E1E0CE1AD108E108F108C114D10400
:10780000F1E0EF06F10488F068E478EE81E090E0C2
:10781000A50194010E94E3CD69017A0181E0C81AB3
:10782000D108E108F10883E001C081E09E81913038
:1078300071F490918100987F892B80938100452875
:1078400046284728D9F52FEF3FEFA90168C0EE8100
:10785000E33071F490919100987F892B809391008F
:1078600045284628472851F52FEF3FEFA90179C059
:10787000FE81F43071F49091A100987F892B809360
:10788000A100452846284728C9F42FEF3FEFA9015A
:107890007AC02E81253071F490912101987F892B37
:1078A0008093210145284628472841F42FEF3FEFD8
:1078B000A9017BC045284628472869F0D801AA0FAE
:1078C000BB1F91010E94D7CA28EE33E040E050E090
:1078D0000E94ABCA03C02FEF3FEFA9018E81823017
:1078E00081F12CF4882361F08130C9F06FC09E8152
:1078F000943009F448C0ACF1953009F456C066C024
:10790000C7BC20932A0430932B0440932C0450933B
:107910002D0480916E00826080936E0057C0D092DB
:107920008900C09288002093260430932704409356
:1079300028045093290480916F00826080936F0027
:1079400045C0C092B3002093960B3093970B4093A1
:10795000980B5093990B8091700082608093700017
:1079600035C0D0929900C0929800209322043093A1
:107970002304409324045093250480917100826075
:107980008093710023C0D092A900C092A8002093D8
:107990001E0430931F0440932004509321048091CF
:1079A000720082608093720011C0D0922901C0924F
:1079B000280120931A0430931B0440931C04509315
:1079C0001D0480917300826080937300ED81EFBF8E
:1079D000C1C0DC01CB018C199D09AE09BF09B7FDFF
:1079E000B9C04698E981FA811682178210861186FD
:1079F000B1C068E478EE81E090E0A50194010E94B6
:107A0000E3CD69017A01F1E0CF1AD108E108F1086C
:107A10002FEFC216D104E104F10441F138F164E220
:107A200074EF80E090E0A50194010E94E3CD69012C
:107A30007A01F1E0CF1AD108E108F1082FEFC21660
:107A4000D104E104F10409F008F4BACE62E17AE766
:107A500080E090E0A50194010E94E3CD69017A01E4
:107A600081E0C81AD108E108F10819C084E0A9CE64
:107A70002FEFC216D104E104F10409F008F463C049
:107A800062E17AE780E090E0A50194010E94E3CDF5
:107A900069017A01F1E0CF1AD108E108F1082FEF6E
:107AA000C216D104E104F104A9F0A0F089819A8101
:107AB000AB81BC812AE0B595A795979587952A95C6
:107AC000D1F76C017D01F1E0CF1AD108E108F1088E
:107AD00087E077CE86E075CE82E073CEEFEFCE16EC
:107AE000D104E104F10469F160F162E17AE780E038
:107AF00090E0A50194010E94E3CD69017A0181E043
:107B0000C81AD108E108F1089FEFC916D104E104B1
:107B1000F104A9F0A0F089819A81AB81BC813AE09F
:107B2000B595A795979587953A95D1F76C017D0105
:107B3000E1E0CE1AD108E108F10885E03CCE84E00E
:107B40003ACE83E038CE84E033CE61E08FE10E940C
:107B500010B3BFCD26960FB6F894DEBF0FBECDBFD3
:107B6000DF91CF911F910F91FF90EF90DF90CF9019
:107B7000BF90AF909F908F907F906F905F904F904D
:107B80003F902F9008950F931F93CF93DF93CDB71E
:107B9000DEB72C970FB6F894DEBF0FBECDBFE7EF70
:107BA000F3E080859185A285B38544815581668106
:107BB0007781008111812281338109831A832B838C
:107BC0003C834D835E836F83788789879A87AB87F1
:107BD000BC87AE01475F5F4FBE016B5F7F4FCE0139
:107BE00001960E941DA923E034E0AE01475F5F4F7C
:107BF000BE016B5F7F4FCE0101960E9496B92C9615
:107C00000FB6F894DEBF0FBECDBFDF91CF911F91AD
:107C10000F9108958091E6039091E703009731F06A
:107C20004AE050E060E070E00C9411C460E070E065
:107C3000CB010895EFDF97FD0AC0ECDF6F3F7105C0
:107C40008105910509F02CF4E5DF862F089580E089
:107C500008958FEF08958091E6039091E703892BB3
:107C600031F0E8DF91E0811103C090E001C091E0C4
:107C7000892F08950F931F93CF938091E6039091DE
:107C8000E703009711F1FC018F01C1912C2F2F7D8B
:107C9000A9F0C53411F0C536B9F7F801108260E0DB
:107CA00070E08091E6039091E7030E94BEC2F80164
:107CB000C083562F472F382F292F0BC060E070E06C
:107CC000CF911F910F910C94BEC250E040E030E084
:107CD00020E0652F742F832F922FCF911F910F914A
:107CE000089581548A3108F042C0E82FF0E04091B5
:107CF000A6165091A7166091A8167091A91604C0F7
:107D000076956795579547958A95D2F7842F817018
:107D100040FF2FC0E457F94E9081992309F1E0917B
:107D20006B16F0916C16E90FF11D908120ED290F73
:107D30002A3098F09E3211F491810CC09D3211F0DE
:107D40009B3271F4918120ED290F2A3030F09E3260
:107D500039F4928190539A3018F42E2F9F2F02C03D
:107D600020E090E02093E6039093E703089580E0FD
:107D700008950895B6DF882341F081E02091E6035D
:107D80003091E703232B09F480E00895FC0123815F
:107D900021110C941E90089580E1E7EFF3E0A4E137
:107DA000BBE001900D928A95E1F708959091C00093
:107DB00095FFFCCF8093C6000895EF92FF921F932A
:107DC000CF93DF937C0160E016DB182F882399F0B6
:107DD000EEEEF9E18491EF012196882319F0E6DFB8
:107DE000FE01F8CFB70182E19CE00E94604D82E283
:107DF000DDDF8AE0DBDF812FDF91CF911F91FF90E4
:107E0000EF900895DF92EF92FF920F931F93CF931D
:107E1000DF93CDB7DEB76E970FB6F894DEBF0FBE17
:107E2000CDBF6091350D7091360D6115710541F131
:107E30004DE150E0CE0101967C010E9466C61E8E87
:107E4000F7018F010E191F09D190DD2019F09AE07A
:107E5000D912F7CFF701E00FF11F1082C701ADDF94
:107E6000882371F0DD20A9F00F5F1F4F8091350D41
:107E70009091360D080F191F1093360D0093350D94
:107E800081E02091350D3091360D232B29F480E0CF
:107E900003C000E010E0F0CF6E960FB6F894DEBF9E
:107EA0000FBECDBFDF91CF911F910F91FF90EF904B
:107EB000DF9008953F924F925F926F927F928F92E0
:107EC0009F92AF92BF92CF92DF92EF92FF920F9369
:107ED0001F93CF93DF931F92CDB7DEB793DF81114E
:107EE0006EC280917C16843008F047C0CFD9AC01B7
:107EF00097FF7CC142C08E3409F0D9C1011511052C
:107F000009F4D5C165E47DE0C8010E9475C67C0115
:107F1000892B09F48EC16EE470E0C80104960E94BA
:107F200053CE009709F485C14AE050E060E070E06C
:107F300001960E9411C460932E0470932F048093C5
:107F40003004909331048090881690908916A09008
:107F50008A16B0908B162FEF821A920AA20AB20AE2
:107F6000681579058A059B0509F465C1EF2809F0B4
:107F700062C182E19DE00E9455B68091C30F8823C3
:107F800009F41DC280917C16811102C010929404E4
:107F9000EE24E39440913D1250913E1260913F12C5
:107FA000709140128091391290913A12A0913B1237
:107FB000B0913C12481759076A077B0708F4E12C77
:107FC00000E010E09924939480E6882E9AE4A92E8C
:107FD0009DE0B92E2DE8322E80917C16843008F079
:107FE000EEC1E110ECC1809194048111E8C180914F
:107FF000941190919511A0919611B0919711809341
:108000003D1290933E12A0933F12B093401241E074
:1080100050E0BE016F5F7F4F8CE891E10E94A59216
:10802000019719F4898190E002C08FEF9FEFF82E3D
:1080300040903D1250903E1260903F12709040125E
:108040004091391250913A1260913B1270913C125A
:10805000EE24E394441655066606770608F4E12CF0
:108060004416550666067706B0F4019609F46AC010
:108070008AE0F81609F489C09DE0F91609F485C074
:1080800023E2F21619F08AE3F81296C08091930465
:10809000811192C06FC00E9436688CE891E10E9405
:1080A0001E908091A711882359F181508093A711C8
:1080B000389EC001112441E061E084559E4E0E942B
:1080C000B3B4E091A71194E0E99FF0011124E855C1
:1080D000FE4E408151816281738140933D125093E5
:1080E0003E1260933F12709340128CE891E10E941F
:1080F000348F8091C40F8823A9F09092C30F12C0CF
:108100001092C30F0E94C8A40E94237E0E94B27DD9
:108110006D3371058105910528F0B092360DA0925E
:10812000350D70DE8091C30F811128C0EDE5FDE0B3
:1081300084916F012FEFC21AD20A8823D9F036DE5C
:10814000F601F6CFE9EDF9E184916F019FEFC91ACD
:10815000D90A882319F02ADEF601F6CFEEE4FDE015
:1081600084916F012FEFC21AD20A882319F01EDE04
:10817000F601F6CF83E2F81208C005C023E2F2123E
:108180001BC100E010E0909294041092930401153A
:10819000110519F40E94F8800CC080917B16889E0E
:1081A000000D111D1124F801EC54F44F108280E0F1
:1081B00058D800E010E010CF0F35110508F00CCFB3
:1081C0009BE3F91202C09092930480919304811171
:1081D00003CF80917B16F801889EE00DF11D1124DC
:1081E000EC54F44FF0820F5F1F4FF6CE982F209182
:1081F0008616309187168A3019F09D3009F0AAC092
:10820000109292042115310519F40E94F88069CE6C
:10821000F901EE5CFB4F10821092871610928616C1
:1082200002E314E0F8018191803209F064CE8F01FD
:10823000F9CFC80179CE6AE270E0C8010E948BCE06
:108240009C01009701F1982F901BF12C992339F094
:108250009150F801E90FF11D8081F826F7CF4AE02F
:1082600050E060E070E0C90101960E9411C4CF2C7B
:10827000D12CE12CF12C6C157D058E059F0531F07C
:1082800083EF9CE078CE89EC9CE075CE80912E0443
:1082900090912F04A0913004B091310480938816FE
:1082A00090938916A0938A16B0938B160EC0809176
:1082B000C10F882351F062EB73E0C8010E945ECECB
:1082C000892B19F08FE99CE056CE809141028111F3
:1082D0001FC067E470E0C8010E9453CE0097C1F050
:1082E0004AE050E060E070E001960E9411C4643002
:1082F00071058105910560F4E8E2FCE084917F015D
:108300009FEFE91AF90A882319F050DDF701F6CF3B
:1083100066EB73E0C8010E945ECE892B11F41092C7
:1083200040026BEB73E0C8010E945ECE892B21F402
:108330008FE19CE00E94D04F60EC73E0C8010E9486
:108340005ECE892B11F40E948F8861E082E394E075
:1083500052D8C7CD2F3531050CF0C3CD9C35C1F4B3
:108360000E94463997FDBDCD209192042111B9CDCF
:108370002091861630918716A9014F5F5F4F509369
:10838000871640938616F901EE5CFB4F8083A9CDDA
:108390009B3319F481E080939204809192048111BF
:1083A000A0CDC90101969093871680938616F90196
:1083B000EE5CFB4F408395CD10929304EBCE0F9073
:1083C000DF91CF911F910F91FF90EF90DF90CF90B1
:1083D000BF90AF909F908F907F906F905F904F90E5
:1083E0003F9008958F929F92AF92BF92EF92FF922B
:1083F0000F931F93CF93DF93CDB7DEB7A0970FB640
:10840000F894DEBF0FBECDBF6115710581059105E2
:1084100089F100E0842E912CA12CB12C102FEE2498
:10842000E394F12CEC0EFD1EE00EF11C07FDFA9416
:10843000A50194010E94ABCAF7016083B901CA018A
:108440000F5F611571058105910541F71F3F21F10E
:10845000E1E0F0E0EC0FFD1FE10FF11D17FDFA95D3
:1084600080818A3010F097E301C090E3890F9EDC91
:108470001150ECCF80E3A0960FB6F894DEBF0FBE8C
:10848000CDBFDF91CF911F910F91FF90EF90BF90E3
:10849000AF909F908F908ACCA0960FB6F894DEBFD5
:1084A0000FBECDBFDF91CF911F910F91FF90EF9045
:1084B000BF90AF909F908F900895CF92DF92EF92F0
:1084C000FF926B017C0197FF0AC08DE26FDCF09494
:1084D000E094D094C094C11CD11CE11CF11C4AE072
:1084E000C701B601FF90EF90DF90CF907BCF8F92C6
:1084F0009F92AF92BF92CF92DF92EF92FF92CF9373
:108500006B017C01B42E20E030E0A9010E94BDC6C1
:1085100087FF06C08DE24ADCF7FAF094F7F8F09492
:10852000C0E060E070E080E09FE3CB1541F02DEC0F
:108530003CEC4CEC5DE30E9422C7CF5FF6CF9B0181
:10854000AC01C701B6010E94E7CA6B017C010E9421
:1085500030CC4B015C014AE045DFCC2379F1C50109
:10856000B4010E94C1C69B01AC01C701B6010E94C3
:10857000E6CA6B017C018EE219DC20E030E040E2CB
:1085800051E4C701B6010E9422C74B015C010E9461
:108590002BCC6B01770FEE08FF08C701B6018DDF0A
:1085A000C701B6010E94C3C69B01AC01C501B4015D
:1085B0000E94E6CA6B017C01C150F9F6CF91FF9091
:1085C000EF90DF90CF90BF90AF909F908F900895E5
:1085D0001F920F920FB60F9211240BB60F922F938A
:1085E0008F939F93EF93FF932091EB0AE091EA0A18
:1085F00081E08E0F8F779091C600281729F0F0E068
:10860000E659F54F9083E82FE093EA0AFF91EF9146
:108610009F918F912F910F900BBE0F900FBE0F90D7
:108620001F9018959C0197FD0EC08436910584F02B
:1086300064E670E00E94D0CDCB016AE070E00E9459
:10864000D0CD805D06C03195219531098DE201C004
:1086500080E28093F2032A30310564F0EAE0F0E032
:10866000C901BF010E94D0CDCB01BF010E94D0CD76
:10867000805D01C080E28093F303C9016AE070E08D
:108680000E94D0CD805D8093F40382EF93E0089543
:108690001F920F920FB60F9211240BB60F922F93C9
:1086A0003F938F939F93EF93FF932091A414309166
:1086B000A5148091A6149091A7142817390731F4B6
:1086C000809131018F7D8093310114C0E091A61417
:1086D000F091A714EC5DFB4E20818091A61490913F
:1086E000A71401968F7799279093A7148093A614C7
:1086F00020933601FF91EF919F918F913F912F91A0
:108700000F900BBE0F900FBE0F901F9018951F92E9
:108710000F920FB60F9211240BB60F922F934F9317
:108720005F938F939F93EF93FF938091300182FD2E
:108730001CC02091360180912815909129154091F7
:108740002A1550912B1501968F77992748175907AD
:1087500071F0E0912815F0912915E855FB4E208322
:10876000909329158093281502C080913601FF91BE
:10877000EF919F918F915F914F912F910F900BBE31
:108780000F900FBE0F901F9018958091450F9091FC
:10879000460F891B8F7019F480E090E00895909146
:1087A000420F992351F0833030F48FEF890F19F085
:1087B0008093420FF1CF1092420FE091460F88E56F
:1087C000E89FF0011124EB56FB4F808180FDE4CF40
:1087D0008091460F8F5F8F708093430F9091460F6B
:1087E0008091440F981304C08091430F8093440FED
:1087F000CF0108950F930FB70F9300916E000F9361
:108800000B7F00936E0000916F000D7F00936F004F
:108810000F930BB70F930CB70F921F922F933F93A9
:108820004F935F936F937F938F939F93AF93BF9378
:10883000EF93FF9311244AD0FF91EF91BF91AF9135
:108840009F918F917F916F915F914F913F912F9168
:108850001F900F900CBF0F910BBF0F910260F89407
:1088600000936F000F9100936E000F910FBF0F9157
:10887000189580911A0A80FF03C089988FEF02C073
:10888000899A81E08093100280911A0A81FF03C0C7
:108890008F9A8FEF02C08F9881E0809311028091B0
:1088A0001A0A82FF09C080910B0180958270809323
:1088B0000901439A8FEF07C080910B01827080936A
:1088C0000901439881E08093120208952F923F920C
:1088D0004F925F926F927F928F929F92AF92BF92D0
:1088E000CF92DF92EF92FF920F931F93CF93DF937C
:1088F000CDB7DEB72D970FB6F894DEBF0FBECDBF54
:10890000F8948FEF9FEF90938900809388002AE07E
:108910002987212C312C44244A94542C32017894F8
:108920008091660A9091670AA091680AB091690ADD
:10893000892B8A2B8B2B09F010C28091521588232A
:10894000E1F0109252158091501590915115892B9C
:1089500009F403C210921B0A10925115109250157F
:108960009091450F8091460F981709F4F6C18091B8
:10897000460F8F5F8F708093460F809150159091B6
:108980005115892B09F4E9C1C090620AD090630A9D
:10899000E090640AF090650A40915E0A50915F0A87
:1089A0006091600A7091610A0091510A10E020E024
:1089B00030E0DB01CA018C199D09AE09BF09081717
:1089C00019072A073B0710F4D901C801482F8C0D5D
:1089D0009D1DAE1DBF1D8093620A9093630AA093F4
:1089E000640AB093650A2091840030918500245E6A
:1089F0003F4FC090370AD090380AE090390AF09083
:108A00003A0A8091270A9091280AA091290AB091E8
:108A10002A0A8C0D9D1DAE1DBF1D8093370A9093B1
:108A2000380AA093390AB0933A0AB7FD1CC0889A55
:108A3000C0905F15D0906015E0906115F0906215C0
:108A400080911002082E000C990BAA0BBB0B8C0D09
:108A50009D1DAE1DBF1D80935F1590936015A09363
:108A60006115B0936215C0903B0AD0903C0AE0902B
:108A70003D0AF0903E0A80912B0A90912C0AA09119
:108A80002D0AB0912E0A8C0D9D1DAE1DBF1D809329
:108A90003B0A90933C0AA0933D0AB0933E0AB7FD6F
:108AA0001CC08E9AC0906315D0906415E090651537
:108AB000F090661580911102082E000C990BAA0BFC
:108AC000BB0B8C0D9D1DAE1DBF1D80936315909338
:108AD0006415A0936515B0936615C0903F0AD090B9
:108AE000400AE090410AF090420A80912F0A90914A
:108AF000300AA091310AB091320A8C0D9D1DAE1D35
:108B0000BF1D80933F0A9093400AA093410AB093FF
:108B1000420AB7FD3EC09091190A80911202992332
:108B2000C1F09091170A92FF02C087FD05C0909195
:108B3000160A992309F4BEC56091170A7091180AA4
:108B400073FF02C087FD0CC09091150A911108C0F7
:108B500006C090910B019095987090930901419AED
:108B6000C0906715D0906815E0906915F0906A156F
:108B7000082E000C990BAA0BBB0B8C0D9D1DAE1D76
:108B8000BF1D8093671590936815A0936915B093E6
:108B90006A15C090430AD090440AE090450AF090CC
:108BA000460A8091330A9091340AA091350AB09117
:108BB000360A8C0D9D1DAE1DBF1D8093430A9093F8
:108BC000440AA093450AB093460AB7FD3AC0809084
:108BD0006B1590906C15A0906D15B0906E15C090AF
:108BE00013020C2C000CDD08EE08FF08C80CD91C81
:108BF000EA1CFB1CC0926B15D0926C15E0926D15AF
:108C0000F0926E15C090230AD090240AE090250AB5
:108C1000F090260A8C199D09AE09BF098093430A7A
:108C20009093440AA093450AB093460A90911A0A79
:108C300080914F0A93FF02C0815001C08F5F8093E3
:108C40004F0A8091370A9091380AA091390AB09161
:108C50003A0AB7FD15C0C090230AD090240AE090CC
:108C6000250AF090260A8C199D09AE09BF09809348
:108C7000370A9093380AA093390AB0933A0A889831
:108C800080913B0A90913C0AA0913D0AB0913E0A26
:108C9000B7FD15C0C090230AD090240AE090250AA1
:108CA000F090260A8C199D09AE09BF0980933B0AF2
:108CB00090933C0AA0933D0AB0933E0A8E9880910F
:108CC0003F0A9091400AA091410AB091420AB7FD33
:108CD0003AC0C090230AD090240AE090250AF09070
:108CE000260A8C199D09AE09BF0980933F0A90930B
:108CF000400AA093410AB093420A8091190A88233E
:108D0000E1F08091170A82FF04C08091120287FD72
:108D100005C08091160A882309F4D3C48091170AEC
:108D20009091180A93FF04C08091120287FD0BC036
:108D30008091150A811107C005C080910B018870D0
:108D4000809309014198415041F0809184009091B5
:108D5000850082179307C8F34CCE80911D02909135
:108D60001E02A0911F02B0912002892B8A2B8B2B0F
:108D700009F08AC08091500A882309F452C080907B
:108D8000620A9090630AA090640AB090650AC0904D
:108D90004B0AD0904C0AE0904D0AF0904E0A809118
:108DA0004F0AC814D904EA04FB0488F420911C0A71
:108DB00030911D0A4091200A5091210A4217530711
:108DC00030F4815080934F0A2150310915C08C1422
:108DD0009D04AE04BF04E8F420911C0A30911D0AE2
:108DE00040911E0A50911F0A2417350790F48F5F97
:108DF00080934F0A2F5F3F4F30931D0A20931C0A28
:108E00004091190250911A0260911B0270911C024C
:108E10000BC04092190250921A0260921B0270928B
:108E20001C024FEF5FEFBA0180914F0A87FD02C02D
:108E3000169801C0169A2091840030918500245E16
:108E40003F4F80914F0A8823B9F0149A80914F0ABE
:108E500087FF02C08F5F01C0815080934F0A149832
:108E600080914F0A882369F3809184009091850056
:108E700082179307C8F3E5CF40931D0250931E025B
:108E800060931F02709320028091660A9091670A96
:108E9000A091680AB091690A892B8A2B8B2B09F063
:108EA0008FC3A0915015B0915115109709F4AEC51C
:108EB000C090620AD090630AE090640AF090650A5C
:108EC00040915E0A50915F0A6091600A7091610A58
:108ED000C416D506E606F706D0F010921B0A1092CB
:108EE0005115109250159091450F8091460F98178B
:108EF00009F48CC58091460F8F5F8F708093460F69
:108F000000ED802E07E0902EA12CB12C8AC140915B
:108F10005A0A50915B0A60915C0A70915D0A4C1587
:108F20005D056E057F0508F46DC04091560A5091AD
:108F3000570A6091580A7091590AD2960D911D9165
:108F40002D913C91D597EE27419FF12D529FC00165
:108F5000629F900D619F800D911D429FF00D811DBC
:108F60009E1F519FF00D811D9E1F609FF00D811D62
:108F70009E1F509FF10D8E1F9E1FF6958E1F9E1FE8
:108F8000349F800D911D359F900D1124FD01EA5BEA
:108F9000FF4F0081118122813381080F191F211D8C
:108FA000311D0093520A1093530A2093540A3093B0
:108FB000550A3497C080D180E280F380C016D10674
:108FC000E206F30640F4C092520AD092530AE092AD
:108FD000540AF092550AC090520AD090530AE09079
:108FE000540AF090550A81E795E121E0FC01859053
:108FF0009590A590B4908C149D04AE04BF0408F421
:1090000066C370C320914B0A30914C0A40914D0ABF
:1090100050914E0A29833A834B835C832C153D057E
:109020004E055F0508F070C04091470A5091480A0C
:109030006091490A70914A0A4A875B876C877D87ED
:10904000D2960D911D912D913C91D597EE27419F80
:10905000F12D529FC001629F900D619F800D911D67
:10906000429FF00D811D9E1F519FF00D811D9E1F7F
:10907000609FF00D811D9E1F509FF10D8E1F9E1F42
:10908000F6958E1F9E1F349F800D911D359F900D6C
:1090900011248C0120E030E08090520A9090530A15
:1090A000A090540AB090550AFD01E65BFF4F0815E9
:1090B00019052A053B05A0F4408151816281738125
:1090C0004D835E836F837887801A910AA20AB30A60
:1090D00084169506A606B70638F44A015B0104C05B
:1090E00080809180A280B38081E795E151E05D832B
:1090F000FC010591159125913491081519052A0552
:109100003B0508F473C380C380914F0A8823D9F0CC
:10911000D8964D915C91D99760E070E0009119026A
:1091200010911A0220911B0230911C024017510726
:109130006207730741F010921D0210921E021092F6
:109140001F02109220024091150250911602609168
:1091500017027091180277FF5CC0AE5BBF4F8D9114
:109160009D910D90BC91A02D21E735E141E0F901E1
:10917000C590D590E590F490C816D906EA06FB068E
:1091800058F4B695A79597958795440F2C5F3F4F58
:1091900075E12D38370759F74093510A8032910510
:1091A000A105B10520F480E290E0A0E0B0E0809756
:1091B000A109B109811538E09307A105B10508F4AB
:1091C000DFC344E0949F900111242F583E4EF901D3
:1091D000329645915491EE27859FB001849F610D91
:1091E0007E1F06946E1F7E1F1124CB01A0E0B0E00D
:1091F000F9014591549160E070E0481B590B6A0BEE
:109200007B0B4093150250931602609317027093E4
:1092100018028090150290901602A0901702B0904C
:1092200018028091501590915115892B09F0C0C1F9
:10923000ACDA9093511580935015892B09F4B8C17D
:10924000E0915015F0915115808183FF3EC08589D2
:109250009689A789B08D80935F1590936015A09330
:109260006115B0936215818D928DA38DB48D80931D
:10927000631590936415A0936515B0936615858D5D
:10928000968DA78DB0A18093671590936815A093D4
:109290006915B0936A1581A192A1A3A1B4A180938D
:1092A0006B1590936C15A0936D15B0936E159091FE
:1092B000450F8091460F981709F4BACF8091460F59
:1092C0008F5F8F708093460FB3CFC588D688E788AD
:1092D000F08C81E0C114D104E104F10409F480E0D0
:1092E000018D128D238D348D011511052105310558
:1092F00009F08260458D568D678D70A1411551052D
:109300006105710509F0846080931B0A1092470A79
:109310001092480A1092490A10924A0A1092560A6C
:109320001092570A1092580A1092590A85A196A1D4
:10933000A7A1B0A580935E0A90935F0AA093600AEC
:10934000B093610A882499245401881A990AAA0AB8
:10935000BB0A8092430A9092440AA092450AB092B6
:10936000460A80923F0A9092400AA092410AB09227
:10937000420A80923B0A90923C0AA0923D0AB09227
:109380003E0A8092370A9092380AA092390AB09227
:109390003A0ACC0CDD1CEE1CFF1CC092270AD092AE
:1093A000280AE092290AF0922A0A000F111F221FB0
:1093B000331F00932B0A10932C0A20932D0A30930D
:1093C0002E0A440F551F661F771F40932F0A509394
:1093D000300A6093310A7093320A41A152A163A10D
:1093E00074A1440F551F661F771F4093330A509393
:1093F000340A6093350A7093360A880F991FAA1FA2
:10940000BB1F8093230A9093240AA093250AB0934C
:10941000260A1092620A1092630A1092640A10924D
:10942000650A82A593A5A4A5B5A580935A0A909331
:109430005B0AA0935C0AB0935D0A86A597A5A0A9D4
:10944000B1A980934B0A90934C0AA0934D0AB09314
:109450004E0A81A58093220A97A99093500A9923D6
:1094600009F124AD35AD3093210A2093200A22ADB5
:1094700033AD30931F0A20931E0A10921D021092E2
:109480001E0210921F021092200240AD51AD60E00A
:1094900070E04093190250931A0260931B0270937C
:1094A0001C0208C04092190250921A0260921B02DC
:1094B00070921C0296A920911A0A92130AC0209158
:1094C000140230E0482F082E000C550B42175307AA
:1094D00029F090931A0A80931402CBD98091A20BA1
:1094E00081110E941AAA40921502509216026092AF
:1094F000170270921802E0915015F0915115EA5B35
:10950000FF4F80819181A281B3818093520A909311
:10951000530AA093540AB093550A21E735E141E07C
:10952000F901C590D590E590F490C816D906EA06E1
:10953000FB0660F4B695A79597958795440F2C5F29
:109540003F4FEDE8F5E1E217F30751F74093510A79
:1095500080329105A105B10520F480E290E0A0E001
:10956000B0E08097A109B109811558E09507A105E0
:10957000B10508F428C264E0969F900111242F5889
:109580003E4EF901329645915491EE27859FB001E8
:10959000849F610D7E1F06946E1F7E1F1124F901AA
:1095A00085909490A12CB12C861A970AA108B10835
:1095B0008092660A9092670AA092680AB092690A3D
:1095C0000091660A1091670A2091680A3091690A31
:1095D00040911D0250911E0260911F027091200265
:1095E000F02E1983F22FE32F4017510762077307FC
:1095F00020F4F42E5983F62FE72F8F2D9981AF2F6A
:10960000BE2F0097E1E0AE07B10520F08FEF9FEF8E
:10961000A0E0B0E0081B190B2A0B3B0B0093660A75
:109620001093670A2093680A3093690A4F3FFFEF4F
:109630005F076F077F0761F0481B590B6A0B7B0BB5
:1096400040931D0250931E0260931F0270932002EC
:10965000F8942091840030918500205F3F4F498528
:1096600041504987442339F0280E391E221633060B
:1096700008F455C901C01901309289002092880070
:1096800078942D960FB6F894DEBF0FBECDBFDF9154
:10969000CF911F910F91FF90EF90DF90CF90BF90EF
:1096A000AF909F908F907F906F905F904F903F9082
:1096B0002F90089590910B019095987090930901C7
:1096C0003BCA80910B0188708093090127CBF694E7
:1096D000E794D794C794220F0496E5E18D389E074E
:1096E00009F084CC2093510AF0E2CF16D104E104B2
:1096F000F10428F410E2C12ED12CE12CF12C30E23F
:10970000C31AD108E108F108C11488E0D806E104C1
:10971000F104F8F0E4E0DE9EC00111248F589E4E63
:10972000FC01329625913491FC2DEE27F39F8001A8
:10973000F29F010D1E1F06940E1F1E1F1124FC0117
:1097400085909490A12CB12C801A910AA108B1089F
:1097500022C0970186013695279517950795F80140
:10976000EC7F9F012F58324FF90185909490F901B9
:10977000329685919491EC2DE770E89F9001E99FD6
:10978000300D1124F3E036952795FA95E1F7821A0A
:10979000930AA12CB12C480D591D6A1D7B1D4093C5
:1097A000560A5093570A6093580A7093590A909139
:1097B000500A80914F0A992309F474C0882309F450
:1097C00030CDD8968D919C91D997A0E0B0E0409192
:1097D000190250911A0260911B0270911C028417A9
:1097E0009507A607B70709F060C01BCDB694A794EC
:1097F000979487944D81440F4D8304966DE875E1ED
:109800006817790709F074CC2D812093510A30E252
:1098100083169104A104B10428F450E2852E912C02
:10982000A12CB12C60E2861A9108A108B10881141C
:1098300078E09706A104B10408F440C0E4E09E9EDD
:10984000C00111248F589E4EFC013296259134910F
:10985000F82DEE27F39F8001F29F010D1E1F069445
:109860000E1F1E1F1124FC0185909490A12CB12C79
:10987000801A910AA108B1084A855B856C857D85AF
:10988000480D591D6A1D7B1D4093470A5093480A95
:109890006093490A70934A0A8091500A811132C03C
:1098A00080914F0A882309F4BCCC10921D021092BB
:1098B0001E0210921F0210922002B3CC9501840167
:1098C0003695279517950795F801EC7F9F012F583E
:1098D000324FF90185919491F901329605911491D5
:1098E000E82DE770E09F9001E19F300D112443E0E7
:1098F000369527954A95E1F74C01821A930AA12CD7
:10990000B12CBACF49815A816B817C812D81420F64
:10991000511D611D711D4C155D056E057F05C8F457
:1099200080914F0A882309F47CCCD8964D915C91A4
:10993000D99760E070E00091190210911A0220910D
:109940001B0230911C02401751076207730709F48C
:1099500068CC10921D0210921E0210921F021092EB
:109960002002D8968D919C91D997A0E0B0E0809389
:10997000190290931A02A0931B02B0931C0251CCBF
:10998000AC01BD017695679557954795FA01EC7F37
:109990009F012F58324FF90145915491F9013296A8
:1099A000659174918770869F9001879F300D112477
:1099B000C901F3E096958795FA95E1F7481B590B95
:1099C00060E070E01ECCAC01BD01769567955795BF
:1099D0004795FA01EC7F9F012F58324FF90185908E
:1099E0009490F9013296459154918770849F90012B
:1099F000859F300D1124C901A3E096958795AA95FE
:109A0000E1F7881A990AA12CB12CD2CD80ED882ECD
:109A100087E0982EA12CB12C0BCCCF92DF92EF9245
:109A2000FF92CF93DF936A017B01FC018491EF01E8
:109A30002196882321F00E94D63EFE01F7CF4AE00E
:109A4000C701B601DF91CF91FF90EF90DF90CF90EB
:109A50000C94F241CF92DF92EF92FF92CF93DF937B
:109A60006A017B01FC018491EF012196882321F09A
:109A70000E94D63EFE01F7CF42E0C701B601DF915A
:109A8000CF91FF90EF90DF90CF900C9477420F939F
:109A90001F93CF93DF938B01FC018491EF012196FB
:109AA000882321F00E94D63EFE01F7CFB801110FA6
:109AB000880B990BDF91CF911F910F910C945D4210
:109AC0000F931F93CF93DF938B01FC018491EF01E0
:109AD0002196882321F00E94D63EFE01F7CFE801AF
:109AE0008991882319F00E94D63EFACFDF91CF9159
:109AF0001F910F9108950F931F93CF93DF9300D081
:109B00001F92CDB7DEB78C0108960E94A3A8698387
:109B10007A838B839C83B8016C5F7F4FAE014F5F6C
:109B20005F4FC8010E9442A79B01AC01F80160850C
:109B30007185828593850E94E6CAF80160877187E6
:109B4000828793870F900F900F900F90DF91CF91A6
:109B50001F910F91089586E40E94713E80939015A5
:109B6000882351F00E943A3E60930C0270930D02DC
:109B700080930E0290930F0283E50E94713E88232A
:109B800051F00E943A3E609308027093090280935C
:109B90000A0290930B0282E40E94713E882351F0E6
:109BA0000E943A3E6093040270930502809306027D
:109BB0009093070208958FEF8EBD0DB407FEFDCF81
:109BC0008EB50895CF92DF92EF92FF92CF93DF93FD
:109BD000EC01C090240BD090250BE090260BF09068
:109BE000270BA7019601688179818A819B810E9458
:109BF000BDC687FF04C0C882D982EA82FB82C090BA
:109C0000280BD090290BE0902A0BF0902B0BA7018A
:109C100096016C817D818E819F810E94BDC687FFE8
:109C200004C0CC82DD82EE82FF82C0902702D090F9
:109C30002802E0902902F0902A02A701960168818B
:109C400079818A819B810E940DCD181624F4C882E7
:109C5000D982EA82FB82C0902B02D0902C02E09045
:109C60002D02F0902E02A70196016C817D818E81DC
:109C70009F810E940DCD181624F4CC82DD82EE82E5
:109C8000FF82C0902C0BD0902D0BE0902E0BF0900B
:109C90002F0BA7019601688579858A859B850E948F
:109CA000BDC687FF04C0C886D986EA86FB86C090F9
:109CB0002F02D0903002E0903102F0903202A701E2
:109CC0009601688579858A859B850E940DCD181639
:109CD00024F4C886D986EA86FB86DF91CF91FF906F
:109CE000EF90DF90CF9008954F925F926F927F92A6
:109CF0008F929F92AF92BF92CF92DF92EF92FF929C
:109D00000F931F93CF93DF93D82EC82FD0E0FE017F
:109D1000EB50F94EC49082E0D81203C081E08093EA
:109D2000190A7E01EE0CFF1CEE0CFF1CF701E75137
:109D3000F94E45905590659074906C2D0C2C000C4C
:109D4000770B880B990B0E94C3C64B015C0120E086
:109D500030E040EC5FE3C301B2010E9422C7A501DD
:109D600094010E9422C7AB01BC0100E010E0980101
:109D70008D2D0E94C799F701E352F94E2591359137
:109D800045915491C501B4010E9422C74B015C0169
:109D900020E030E0A9010E94BDC6882309F448C034
:109DA00000E010E09801B501A40170588D2D0E94CB
:109DB000C799FE01E652F94EC491C11117C0EEEEEB
:109DC000F9E18491EF012196882321F00E94D63E8B
:109DD000FE01F7CFE8EBF6E18491EF0121968823AD
:109DE00021F00E94D63EFE01F7CFCAE0F701E1560E
:109DF000FB4D45905590659074906C2F70E080E01D
:109E000090E00E94C3C69B01AC01C301B2010E9455
:109E1000C3CB2B013C01A5019401C501B4010E94F3
:109E2000E7CAAB01BC01930182018D2D0E94C79945
:109E300082E0D81249C04090F5155090F615609018
:109E4000F7157090F81520E030E0A901C301B201C8
:109E50000E940DCD5301420187FF04C0B7FAB094B0
:109E6000B7F8B09420E030E0A901C501B4010E9428
:109E7000BDC6882349F120E030E0A901C301B20149
:109E80001C142CF40E940DCD18162CF008C00E9452
:109E9000BDC687FF04C081E08093160A03C081E03D
:109EA0008093150A1C1424F4B7FAB094B7F8B09450
:109EB00000E010E09801B501A40182E00E94C7997A
:109EC0001092160A1092150A1092190A81E090E079
:109ED0000D2C01C0880F0A94EAF79091F603982B95
:109EE0009093F6039091130B892B8093130BF7013A
:109EF000E95FF44F10821182128213828D2D0E942D
:109F0000279CF701E455F94E85919591A591B4915F
:109F1000E701C950DC4F88839983AA83BB830E94E1
:109F2000C33DF701EC5EF44F88819981AA81BB8122
:109F300080839183A283B383DF91CF911F910F918F
:109F4000FF90EF90DF90CF90BF90AF909F908F9059
:109F50007F906F905F904F90089525EE32E0FC0166
:109F60003183208304960C94C63E5F9A8091F60359
:109F70008E7F8093F6038A9A479A8091F6038D7FAD
:109F80008093F6038091080180958170809306018B
:109F9000479A8091F6038B7F8093F603129A089577
:109FA000E9EDF9E18491EF012196882321F00E94E7
:109FB000D63EFE01F7CFECE8F6E18491EF01219661
:109FC000882321F00E94D63EFE01F7CF0E94387E02
:109FD000CCDFE8E8F6E18491EF01882349F0082E10
:109FE000000C990B0E947C752196FE018491F5CF9F
:109FF0008DE090E00E947C758AE090E00E947C7584
:10A00000FFEF2BE48DE1F15020408040E1F700C0EC
:10A010000000F8949FEFE4E3FCE09150E040F04052
:10A02000E1F700C000000E94387EA895FECF2F9275
:10A030003F924F925F926F927F928F929F92AF92D8
:10A04000BF92CF92DF92EF92FF920F931F93CF9325
:10A05000DF9300D01F92CDB7DEB70E94AC2A0E94DA
:10A060004BB46B017C0110912202112309F47BC0D7
:10A070008091F90A882309F476C040913C0B5091F5
:10A080003D0B60913E0B70913F0B46015701841AC6
:10A09000950AA60AB70AB7FC78C0833051F134F4A8
:10A0A00081300CF460C0EEEEF9E106C0843009F0B6
:10A0B0005AC0EEEEF9E13BC084919F012F5F3F4F04
:10A0C0003B832A83882329F00E94D63EEA81FB81C4
:10A0D000F3CFE6E0F6E184919F012F5F3F4F3B8392
:10A0E0002A83882309F43FC00E94D63EEA81FB817F
:10A0F000F2CFEEEEF9E184919F012F5F3F4F3B835A
:10A100002A83882329F00E94D63EEA81FB81F3CF7F
:10A11000EFEEF5E184919F012F5F3F4F3B832A8350
:10A12000882309F10E94D63EEA81FB81F3CF849116
:10A130009F012F5F3F4F3B832A83882329F00E9492
:10A14000D63EEA81FB81F3CFE7EDF5E184919F01F3
:10A150002F5F3F4F3B832A83882329F00E94D63EFE
:10A16000EA81FB81F3CF212F30E0A8EEB3E00E941B
:10A17000D7CAC60ED71EE81EF91EC0923C0BD0925D
:10A180003D0BE0923E0BF0923F0B89B182FB88279A
:10A1900080F980931E1490911F1498170CF049C0F9
:10A1A0008091201490912114A0912214B091231435
:10A1B0000196A11DB11D883B3DE39307A105B105A3
:10A1C0004CF48093201490932114A0932214B09304
:10A1D00023143BC0109220141092211410922214C8
:10A1E000109223148091C30F882319F00E94E47603
:10A1F0001DC0E8E1F6E18491FB83EA83882371F0D6
:10A20000082E000C990B0E947C752A813B812F5FE0
:10A210003F4F3B832A83F9018491F0CF8DE090E09A
:10A220000E947C758AE090E00E947C7580911E14EB
:10A230000AC0891751F01092201410922114109224
:10A2400022141092231480931F1480917C16843062
:10A2500010F40E945A3F0E944BB4C090FE0AD09066
:10A26000FF0AE090000BF090010BC114D104E1044F
:10A27000F10481F10091FA0A1091FB0A2091FC0A85
:10A280003091FD0A0C0D1D1D2E1D3F1D4B015C0163
:10A29000801A910AA20AB30AB7FC1CC0E9EDF9E1E1
:10A2A00084919F012F5F3F4F3B832A83882329F0AE
:10A2B0000E94D63EEA81FB81F3CF60916B167091CC
:10A2C0006C168EE496E1FCDB8AE00E94D63E85E4C3
:10A2D00096E181C0C0902302D0902402E090250234
:10A2E000F0902602C114D104E104F104E9F13091A7
:10A2F000450F2091460F321749F06093FA0A709388
:10A30000FB0A8093FC0A9093FD0A2EC00091FA0A82
:10A310001091FB0A2091FC0A3091FD0A0C0D1D1DC5
:10A320002E1D3F1DDC01CB01801B910BA20BB30B3B
:10A33000B7FD1AC05F9A8091F6038E7F8093F60373
:10A340008A9A479A8091F6038D7F8093F6038091D5
:10A3500008018095817080930601479A8091F603E9
:10A360008B7F8093F603129A80914C0B90914D0B4A
:10A37000909902C0019604C0181619062CF4019792
:10A3800090934D0B80934C0B80914C0B90914D0B07
:10A390008E3E92400CF1E9EDF9E184919F012F5F2F
:10A3A0003F4F3B832A83882329F00E94D63EEA81CF
:10A3B000FB81F3CFE5E2F6E184919F012F5F3F4FF0
:10A3C0003B832A83882329F00E94D63EEA81FB81C1
:10A3D000F3CF8CE196E1E4DD0E944BB40091480B91
:10A3E0001091490B20914A0B30914B0B4B015C01B2
:10A3F000801A910AA20AB30AB7FC4EC08B019C01D5
:10A400000C53164F2F4F3F4F0093480B1093490B9F
:10A4100020934A0B30934B0B4F9BA9C17A9BA7C14A
:10A420002091060120FFA3C12091951521119FC104
:10A43000379B9DC1379B9BC1029B99C10091440BE7
:10A440001091450B2091460B3091470B01151105DA
:10A450002105310599F0DC01CB01801B910BA20B8A
:10A46000B30B80569A4EA109B1098827B7FD839591
:10A470009927AA27BB27682F619501C060E0262F86
:10A4800030E080910201611180958071809300011C
:10A49000B90187E00E944CB39091450F8091460F1F
:10A4A000981791F0E091460F28E5E29FF001112402
:10A4B000E951FB4F60818091460F9091450F9817AD
:10A4C00029F08F5F8F70F9CF6091070470E089E009
:10A4D0000E944CB380919015882309F4F8C0009134
:10A4E00008021091090280900A028C8290900B025F
:10A4F0009A8260910F04709110046E5F7F4F072E57
:10A50000000C880B990B0E94C3C69801A4010E94FD
:10A51000BDC687FDDCC0F090460F212C312CE12C0C
:10A5200019828091450F8F1509F462C08F2D90E03C
:10A5300038E5A32EA89EF001A99EF00D1124EB563C
:10A54000FB4F458956896789708D452B462B472BD4
:10A5500081F4418D528D638D748D452B462B472B95
:10A5600041F4458D568D678D70A1452B462B472BA9
:10A57000D1F128E5B22EB89E9001B99E300D11247C
:10A58000C9018B569B4F6C01FC01618172818381F3
:10A5900094810E9452CD4B015C01F60161A172A130
:10A5A00083A194A10E94C1C62B013C01F60165A1C3
:10A5B00076A187A190A50E94C1C69B01AC01C301F1
:10A5C000B2010E94C3CBA50194010E9422C75B0186
:10A5D0006C0191014E2D59810E940DCD18161CF46D
:10A5E0001501EC2CD98281E08F0D8F70F82E99CF58
:10A5F00020910C0230910D0240910E0250910F02F9
:10A60000B1018E2D99810E9422C798014C815A81F7
:10A610000E94E7CA6B017C019B01AC01B8018C81EF
:10A620009A810E940DCD1816ACF000910402109191
:10A630000502809006028C82909007029A8298010F
:10A64000A401B601C7010E940DCD18161CF08601A9
:10A65000EC82FA82C090400BD090410BE090420B0C
:10A66000F090430B98014C815A81C701B6010E94BA
:10A670000DCD1816D4F420E037ED43EA5CE3B801C1
:10A680008C819A810E9422C74B015C0128E431EE43
:10A690004AE75FE3C701B6010E9422C7A501940102
:10A6A0000E94E7CA8B018C839A83C801AC81BA816E
:10A6B0008093400B9093410BA093420BB093430BBC
:10A6C000B801CD010E942BCCCB010E941A740E94CC
:10A6D000F88083EA9FE00E94173AA090060BA982B7
:10A6E000AA2009F44DC00E944BB40091020B1091B6
:10A6F000030B2091040B3091050BDC01CB01801B77
:10A70000910BA20BB30BB7FD3BC00E944BB46B0186
:10A710007C01B9802B2D30E0A8EEB3E00E94D7CAAF
:10A72000C60ED71EE81EF91EC092020BD092030B74
:10A73000E092040BF092050B0E943A7B8AE00F90A6
:10A740000F900F900F90DF91CF911F910F91FF907D
:10A75000EF90DF90CF90BF90AF909F908F907F90C1
:10A760006F905F904F903F902F900C94D63E6093E7
:10A77000440B7093450B8093460B9093470B5ECE32
:10A780000F900F900F900F90DF91CF911F910F912D
:10A79000FF90EF90DF90CF90BF90AF909F908F9001
:10A7A0007F906F905F904F903F902F9008952F92E1
:10A7B0003F924F925F926F927F928F929F92AF9251
:10A7C000BF92CF92DF92EF92FF920F931F93CF939E
:10A7D000DF93CDB7DEB7CC54D1090FB6F894DEBF06
:10A7E0000FBECDBF80912102882319F084E19BE048
:10A7F000E9D980918B0B83FDA9C0C090200BD0902C
:10A80000210BE090220BF090230B20910304309158
:10A8100004044091050450910604C701B6010E944A
:10A82000BDC6882309F492C080918A0B811133C080
:10A83000609111047091120480911304909114049A
:10A840000E942BCC20913702309138026217730797
:10A8500014F5C0920304D0920404E0920504F0922F
:10A860000604EEEEF9E184917F019FEFE91AF90AFF
:10A87000882321F00E94D63EF701F5CFECEBF5E1FD
:10A8800084917F01AFEFEA1AFA0A882321F00E942F
:10A89000D63EF701F5CF8090200B9090210BA09031
:10A8A000220BB090230B20910304309104044091BB
:10A8B000050450910604C501B4010E94E6CA6B016B
:10A8C0007C0120E030E0A9010E940DCD87FF04C08B
:10A8D000F7FAF094F7F8F094E091F80AB4E0EB9FFF
:10A8E000F0011124ED5CFD4F2081318142815381C3
:10A8F000C701B6010E9422C720E030E048E453E4DB
:10A900000E940DCD181614F5809203049092040451
:10A91000A0920504B0920604EEEEF9E184917F0165
:10A920009FEFE91AF90A882321F00E94D63EF70129
:10A93000F5CFEDE9F5E184917F01AFEFEA1AFA0A6C
:10A94000882321F00E94D63EF701F5CF809175163D
:10A950006090020270900302C090140BD090150B0F
:10A96000E090160BF090170B8090180B9090190B3D
:10A97000A0901A0BB0901B0B882309F481C2209081
:10A98000761630907716409078165090791620E021
:10A9900030E0A901C201B1010E94BDC6882379F04F
:10A9A00020911C0B30911D0B40911E0B50911F0BE1
:10A9B000C201B1010E940DCD18160CF061C2B301A5
:10A9C000770C880B990B0E94C3C620914B023091E3
:10A9D0004C0240914D0250914E020E9422C72AE043
:10A9E00037ED43E25CE30E9422C76DA77EA78FA7E5
:10A9F00098AB2091F7033091F8034091F9035091FF
:10AA0000FA03C701B6010E94E6CA2B013C0120915E
:10AA1000FB033091FC034091FD035091FE03C501FF
:10AA2000B4010E94E6CA25966CAF7DAF8EAF9FAF92
:10AA3000259720E030E0A901C301B2010E94BDC604
:10AA4000811141C020E030E0A90125966CAD7DADBB
:10AA50008EAD9FAD25970E94BDC6811134C0709008
:10AA6000F80A19AA1AAA1BAA1CAAC982DA82EB82BE
:10AA7000FC828D829E82AF82B88680911C0B909161
:10AA80001D0BA0911E0BB0911F0B89879A87AB8776
:10AA9000BC87AE01475F5F4FBE016B5F7F4FCE014A
:10AAA00001960E941DA9FE01F1966F01E72C8E010F
:10AAB000035D1F4F20E23BE0AE01475F5F4FBE01E9
:10AAC0006B5F7F4F2AC22091FF03309100044091B9
:10AAD00001045091020460911C0B70911D0B809138
:10AAE0001E0B90911F0B0E94E6CA29966CAF7DAF9A
:10AAF0008EAF9FAF299720910304309104044091B9
:10AB00000504509106046091200B7091210B8091F7
:10AB1000220B9091230B0E94E6CA21966CAF7DAF69
:10AB20008EAF9FAF2197A3019201C301B2010E9492
:10AB300022C76B017C0125962CAD3DAD4EAD5FADBE
:10AB40002597CA01B9010E9422C79B01AC01C70128
:10AB5000B6010E94E7CA6B017C0129962CAD3DAD80
:10AB60004EAD5FAD2997CA01B9010E9422C79B0172
:10AB7000AC01C701B6010E94E7CA0E9452CD6B0129
:10AB80007C012DEB37E346E855E30E94BDC687FF05
:10AB900017C020E030E0A90121966CAD7DAD8EADEF
:10ABA0009FAD21970E940DCD2196CCACDDACEEACD3
:10ABB000FFAC219787FF04C0F7FAF094F7F8F09400
:10ABC0002DEB37E346E855E3C701B6010E94BDC649
:10ABD00087FDA6C120E030E040EA50E4C701B6019D
:10ABE0000E94C3CB0E9430CC1B01672B19F4222496
:10ABF0002394312CB10180E090E00E94C1C69B01FA
:10AC0000AC0160E070E080E89FE30E94C3CB4B01A1
:10AC10005C019B01AC01C701B6010E9422C72D96C1
:10AC20006CAF7DAF8EAF9FAF2D97A5019401C3018F
:10AC3000B2010E9422C7698B7A8B8B8B9C8BA501FA
:10AC4000940125966CAD7DAD8EAD9FAD25970E948C
:10AC500022C76D8B7E8B8F8B988FA50194012996CF
:10AC60006CAD7DAD8EAD9FAD29970E9422C7698FD7
:10AC70007A8F8B8F9C8FA501940121966CAD7DAD51
:10AC80008EAD9FAD21970E9422C76D8F7E8F8F8FD3
:10AC900098A380E1E7EFF3E0DE01119601900D92B9
:10ACA0008A95E1F799249394F1E02F1A310809F07D
:10ACB0004BC0E090F80A2D968CAD9DADAEADBFAD0A
:10ACC0002D9789AF9AAFABAFBCAF8091140B909129
:10ACD000150BA091160BB091170B89A39AA3ABA3E8
:10ACE000BCA38091180B9091190BA0911A0BB091F5
:10ACF0001B0B8DA39EA3AFA3B8A780911C0B9091B3
:10AD00001D0BA0911E0BB0911F0B89A79AA7ABA793
:10AD1000BCA7AE01475D5F4FBE016B5D7F4FCE01AB
:10AD200081960E941DA9DE01D9966D018E01035DF9
:10AD30001F4F20E23BE0AE01475D5F4FBE016B5D00
:10AD40007F4FCE018196EBC08091340B811112C0F0
:10AD50000E944BB4DC01CB0188539F4FAF4FBF4FD4
:10AD60008093300B9093310BA093320BB093330B45
:10AD70009092340B0E94F8800E944BB4C090300B2C
:10AD8000D090310BE090320BF090330BDC01CB0113
:10AD90008C199D09AE09BF09B7FD11C00E944BB4C3
:10ADA000DC01CB0188539F4FAF4FBF4F8093300BD7
:10ADB0009093310BA093320BB093330B38D96E01C3
:10ADC000B1E1CB0ED11CFE0131967F015601D601B7
:10ADD0002D913D914D915D916D01F70160817181E2
:10ADE000828193810E94E7CAD7016D937D938D93F1
:10ADF0009D937D01AA16BB0651F7E090F80A2D96A7
:10AE00008CAD9DADAEADBFAD2D978DAB9EABAFAB59
:10AE1000B8AF89819A81AB81BC8189A39AA3ABA386
:10AE2000BCA38D819E81AF81B8858DA39EA3AFA366
:10AE3000B8A789859A85AB85BC8589A79AA7ABA752
:10AE4000BCA7AE01475D5F4FBE016B5D7F4FCE017A
:10AE500081960E941DA9DE01D5966D018E01035DCC
:10AE60001F4F9E01235F3F4FAE01475D5F4FBE0105
:10AE70006B5D7F4FCE018196D6D0811115CF19CF52
:10AE8000B301770C880B990B0E94C3C620914B022B
:10AE900030914C0240914D0250914E020E9422C7C7
:10AEA0002AE037ED43E25CE30E9422C769AB7AAB4C
:10AEB0008BAB9CAB7090F80A80911C0B90911D0B92
:10AEC000A0911E0BB0911F0BC982DA82EB82FC822B
:10AED000898A9A8AAB8ABC8A89A39AA3ABA3BCA3AA
:10AEE0001DA61EA61FA618AAAE014F5D5F4FBE018C
:10AEF0006F5E7F4FCE0101960E941DA9FE01BD9697
:10AF00006F01E72C8E010F5C1F4F20E23BE0AE018A
:10AF10004F5D5F4FBE016F5E7F4FCE01019683D0C4
:10AF200080E1E4E1FBE0A7EFB3E001900D928A95A8
:10AF3000E1F7C45BDF4F0FB6F894DEBF0FBECDBFA5
:10AF4000DF91CF911F910F91FF90EF90DF90CF9005
:10AF5000BF90AF909F908F907F906F905F904F9039
:10AF60003F902F900895CF93DF9380E00E949BA4A1
:10AF7000CCEEDAE0688379838A839B8381E00E9448
:10AF80009BA46C837D838E839F8382E00E949BA41D
:10AF9000688779878A879B87DF91CF910895CF93C0
:10AFA000DF93E0917A16F0E0E155F44F8081882339
:10AFB00081F0EAE9F5E18491EF012196882321F0FF
:10AFC0000E94D63EFE01F7CF8AE0DF91CF910C942C
:10AFD000D63EDF91CF910895CF93DF938091EA0A17
:10AFE0008093EB0AE1E9F5E18491EF012196882352
:10AFF00021F00E94D63EFE01F7CF809188169091F5
:10B000008916A0918A16B0918B16BC01CD016F5F95
:10B010007F4F8F4F9F4F0E945D428AE00E94D63E35
:10B02000DF91CF91BCCF2F923F924F925F926F9260
:10B030007F928F929F92AF92BF92CF92DF92EF92C8
:10B04000FF920F931F93CF93DF93CDB7DEB7C8570F
:10B05000D1090FB6F894DEBF0FBECDBFE0919215B7
:10B06000F0919315EF2B11F00C94DC602896DFAE75
:10B07000CEAE28976E2C79016A015B01FC0120811C
:10B080003181428153816C962CAF3DAF4EAF5FAFA3
:10B090006C972091E3163091E4164091E51650919B
:10B0A000E6166C966CAD7DAD8EAD9FAD6C970E9433
:10B0B00022C70E9418CDE0966CAF7DAF8EAF9FAFD8
:10B0C000E097D5018D919D910D90BC91A02DA096FA
:10B0D0008CAF9DAFAEAFBFAFA0972091E716309178
:10B0E000E8164091E9165091EA16BC01CD010E9484
:10B0F00022C70E9418CDE4966CAF7DAF8EAF9FAF94
:10B10000E497D6012D913D914D915C91A4962CAF81
:10B110003DAF4EAF5FAFA4972091EB163091EC1688
:10B120004091ED165091EE16A4966CAD7DAD8EADAE
:10B130009FADA4970E9422C70E9418CDE8966CAFDD
:10B140007DAF8EAF9FAFE897D7012D913D914D9187
:10B150005C9122962CAF3DAF4EAF5FAF229720910E
:10B16000EF163091F0164091F1165091F21622969A
:10B170006CAD7DAD8EAD9FAD22970E9422C70E941F
:10B1800018CD60966CAF7DAF8EAF9FAF609780910A
:10B190008B0B83FF1CC060962CAD3DAD4EAD5FADFB
:10B1A00060972093770F3093780F4093790F5093E7
:10B1B0007A0F22968CAD9DADAEADBFAD2297809338
:10B1C000670F9093680FA093690FB0936A0FD8012F
:10B1D000BC91BDA3F801F181F9ABD8011296BC91E5
:10B1E000BEABF801F381FAAF8091450F9091460F05
:10B1F000891B8F708F3019F40E941750F5CF009182
:10B20000450FE9960FAFE9978091450F082F10E0A1
:10B210001CA30BA380916B0F90916C0FA0916D0FED
:10B22000B0916E0FE0968CAC9DACAEACBFACE0972D
:10B23000881A990AAA0ABB0A80916F0F9091700F21
:10B24000A091710FB091720FE4962CAC3DAC4EAC56
:10B250005FACE497281A390A4A0A5B0A8091730F97
:10B260009091740FA091750FB091760FE8962CAD68
:10B270003DAD4EAD5FADE897281B390B4A0B5B0B1C
:10B280002DA73EA74FA758AB8091770F9091780FCD
:10B29000A091790FB0917A0F60960CAD1DAD2EADD7
:10B2A0003FAD6097081B190B2A0B3B0B09A71AA788
:10B2B0002BA73CA7012B022B032B09F4BCC08091C8
:10B2C0008A0B81114BC0609111047091120480911E
:10B2D0001304909114040E942BCC209137023091DA
:10B2E0003802621773070CF039C060962CAD3DAD83
:10B2F0004EAD5FAD60972093770F3093780F4093FA
:10B30000790F50937A0F22968CAD9DADAEADBFAD47
:10B3100022978093670F9093680FA093690FB09363
:10B320006A0FEEEEF9E184918F010F5F1F4F8111DB
:10B3300003C0E7E1F7E104C00E94D63EF801F3CF75
:10B3400084918F010F5F1F4F882321F00E94D63E0A
:10B35000F801F6CF19A61AA61BA61CA694E0699EB2
:10B36000800111240D5C1D4F69A57AA58BA59CA5B4
:10B370000E94C3C6D8012D913D914D915C910E94D0
:10B3800022C76B017C0120E030E0A9010E940DCDB5
:10B3900087FF04C0F7FAF094F7F8F0946091EF1685
:10B3A0007091F0168091F1169091F2160E942BCCBC
:10B3B0009B01AC01A8ECB0E00E94CDCA0E94C3C6BC
:10B3C000A70196010E94BDC687FF39C060960CADEB
:10B3D0001DAD2EAD3FAD60970093770F1093780FA2
:10B3E0002093790F30937A0F22962CAD3DAD4EAD60
:10B3F0005FAD22972093670F3093680F4093690FDA
:10B4000050936A0FEEEEF9E184918F010F5F1F4FA9
:10B41000811103C0E8EFF6E104C00E94D63EF801B6
:10B42000F3CF84918F010F5F1F4F882321F00E947B
:10B43000D63EF801F6CF19A61AA61BA61CA6D50162
:10B44000C4018827B7FD83959927AA27BB27782EA3
:10B4500057FE03C0382F3260732E8DA59EA5AFA571
:10B46000B8A9B7FF03C0972D9460792E09A51AA536
:10B470002BA53CA537FF03C0172D1860712E24E0C3
:10B48000629E800111240D5C1D4F69A57AA58BA5D4
:10B490009CA50E94C3C6D8012D913D914D915C9110
:10B4A0000E9422C76B017C0120E030E0A9010E94CC
:10B4B0000DCD87FF04C0C701B601905802C0C70177
:10B4C000B60120E030E040E05FE30E94E7CA0E945E
:10B4D00030CC6AAB7BAB8CAB9DAB88E50BA11CA1E0
:10B4E000809FF001819FF00D1124EB56FB4F1082DD
:10B4F00076AAB501A401B7FE07C044275527BA01B3
:10B50000481959096A097B0988E50BA11CA1809F8C
:10B51000F001819FF00D1124EB56FB4F458B568BAC
:10B52000678B708F2C962CAE3DAE4EAE5FAE2C97D7
:10B5300057FE0DC088279927DC0182199309A409B9
:10B54000B5092C968CAF9DAFAEAFBFAF2C9728E559
:10B550000BA11CA1209FF001219FF00D1124EB569F
:10B56000FB4F2C968CAD9DADAEADBFAD2C97818FB2
:10B57000928FA38FB48F0DA51EA52FA538A937FFD5
:10B5800007C030952095109501951F4F2F4F3F4FC5
:10B59000E8E57E2EABA1BCA17A9EF0017B9EF00D6A
:10B5A0001124EB56FB4F058F168F278F30A38AA9E6
:10B5B0009BA9ACA9BDA981A392A3A3A3B4A32396DD
:10B5C0004FAF2397752EF62FE72F2C968CAD9DADA0
:10B5D000AEADBFAD2C97481759076A077B0778F4C3
:10B5E00029969FAD299723969FAF23972A967FACE4
:10B5F0002A972B96FFAD2B972C96EFAD2C97239681
:10B600008FAD2397972DAF2FBE2F80179107A207DD
:10B61000B30710F4D901C8010AA91BA92CA93DA997
:10B6200080179107A207B30710F4D901C80128E5D4
:10B630000BA11CA1209FF001219FF00D1124EB56BE
:10B64000FB4F85A396A3A7A3B0A70697A105B105B5
:10B6500008F4ABC5DF01AE5ABF4F8091070490914B
:10B6600008048D939C9361A6452B462B472B09F02C
:10B670005F9888E50BA11CA1809FF001819FF00DD0
:10B680001124EB56FB4F818D928DA38DB48D892BA8
:10B690008A2B8B2B11F08A98479888E50BA11CA167
:10B6A000809FF001819FF00D1124EB56FB4F858D9B
:10B6B000968DA78DB0A1892B8A2B8B2B31F0809191
:10B6C000080181708093060147982AA93BA94CA9DB
:10B6D0005DA9232B242B252B09F470C58091900B99
:10B6E000882319F081508093900B611004C0129848
:10B6F00080E28093900B6090860B7090870B009196
:10B70000880B1091890B9301A8016DA179A98EA9CD
:10B710009AAD0E94BDC687FF04C06DA279AA0EAB88
:10B720001AAFC501B4010E94C3C62091D31630914F
:10B73000D4164091D5165091D6160E9422C726964F
:10B740006CAF7DAF8EAF9FAF2697698B7A8B8B8B5B
:10B750009C8BC201B1010E94C3C62091D7163091C3
:10B76000D8164091D9165091DA160E9422C72B01A3
:10B770003C016D8B7E8B8F8B988F6DA57EA58FA5E1
:10B7800098A90E94C3C62091DB163091DC16409127
:10B79000DD165091DE160E9422C74B015C01698FB5
:10B7A0007A8F8B8F9C8F2091DF163091E01640911D
:10B7B000E1165091E216C701B6010E9422C76B0143
:10B7C0007C016D8F7E8F8F8F98A388E50BA11CA1C4
:10B7D000809FF001819FF00D1124EB56FB4F2589CE
:10B7E00036894789508D2DA73EA74FA758AB2630E5
:10B7F00031054105510508F4EAC42896AEADBFAD48
:10B800002897CD90DD90ED90FC9020E030E0A901EC
:10B81000C701B6010E94BDC68111F8C426962CADA1
:10B820003DAD4EAD5FAD2697CA01B9010E9422C75A
:10B830006B017C01A3019201C301B2010E9422C7E6
:10B840009B01AC01C701B6010E94E7CA6B017C01F4
:10B85000A5019401C501B4010E9422C79B01AC015E
:10B86000C701B6010E94E7CA0E9452CD28E50BA18C
:10B870001CA1209FF001219FF00D1124EB56FB4FDE
:10B88000658776878787908B88E50BA11CA1809FB1
:10B89000F001819FF00D1124EB56FB4F4584568437
:10B8A00067847088A301920160E070E080E89FE304
:10B8B0000E94C3CB64966CAF7DAF8EAF9FAF649791
:10B8C0002DA139A94EA95AAD0E9422C74B015C0196
:10B8D0008091450F9091430F891B8F7027968FAFF2
:10B8E0002797A501940160E074E284E799E40E943F
:10B8F000C3CB0E9418CD6B017C0127968FAD279793
:10B900008250863008F491C4A5019401C301B201AC
:10B910000E9422C79B01AC010E9422C768966CAFAF
:10B920007DAF8EAF9FAF689788E5ABA1BCA18A9F22
:10B9300080018B9F100D11240B561B4F68962CAD68
:10B940003DAD4EAD5FAD6897D80111962D933D93F7
:10B950004D935C93149795962D913D914D915C91EB
:10B9600098972EAB3FAB48AF59AFCA01B9010E94BF
:10B97000C1C66AAF7BAF8CAF9DAF9B01AC01C50167
:10B98000B4010E9422C70E94ADCB0E9430CCA89681
:10B990006CAF7DAF8EAF9FAFA897F801EE5BFF4F06
:10B9A00060837183828393838E010F5E1F4F2A967B
:10B9B0001FAF0EAF2A970051110924961FAF0EAF8B
:10B9C00024970EE61BE0AC961FAF0EAFAC978E012E
:10B9D0000F5D1F4F1AA309A324960EAD1FAD249728
:10B9E000AA961FAF0EAFAA97312C212C10E81DA3E9
:10B9F0000FE309AB2A96AEADBFAD2A972D913D91CD
:10BA00004D915D912A96BFAFAEAF2A97C501B401A3
:10BA10000E9422C76B017C01AA96EEADFFADAA97EA
:10BA20006193719381939193AA96FFAFEEAFAA971A
:10BA300020E030E0A9010E940DCD87FF04C0F7FA95
:10BA4000F094F7F8F094AC96AEADBFADAC974D90D6
:10BA50005D906D907D90AC96BFAFAEAFAC97A701F7
:10BA60009601C301B2010E94BDC687FD18C409A199
:10BA70001AA12A962EAD3FAD2A970217130709F097
:10BA8000B9CF20E030E040E85FE3632D722D8DA157
:10BA900099A90E94BDC687FF58C07E0131E1E30E1F
:10BAA000F11C24960EAD1FAD2497232D322D4DA1F0
:10BAB00059A9D8016D917D918D919C910E9422C7C9
:10BAC000F80161937193819391938F01EE16FF06B4
:10BAD00061F728E50BA11CA1209FC001219F900DBB
:10BAE00011249C012B563B4F790189010E5B1F4F9E
:10BAF000A8966CAD7DAD8EAD9FADA8970E94C1C6D6
:10BB0000232D322D4DA159A90E9422C70E9430CC6D
:10BB1000D8016D937D938D939C931397232D322D94
:10BB20004DA159A9632D722D8DA199A90E9422C7FB
:10BB300068962CAD3DAD4EAD5FAD68970E9422C7B3
:10BB4000F70161837283838394832AAD3BAD4CAD4F
:10BB50005DAD64966CAD7DAD8EAD9FAD64970E947A
:10BB600022C76DA37EA38FA398A70DA51EA52FA501
:10BB700038A9012B022B032B09F0A9C388E52BA1BF
:10BB80003CA1829F8001839F100D11240B561B4FF7
:10BB9000F801818D928DA38DB48D892B8A2B8B2BEF
:10BBA00009F095C3858D968DA78DB0A1892B8A2B21
:10BBB0008B2B09F08CC320916A0B30916B0B409159
:10BBC0006C0B50916D0B6DA17EA18FA198A50E9469
:10BBD00022C70E94ADCB0E9430CC2B013C01D80182
:10BBE000D7961C9288E52BA13CA1829F8001839F60
:10BBF000100D11240B561B4FF801E25BFF4F4082E2
:10BC0000518262827382C301B2010E94C1C66B017C
:10BC10007C012DA13EA14FA158A50E94C3CB6AAFC4
:10BC20007BAF8CAF9DAFD80151966D937D938D9373
:10BC30009C9354972DEB37E346E051E4C701B601DE
:10BC40000E9422C70E9430CCF80162AB73AB84AB78
:10BC500095AB87A9882371F1FE9620915E0B3091F8
:10BC60005F0B4091600B5091610B6081718182810B
:10BC700093810E9422C72AAD3BAD4CAD5DAD0E94C1
:10BC800022C72091EF163091F0164091F116509195
:10BC9000F2160E9422C79B01AC0160E074E284EFBF
:10BCA00099E40E94C3CB0E9430CCD801D9967C93F2
:10BCB0006E93D89788E50BA11CA1809FF001819F0E
:10BCC000F00D1124EB56FB4F2181328143815481C9
:10BCD0002C962CAF3DAF4EAF5FAF2C97CA01B90188
:10BCE0000E9452CD362E272E8C014EE45BE06296E8
:10BCF0005FAF4EAF62973E0151E1650E711C8EE45D
:10BD00009BE09FAB8EAB24964EAC5FAC249739A6DC
:10BD10002DA60DA319AB1AAAD201CD90DD90ED90FE
:10BD2000FD902D0120E030E0A901C701B6010E947D
:10BD30000DCD87FF04C0F7FAF094F7F8F094EEA960
:10BD4000FFA981909190A190B190FFABEEABA701BC
:10BD50009601C501B4010E94BDC687FDD4C5641417
:10BD60007504D1F627965FAD2797552309F444C68D
:10BD7000C090470FD090480FE090490FF0904A0FC5
:10BD80002DEB37E346E855E3C701B6010E94BDC677
:10BD900087FD32C6C701B6010E9452CD6B017C01FE
:10BDA0009B01AC01632D722DC8010E94BDC687FDA9
:10BDB00003C03C2C2D2C87019601A701632D722D09
:10BDC000C8010E94C3CB68966CAF7DAF8EAF9FAFAA
:10BDD00068978BE49FE028969FAF8EAF289720E06E
:10BDE00030E040E85FE32AAB3BAB4CAB5DAB1EAA57
:10BDF0002896AEADBFAD28972D913D914D915D91A7
:10BE00002896BFAFAEAF289768966CAD7DAD8EAD6E
:10BE10009FAD68970E9422C74B015C012496EEAD4E
:10BE2000FFAD2497C190D190E190F1902496FFAF9F
:10BE3000EEAF2497FEA9FF2391F02AA93BA94CA9B4
:10BE40005DA90E9422C74B015C012AA93BA94CA90C
:10BE50005DA9C701B6010E9422C76B017C01A70141
:10BE60009601C501B4010E940DCD20E030E0A9018A
:10BE700018160CF08EC5C701B6010E940DCD18161C
:10BE80000CF482C520E030E0A901C501B4010E9494
:10BE9000BDC687FD79C52601370177FA709477F81A
:10BEA0007094A3019201C501B4010E940DCD181632
:10BEB00014F4240135016296AEADBFAD6297CD900A
:10BEC000DD90ED90FD906296BFAFAEAF6297A3019B
:10BED0009201C701B6010E94BDC687FF15C0A3012C
:10BEE0009201C701B6010E94C3CB9B01AC016AA9B4
:10BEF0007BA98CA99DA90E9422C76AAB7BAB8CABA6
:10BF00009DABBEA9BF5FBEABEBE5FFE028962EADB3
:10BF10003FAD2897E217F30709F06ACF3EA9332314
:10BF200061F02AA93BA94CA95DA9632D722DC80116
:10BF30000E9422C7362E272E8C0124EA30E74DE7D7
:10BF40005FE3632D722DC8010E9422C76B017C0143
:10BF500020918C0B30918D0B40918E0B50918F0B5B
:10BF60000E94BDC687FD3EC589A59DA5ADA1B9A905
:10BF700080938C0B90938D0BA0938E0BB0938F0BB3
:10BF800028E54BA15CA1249FC001259F900D1124A1
:10BF9000DC01AB56BB4F7D01232D322DA801632D53
:10BFA000722DC8010E9422C7F701618772878387BB
:10BFB00094876AAD7BAD8CAD9DAD90589B01AC0173
:10BFC0000E94E7CAD7011D962D913D914D915C913C
:10BFD00050970E9422C79B01AC016BE077ED83E292
:10BFE0009BE30E94E6CA9B01AC018BE097EDA3E2C4
:10BFF000BBE3F70185839683A783B08710812C96D6
:10C000006CAD7DAD8EAD9FAD2C970E94BDC6181650
:10C010000CF4F7C483E0182B88E52BA13CA1829F88
:10C02000F001839FF00D1124EB56FB4F108380E14C
:10C03000FE013196ABE4BFE001900D928A95E1F7E5
:10C040002C968CAD9DADAEADBFAD2C978093470FB8
:10C050009093480FA093490FB0934A0FE0960CAD10
:10C060001DAD2EAD3FADE09700936B0F10936C0F9D
:10C0700020936D0F30936E0FE4962CAD3DAD4EAD19
:10C080005FADE49720936F0F3093700F4093710F63
:10C090005093720FE8968CAD9DADAEADBFADE897F5
:10C0A0008093730F9093740FA093750FB093760FD6
:10C0B00060960CAD1DAD2EAD3FAD60970093770F30
:10C0C0001093780F2093790F30937A0F6C962CADE4
:10C0D0003DAD4EAD5FAD6C9720935B0F30935C0F21
:10C0E00040935D0F50935E0FA0968CAD9DADAEADAD
:10C0F000BFADA09780935F0F9093600FA093610FE7
:10C10000B093620FA4960CAD1DAD2EAD3FADA497BC
:10C110000093630F1093640F2093650F3093660FA5
:10C1200022962CAD3DAD4EAD5FAD22972093670FAB
:10C130003093680F4093690F50936A0F9091450FA9
:10C140008091460F981303C084E68093420FE996CE
:10C150008FADE9978F5F8F708093450F8091450F6A
:10C160009091440F81508F7089134DC41091460FE8
:10C170001BA30091450F09A728E51BA109A51013D2
:10C18000CDC4812C912CA12CB12C1DA61DA219AAC5
:10C190001EAE212C312C00E010E029A53BA1231379
:10C1A000CAC42114310409F079C580916F008260FE
:10C1B00080936F0081E0E2C680E0E0C66090820B71
:10C1C0007090830B0091840B1091850B9CCA818D1C
:10C1D000928DA38DB48D0697A105B10508F00DCB06
:10C1E000858D968DA78DB0A10697A105B10508F0A4
:10C1F00004CB20E030E0A901C701B6010E940DCDBB
:10C2000087FF04C0F7FAF094F7F8F09488E50BA1E3
:10C210001CA1809FF001819FF00D1124EB56FB4F74
:10C22000C586D686E786F08A2FCB80917E0B9091CB
:10C230007F0BA091800BB091810BC816D906EA063E
:10C24000FB0608F061CB8C199D09AE09BF09BC0142
:10C25000CD01660F771F881F991F27964FAD27972F
:10C26000042F10E020E030E0A90198010E94ABCA41
:10C27000CA01B9010E94C1C60E9418CD6C0D7D1D76
:10C280008E1D9F1D0E94C1C69B01AC0160E074E23F
:10C2900084E799E40E94C3CB4B015C0135CBA70135
:10C2A0009601C301B2010E94C3CB7B018C019B01AB
:10C2B000AC01632D722D8DA199A90E940DCD181688
:10C2C0000CF0D5CB3E2C2F2C0DA319ABD0CB0AA94B
:10C2D0001BA92CA93DA9012B022B032B49F020916E
:10C2E000660B3091670B4091680B5091690B08C049
:10C2F0002091620B3091630B4091640B5091650B60
:10C300006DA17EA18FA198A50E9422C70E94ADCBEE
:10C310000E9430CC2B013C012AA93BA94CA95DA964
:10C32000232B242B252BC9F020E030E0A9016091BC
:10C330005E0B70915F0B8091600B9091610B0E947E
:10C34000BDC6882351F081E009A51AA52BA53CA5FF
:10C3500010161106120613060CF080E098E52BA1CA
:10C360003CA1929F8001939F100D11240B561B4FEF
:10C37000D801D7968C93882309F4B2C020915B0F23
:10C3800030915C0F40915D0F50915E0F6C966CADDB
:10C390007DAD8EAD9FAD6C970E94E6CA69A77AA766
:10C3A0008BA79CA720915F0F3091600F4091610F88
:10C3B0005091620FA0966CAD7DAD8EAD9FADA097F4
:10C3C0000E94E6CA4B015C012091630F3091640F1B
:10C3D0004091650F5091660FA4966CAD7DAD8EAD0A
:10C3E0009FADA4970E94E6CA6B017C0129A53AA5DE
:10C3F0004BA55CA5CA01B9010E9422C769A77AA70B
:10C400008BA79CA7A5019401C501B4010E9422C776
:10C410009B01AC0169A57AA58BA59CA50E94E7CAE2
:10C420004B015C01A7019601C701B6010E9422C71A
:10C430009B01AC01C501B4010E94E7CA0E9452CD24
:10C440006B017C012091670F3091680F4091690F5B
:10C4500050916A0F22966CAD7DAD8EAD9FAD229747
:10C460000E94E6CAA70196010E94C3CB6B017C0122
:10C47000F801FE96608371838283938320E030E02D
:10C4800040E450E40E940DCD18161CF4F80117AAE0
:10C4900027C020915E0B30915F0B4091600B509153
:10C4A000610BC701B6010E9422C79B01AC016091DC
:10C4B0005A0B70915B0B80915C0B90915D0B0E940D
:10C4C000C3CB2DA13EA14FA158A50E9422C70E9417
:10C4D00030CC641575058605970510F42B013C01D9
:10C4E0008091AF169091B016A091B116B091B2168E
:10C4F0000EA91FA928AD39AD80179107A207B30770
:10C5000008F4DFC02DA53EA54FA558A9232B242B49
:10C51000252B41F16091B3167091B4168091B51638
:10C520009091B6166415750586059705D8F42EA961
:10C530003FA948AD59AD0E949CCA6B017C012DA555
:10C540003EA54FA558A9C301B2010E949CCAC616B8
:10C55000D706E806F90630F4C701B6010E94ABCA57
:10C5600029013A0188E50BA11CA1809FF001819F60
:10C57000F00D1124EB56FB4FC18CD28CE38CF48C64
:10C58000C114D104E104F10431F16091B716709146
:10C59000B8168091B9169091BA166415750586057E
:10C5A0009705C8F42EA93FA948AD59AD0E949CCA71
:10C5B0004B015C01A7019601C301B2010E949CCA14
:10C5C00086169706A806B90630F4C501B4010E9484
:10C5D000ABCA29013A0188E50BA11CA1809FF0019B
:10C5E000819FF00D1124EB56FB4FC58CD68CE78C48
:10C5F000F0A0C114D104E104F10431F16091BB1643
:10C600007091BC168091BD169091BE16641575058B
:10C6100086059705C8F42EA93FA948AD59AD0E94DB
:10C620009CCA4B015C01A7019601C301B2010E94A3
:10C630009CCA86169706A806B90630F4C501B4014F
:10C640000E94ABCA29013A0188E50BA11CA1809F79
:10C65000F001819FF00D1124EB56FB4FC1A0D2A039
:10C66000E3A0F4A0C114D104E104F10409F4BACAAE
:10C670006091BF167091C0168091C1169091C2163C
:10C68000641575058605970508F0ACCA2EA93FA963
:10C6900048AD59AD0E949CCA4B015C01A7019601AF
:10C6A000C301B2010E949CCA86169706A806B90665
:10C6B00008F098CAC501B4010E94ABCA29013A0129
:10C6C00091CA2DA53EA54FA558A9232B242B252B78
:10C6D000C9F16091B3167091B4168091B51690911E
:10C6E000B616641575058605970560F50E94C1C6E6
:10C6F0002AAD3BAD4CAD5DAD0E9422C76B017C0104
:10C700006DA57EA58FA598A90E94C1C64B015C01AD
:10C71000C301B2010E94C1C6A50194010E9422C7B3
:10C720009B01AC01C701B6010E94BDC687FF0AC0CC
:10C73000A5019401C701B6010E94C3CB0E9430CC71
:10C740002B013C0188E50BA11CA1809FF001819F7A
:10C75000F00D1124EB56FB4F818C928CA38CB48C82
:10C7600081149104A104B104B9F16091B7167091DC
:10C77000B8168091B9169091BA166415750586059C
:10C78000970550F50E94C1C62AAD3BAD4CAD5DADDD
:10C790000E9422C76B017C01C501B4010E94C1C681
:10C7A0004B015C01C301B2010E94C1C6A501940105
:10C7B0000E9422C79B01AC01C701B6010E94BDC601
:10C7C00087FF0AC0A5019401C701B6010E94C3CB2F
:10C7D0000E9430CC2B013C0188E50BA11CA1809F5D
:10C7E000F001819FF00D1124EB56FB4F858C968C48
:10C7F000A78CB0A081149104A104B104B9F1609197
:10C80000BB167091BC168091BD169091BE16641532
:10C8100075058605970550F50E94C1C62AAD3BAD4A
:10C820004CAD5DAD0E9422C76B017C01C501B40116
:10C830000E94C1C64B015C01C301B2010E94C1C686
:10C84000A50194010E9422C79B01AC01C701B6015A
:10C850000E94BDC687FF0AC0A5019401C701B601A9
:10C860000E94C3CB0E9430CC2B013C0188E50BA178
:10C870001CA1809FF001819FF00D1124EB56FB4F0E
:10C88000C1A0D2A0E3A0F4A0C114D104E104F1043A
:10C8900009F4A8C96091BF167091C0168091C116A5
:10C8A0009091C216641575058605970508F09AC91A
:10C8B0000E94C1C62AAD3BAD4CAD5DAD0E9422C702
:10C8C0004B015C01C701B6010E94C1C66B017C012E
:10C8D000C301B2010E94C1C6A70196010E9422C7EE
:10C8E0009B01AC01C501B4010E94BDC687FF7AC996
:10C8F000A7019601C501B4010E94C3CB0E9430CCB0
:10C900002B013C016FC9FAA9FF2331F1A501940164
:10C91000632D722DC8010E9422C74B015C0129A51D
:10C920003DA54DA159A9C701B6010E9422C79B018F
:10C93000AC01C501B4010E94BDC687FF22C0A7019A
:10C940009601C501B4010E94C3CB69A77DA78DA341
:10C9500099AB21E02AAB03CAA7019601C501B40136
:10C960000E94C3CB9B01AC0169A57DA58DA199A9AE
:10C970000E9422C769A77DA78DA399AB31E03AAB8E
:10C98000EEC941E04AABEBC9A7019601C501B4016C
:10C9900013C0C701B6010E94BDC687FD09C020E0D3
:10C9A00030E0A901C501B4010E940DCD18164CF468
:10C9B000A5019401C701B6010E94E6CA2B013C0102
:10C9C0007ACA2401350177FA709477F87094A3013C
:10C9D0009201C701B6010E94BDC687FD6CCA26013F
:10C9E000370169CA29A53DA54DA159A9C701B601BD
:10C9F0000E94BDC687FFB8CA39A42DA40DA119A9EC
:10CA0000B3CA81E008CBF090450F8FEF8F0D8F7088
:10CA10008BA3B090440F8091450FB81609F454C011
:10CA2000C12CD12C0BA10B1509F44EC0602E712C1A
:10CA300028E5269D8001279D100D11240B561B4FC4
:10CA4000D8018C9183FD2BC00EAF1AAB01151105D7
:10CA500041F11996BC91B9A7F801F285FDA7D8015B
:10CA60001B96BC91BDA3F801F485F9ABD8011596CE
:10CA70002D903D904D905C901897A201910169A571
:10CA80007DA58DA19F2F0E94BDC6811180C1C114BB
:10CA9000D10439F0F601808180FD79C102C0CEAEAB
:10CAA000DAAA8BA181508F708BA38091440F8B11D8
:10CAB00003C0CEACDAA8B6CF0BA10B1529F081E0EC
:10CAC0008B0D8F70B82EF1CF1091440F1BA3C12C8A
:10CAD000D12C8091450F0BA1801709F447CB802EF4
:10CAE000912C28E5289D8001299D100D11240B56BD
:10CAF0001B4FD8018C9183FD0AC05801C114D10489
:10CB000039F0C6010E947084811102C0BFC1560174
:10CB10008BA18F5F8F708BA36501DBCF802F81503E
:10CB20008F70289FF0011124EB56FB4F908193FFEB
:10CB300028CB89A722CB48E5439FC0011124DC0103
:10CB4000AB56BB4F1D018C9183FD19C015966D919D
:10CB50007D918D919C9118970E9452CDF62EE72ED3
:10CB6000D82EC92E0115110509F48AC0F80180815B
:10CB700080FD0AC0D1018C9180FD06C081C0FDA45A
:10CB8000EDA0D9A8CEAC81C0F801808181608083FE
:10CB9000C8010E94708481116FC0F80161817281A7
:10CBA000838194810E9452CD2B013C019B01AC01F9
:10CBB00060E070E080E89FE30E94C3CB4B015C0122
:10CBC0009B01AC016F2D7E2D8D2D9C2D0E9422C7C7
:10CBD00069837A838B839C832DA53DA149A95EAD92
:10CBE000C501B4010E9422C7698B7A8B8B8B9C8B09
:10CBF000AE014F5F5F4FBE016F5E7F4FC8010E9465
:10CC00006BA5D801D7968C918823B1F120915E0B4A
:10CC100030915F0B4091600B5091610BF801FE96D3
:10CC200060817181828193810E9422C72091EF16D9
:10CC30003091F0164091F1165091F2160E9422C7E1
:10CC40004B015C019B01AC01C301B2010E9422C7F0
:10CC50000E9430CCF80173AF62AFA50194016F2D33
:10CC60007E2D8D2D9C2D0E9422C70E9430CCD80194
:10CC7000DD967C936E93DC97F80180818E7F8083B4
:10CC80008F2C9E2CAD2CBC2C81018BA18F5F8F70C3
:10CC90008BA3FDA6EDA2D9AACEAE7FCAD1018C91FD
:10CCA00081608C93C8010E94708481116BC0F10176
:10CCB00061817281838194810E9452CD6B017C01DC
:10CCC0009B01AC0160E070E080E89FE30E94C3CB71
:10CCD0002B013C012DEC3CEC4CE45DE30E9422C7AF
:10CCE00069837A838B839C839401A501C301B2017C
:10CCF0000E9422C7698B7A8B8B8B9C8BAE014F5F16
:10CD00005F4FBE016F5E7F4FC1010E946BA5D101D5
:10CD1000D7968C918823B1F120915E0B30915F0BF7
:10CD20004091600B5091610BF101FE966081718121
:10CD3000828193810E9422C72091EF163091F016D4
:10CD40004091F1165091F2160E9422C74B015C01EE
:10CD50009B01AC01C701B6010E9422C70E9430CCE2
:10CD6000F10173AF62AF2DEC3CEC4CE45DE3C50127
:10CD7000B4010E9422C70E9430CCD101DD967C9381
:10CD80006E93DC97F10180818E7F80830ECA28E547
:10CD9000269DF001279DF00D1124EB56FB4F80815D
:10CDA00081FD43C0C114D10441F0D6011596CD9048
:10CDB000DD90ED90FC90189708C08BE0C82E87EDB1
:10CDC000D82E83E2E82E8BE3F82EB8E5B69DF0016D
:10CDD000B79DF00D1124EB56FB4F81899289A389F1
:10CDE000B489BC01CD0190589B01AC010E94E7CAF7
:10CDF000F80125853685478550890E9422C79B0109
:10CE0000AC01C701B6010E94E6CAE62E872E982E15
:10CE1000A92E262F372F482F592F69A57DA58DA123
:10CE200099A90E94BDC687FF04C0E9A48DA49DA056
:10CE3000A9A82E2D382D492D5A2DC201B1010E94CD
:10CE4000BDC6882309F42DCEF8E5F69DC001F79DF7
:10CE5000900D11249C012B563B4F6901D9018C91F7
:10CE600081608C93C8010E947084882329F0F601A8
:10CE700080818E7F808315CE8E2D982DA92DBA2D81
:10CE8000F60185839683A783B0870BCED6018C915C
:10CE900081FD52C0D60115962D913D914D915C9129
:10CEA000189729A73AA74BA75CA71501B5E02B0E49
:10CEB000311CF8014580568067807084A30192017F
:10CEC00069A57AA58BA59CA50E94BDC687FF34C025
:10CED000F60181899289A389B489BC01CD0190585A
:10CEE0009B01AC010E94E7CAD6011D962D913D9190
:10CEF0004D915C9150970E9422C79B01AC0169A59E
:10CF00007AA58BA59CA50E94E6CA6B017C019B01BA
:10CF1000AC01C301B2010E940DCD18166CF4D8010A
:10CF20008C9181608C93C5010E9470848823E1F00C
:10CF3000F80180818E7F808318E5189DF001199D8E
:10CF4000F00D1124EB56FB4F218532854385548526
:10CF500065817681878190850E94BDC68111D8CD7B
:10CF60000BA10093440FD4CDD101CD92DD92ED926F
:10CF7000FC9213970BA10093440FDECFC858DF4FEC
:10CF80000FB6F894DEBF0FBECDBFDF91CF911F91DA
:10CF90000F91FF90EF90DF90CF90BF90AF909F9058
:10CFA0008F907F906F905F904F903F902F9008955B
:10CFB0008091450F9091460F891B8F708F3019F427
:10CFC0000E941750F5CF8091450F8F5F8F70E091D1
:10CFD000450F98E59E9FF0011124EB56FB4FDF01B2
:10CFE0001D929A95E9F798E0908340916B0F5091CC
:10CFF0006C0F60916D0F70916E0F458B568B678B28
:10D00000708F40916F0F5091700F6091710F709100
:10D01000720F418F528F638F748F4091730F5091B5
:10D02000740F6091750F7091760F458F568F678FD3
:10D0300070A34091770F5091780F6091790F7091A4
:10D040007A0F41A352A363A374A32091450F90913B
:10D05000460F291303C094E69093420F8093450F27
:10D0600080916F00826080936F0008959091450FCA
:10D070008091460F981306C0809192159091931558
:10D08000892B19F00E941750F1CF0895CF93DF93A9
:10D090008B3D9240B1F0E9EDF9E18491EF012196E9
:10D0A000882321F00E94D63EFE01F7CFE2E3F7E1AC
:10D0B0008491EF012196882331F00E94D63EFE0133
:10D0C000F7CF80E001C081E0DF91CF9108952F92EA
:10D0D0003F924F925F926F927F928F929F92AF9208
:10D0E000BF92CF92DF92EF92FF920F931F93CF9355
:10D0F000DF93CDB7DEB7C757D1090FB6F894DEBFBF
:10D100000FBECDBF2DB63EB6A7961FAE1EAEA797DB
:10D1100084E690E0A9969FAF8EAFA99701E09E01AB
:10D120002B593F4F44E050E0BE01655A7F4FCE017E
:10D1300089599F4F0E94D7AA9E012B593F4F42E029
:10D1400050E0BE0167597F4FCE0189599F4F0E9421
:10D15000D7AA43E050E0BE01655A7F4F87ED92E0C9
:10D160000E946ECE892B09F43FC06F968FAD6F97EA
:10D17000882339F08FE36C968FAF6C976D961FAE56
:10D180006D97EEEEF9E184917F012FEFE21AF20A3A
:10D19000811103C0E5EFF7E104C00E94D63EF7011C
:10D1A000F2CF84917F013FEFE31AF30A882321F045
:10D1B0000E94D63EF701F5CFBE01655A7F4F8CEE37
:10D1C00097E10E94604DEEEDF7E184917F019FEFC2
:10D1D000E91AF90A882321F00E94D63EF701F5CF1B
:10D1E00081E08093910B54C5EDB7FEB7E696FFAF93
:10D1F000EEAFE6976B961CAE1DAE1EAE1FAE6B97E4
:10D20000A7961FAE1EAEA79701E09E012B593F4F78
:10D2100041E050E0BE0160597F4FCE0189599F4FD8
:10D220000E94D7AA80E1E3E5F2E0DE019196019049
:10D230000D928A95E1F780E1E3E6F2E0DE01519696
:10D2400001900D928A95E1F780E1E3E7F2E0DE01DB
:10D25000119601900D928A95E1F7E1964FADE19715
:10D2600050E04D5F5F4F440F551F440F551F2DB7C2
:10D270003EB7241B350B0FB6F8943EBF0FBE2DBF33
:10D280008DB79EB701967C0100E09E012B593F4F60
:10D29000BC01CE0189599F4F0E94D7AA9E012B59EC
:10D2A0003F4F44E050E06EE77BE0CE0189599F4F4D
:10D2B0000E94D7AAE1968FACE197912C93E0890E5A
:10D2C000911C880C991C880C991CEDB7FEB7E819C5
:10D2D000F9090FB6F894FEBF0FBEEDBF2DB73EB7EC
:10D2E0002F5F3F4F69018DB79EB7881999090FB617
:10D2F000F8949EBF0FBE8DBFEDB7FEB731965F01AC
:10D300009E012B593F4FA401B601CE0189599F4F71
:10D310000E94D7AA9E012B593F4FA401B501CE010F
:10D3200089599F4F0E94D7AA1091920B112309F49B
:10D33000A7C000E09E012B593F4F44E050E066E655
:10D340007BE0CE0189599F4F0E94D7AA9E012B599D
:10D350003F4F44E050E06AE67BE0CE0189599F4FA1
:10D360000E94D7AA9E012B593F4F44E050E062E64D
:10D370007BE0CE0189599F4F0E94D7AA9E012B596D
:10D380003F4F44E050E066E87BE0CE0189599F4F73
:10D390000E94D7AA9E012B593F4F44E050E062E81B
:10D3A0007BE0CE0189599F4F0E94D7AA9E012B593D
:10D3B0003F4F40E150E06EE47BE0CE0189599F4F42
:10D3C0000E94D7AA9E012B593F4F44E050E0BE0176
:10D3D000695A7F4FCE0189599F4F0E94D7AA9E015B
:10D3E0002B593F4F4CE050E063EA7BE0CE01895976
:10D3F0009F4F0E94D7AA9E012B593F4F44E050E017
:10D4000061EF75E1CE0189599F4F0E94D7AA9E0115
:10D410002B593F4F44E050E0BE01695A7F4FCE0187
:10D4200089599F4F0E94D7AA01E09E012B593F4F77
:10D4300041E050E0BE0161597F4FCE0189599F4FB5
:10D440000E94D7AA9E012B593F4F41E050E0BE01F8
:10D4500062597F4FCE0189599F4F0E94D7AA11115F
:10D460008AC06B968CAD9DADAEADBFAD6B97809312
:10D47000F9159093FA15A093FB15B093FC157BC09A
:10D48000E1968FADE19790E002962EE63BE0E496C0
:10D490003FAF2EAFE497B501DE011196E3EE8E2E7D
:10D4A000E6E19E2EAE014F5E5F4FF3ECAF2EF6E14C
:10D4B000BF2EE896FFAEEEAEE8977E0131E2E30EB6
:10D4C000F11C20E030E0821793072CF0E896EEADD7
:10D4D000FFADE89701C0F701408051806280738002
:10D4E000F50141925192619271925F018217930707
:10D4F00014F0F60101C0FA0140805180628073800F
:10D50000F40141925192619271924F0182179307F7
:10D5100034F0FB01408051806280738005C04D90E3
:10D520005D906D907C901397E496EEADFFADE4971F
:10D530004192519261927192E496FFAFEEAFE497FF
:10D540002F5F3F4F6C5F7F4F1496F4E0CF0ED11CDE
:10D550004C5F5F4FE896EEADFFADE8973496E896E6
:10D56000FFAFEEAFE897F4E0EF0EF11C2430310589
:10D5700009F0A9CFDECEE0968FADE097853099F423
:10D58000AF968FADAF97853071F400E09E012B59B7
:10D590003F4F44E650E06DEF75E1CE0189599F4F52
:10D5A0000E94D7AA24C0111102C00E940AAAE096C4
:10D5B0008FADE097AF96CFACAF978C9D60011124F3
:10D5C000E12CF12CEC14FD0491F000E09E012B59AC
:10D5D0003F4F44E050E0BE01695A7F4FCE01895968
:10D5E0009F4F0E94D7AA2FEFE21AF20AEBCF00E07A
:10D5F0009E012B593F4F44E050E0BE016D5A7F4FD2
:10D60000CE0189599F4F0E94D7AA1AE0115079F094
:10D6100000E09E012B593F4F44E050E0BE01695AA3
:10D620007F4FCE0189599F4F0E94D7AAEFCF01E0CB
:10D630009E012B593F4F41E050E0BE0163597F4F9F
:10D64000CE0189599F4F0E94D7AA9E012B593F4F67
:10D6500041E050E0BE0164597F4FCE0189599F4F90
:10D660000E94D7AA00E09E012B593F4F44E050E0B2
:10D67000BE01635C7F4FCE0189599F4F0E94D7AA9C
:10D680009E012B593F4F44E050E0BE016F5C7F4F3D
:10D69000CE0189599F4F0E94D7AAAE968FADAE9703
:10D6A000AD96CFACAD978C9D60011124E12CF12C8F
:10D6B00000E09E012B593F4FCE14DF0471F044E08F
:10D6C00050E0BE01695A7F4FCE0189599F4F0E9499
:10D6D000D7AA3FEFE31AF30AEBCF41E050E0BE01D7
:10D6E0006F587F4FCE0189599F4F0E94D7AA9E0144
:10D6F0002B593F4F41E050E0BE0165597F4FCE01AD
:10D7000089599F4F0E94D7AA9E012B593F4F44E051
:10D7100050E0BE01695A7F4FCE0189599F4F0E9448
:10D72000D7AA9E012B593F4F44E050E0BE01695AF1
:10D730007F4FCE0189599F4F0E94D7AA9E012B5936
:10D740003F4F44E050E065EF75E1CE0189599F4FAE
:10D750000E94D7AA9E012B593F4F44E050E0BE01E2
:10D76000615B7F4FCE0189599F4F0E94D7AA9E01CE
:10D770002B593F4F44E050E0BE01655B7F4FCE0127
:10D7800089599F4F0E94D7AA9E012B593F4F44E0D1
:10D7900050E0BE01695B7F4FCE0189599F4F0E94C7
:10D7A000D7AA10E000E09E012B593F4F44E050E023
:10D7B000BE01695A7F4FCE0189599F4F0E94D7AA57
:10D7C000111110C06B96CCACDDACEEACFFAC6B971E
:10D7D00020E030E84BE355E4C701B6010E94BDC626
:10D7E000811103C054E0F52E33C08091920B81115A
:10D7F00008C0C0928415D0928515E0928615F092EB
:10D80000871500E09E012B593F4F44E050E060E84F
:10D8100075E1CE0189599F4F0E94D7AA9E012B59CD
:10D820003F4F44E050E068E875E1CE0189599F4FD1
:10D830000E94D7AA9E012B593F4F44E050E0BE0101
:10D84000695A7F4FCE0189599F4F0E94D7AA12C0B3
:10D85000FA94FF2079F000E09E012B593F4F44E0FD
:10D8600050E0BE01695A7F4FCE0189599F4F0E94F7
:10D87000D7AAEECF1F5F153009F094CF00E09E01CC
:10D880002B593F4F42E050E0BE016D597F4FCE0112
:10D8900089599F4F0E94D7AA9E012B593F4F44E0C0
:10D8A00050E0BE01695A7F4FCE0189599F4F0E94B7
:10D8B000D7AA6B96CCACDDACEEACFFAC6B9720E09E
:10D8C00030E84BE355E4C701B6010E94BDC688238A
:10D8D00029F18091920B811108C0C0927C15D092E1
:10D8E0007D15E0927E15F0927F1500E09E012B5988
:10D8F0003F4F44E050E068E775E1CE0189599F4F02
:10D900000E94D7AA9E012B593F4F44E050E064E7A4
:10D9100075E1CE0189599F4F0E94D7AA00E09E0170
:10D920002B593F4F42E050E0BE016F597F4FCE016F
:10D9300089599F4F0E94D7AA9E012B593F4F41E022
:10D9400050E0BE016F587F4FCE0189599F4F0E9412
:10D95000D7AA19E0115000E09E012B593F4F112327
:10D9600059F044E050E0BE01695A7F4FCE01895919
:10D970009F4F0E94D7AAEECF41E050E061E676E1EA
:10D98000CE0189599F4F0E94D7AAF12C00E09E0139
:10D990002B593F4F44E050E0BE01695A7F4FCE0102
:10D9A00089599F4F0E94D7AA1091920B111110C054
:10D9B000F1100EC06B968CAD9DADAEADBFAD6B974B
:10D9C0008093661690936716A0936816B0936916B5
:10D9D000F39485E0F812DACF111102C00E943944A5
:10D9E0004CE0F42EFA94F11003C03CE0F32E0FC08B
:10D9F00000E09E012B593F4F42E050E0BE01615ACA
:10DA00007F4FCE0189599F4F0E94D7AAEBCFFA943E
:10DA100000E09E012B593F4FFF2059F044E050E0B9
:10DA2000BE016D5B7F4FCE0189599F4F0E94D7AADF
:10DA3000EECF46E050E0BE01635C7F4FCE018959D6
:10DA40009F4F0E94D7AA9E012B593F4F44E050E0C0
:10DA50006EE57BE0CE0189599F4F0E94D7AA9E01B7
:10DA60002B593F4F4CE050E0BE016F5C7F4FCE0121
:10DA700089599F4F0E94D7AA2CE1F22EFA94F110F7
:10DA800003C094E0F92E1DC000E09E012B593F4FCA
:10DA900044E050E0BE01695A7F4FCE0189599F4F43
:10DAA0000E94D7AAEBCF00E09E012B593F4F44E0E4
:10DAB00050E0BE01695A7F4FCE0189599F4F0E94A5
:10DAC000D7AAFA94F110EFCF8BE0F82EFA94FF204A
:10DAD00079F000E09E012B593F4F44E050E0BE0139
:10DAE000695A7F4FCE0189599F4F0E94D7AAEECF26
:10DAF000A9968EAD9FADA99784569109C7DA8093F8
:10DB0000910B882309F1EEEEF9E184917F019FEFFB
:10DB1000E91AF90A882321F00E94D63EF701F5CFD1
:10DB2000A9966EAD7FADA9976456710986ED97E110
:10DB30000E94474D6BED72E08EEC97E10E94474DDD
:10DB40008AE00E94D63E99C0A7962EAD3FADA7971A
:10DB5000AB968EAD9FADAB972817390709F44BC034
:10DB600081E08093910BE9EDF9E184917F012FEF42
:10DB7000E21AF20A811103C0EEEAF7E104C00E9442
:10DB8000D63EF701F2CF84917F013FEFE31AF30A0B
:10DB9000882321F00E94D63EF701F5CFAB966EADFB
:10DBA0007FADAB9780E090E04AE00E94F241E9EA65
:10DBB000F7E184917F019FEFE91AF90A882321F0A8
:10DBC0000E94D63EF701F5CFA7966EAD7FADA79721
:10DBD00080E090E04AE00E94F241E9E9F7E18491B7
:10DBE0007F012FEFE21AF20A882309F446C00E944F
:10DBF000D63EF701F4CF111142C0EEEEF9E1849167
:10DC00007F013FEFE31AF30A811103C007ED12E031
:10DC100004C00E94D63EF701F2CFF80181918F0136
:10DC2000882319F00E94D63EF8CFA9966EAD7FAD3D
:10DC3000A997645671098CE797E10E94474DA79612
:10DC40004EAD5FADA79760E070E08FE697E10E9470
:10DC50000D4DECE6F7E184917F012FEFE21AF20A15
:10DC6000811107C08091910B811109C00E9496AB70
:10DC700006C00E94D63EF701EECF112399F3E69637
:10DC80008EAD9FADE6970FB6F8949EBF0FBE8DBFC9
:10DC90008091920B811102C00E94A69E9091910BDF
:10DCA00081E089270FB6F8943EBE0FBE2DBEC9583D
:10DCB000DF4F0FB6F894DEBF0FBECDBFDF91CF911F
:10DCC0001F910F91FF90EF90DF90CF90BF90AF909A
:10DCD0009F908F907F906F905F904F903F902F908C
:10DCE000089581E08093920BF2D91092920B8111EA
:10DCF000EEC90E943AA381E008958F929F92AF925D
:10DD0000BF92CF92DF92EF92FF920F931F93CF9328
:10DD1000DF93CDB7DEB7CA5AD1090FB6F894DEBF8C
:10DD20000FBECDBFE9961CAE1DAE1EAE1FAEE9976D
:10DD30008091C5039091C603A091C703B091C80319
:10DD4000ED968CAF9DAFAEAFBFAFED97C556DF4F31
:10DD500019821882CB59D04084E690E0C356DF4F39
:10DD600099838883CD59D0401092910B9E012556FE
:10DD70003F4F44E050E0BE0167587F4FCE018356CD
:10DD80009F4F0E9423ABC356DF4F88819981CD59A5
:10DD9000D0400296C356DF4F99838883CD59D04037
:10DDA000C556DF4F19821882CB59D04081E0CD553E
:10DDB000DF4F8883C35AD0409E0125563F4F41E034
:10DDC00050E0BE016D557F4FCE0183569F4F0E949C
:10DDD00023AB9E0125563F4F40E150E063EC76E1D6
:10DDE000CE0183569F4F0E9423AB9E0125563F4F85
:10DDF00044E050E06EE77BE0CE0183569F4F0E94E7
:10DE000023AB9E0125563F4F40E150E063EE76E1A3
:10DE1000CE0183569F4F0E9423AB9E0125563F4F54
:10DE200040E150E06EE67BE0CE0183569F4F0E94BA
:10DE300023AB9E0125563F4F44E050E066E67BE071
:10DE4000CE0183569F4F0E9423AB9E0125563F4F24
:10DE500044E050E06AE67BE0CE0183569F4F0E948B
:10DE600023AB9E0125563F4F44E050E062E67BE045
:10DE7000CE0183569F4F0E9423AB9E0125563F4FF4
:10DE800044E050E066E87BE0CE0183569F4F0E945D
:10DE900023AB9E0125563F4F44E050E062E87BE013
:10DEA000CE0183569F4F0E9423AB9E0125563F4FC4
:10DEB00040E150E06EE47BE0CE0183569F4F0E942C
:10DEC00023AB8AE097EDA3EABCE3E9968CAF9DAF64
:10DED000AEAFBFAFE9979E0125563F4F44E050E0FB
:10DEE000BE016B587F4FCE0183569F4F0E9423ABDC
:10DEF0009E0125563F4F4CE050E063EA7BE0CE01A7
:10DF000083569F4F0E9423AB80917616909177168F
:10DF1000A0917816B0917916C358DF4F8883998302
:10DF2000AA83BB83CD57D0409E0125563F4F44E086
:10DF300050E0BE0163587F4FCE0183569F4F0E9431
:10DF400023AB85E0CC55DF4F8883C45AD040CB55F6
:10DF5000DF4F8883C55AD0409E0125563F4F44E08D
:10DF600050E069EF75E1CE0183569F4F0E9423ABCD
:10DF70009E0125563F4F41E050E0BE016C557F4F5A
:10DF8000CE0183569F4F0E9423AB9E0125563F4FE3
:10DF900041E050E0BE016B557F4FCE0183569F4F4D
:10DFA0000E9423AB9E0125563F4F44E650E06DEFA3
:10DFB00075E1CE0183569F4F0E9423ABCF57DF4FB1
:10DFC000188219821A821B82C158D0409E012556A0
:10DFD0003F4F44E050E0BE016F577F4FCE01835664
:10DFE0009F4F0E9423ABE9961CAE1DAE1EAE1FAE26
:10DFF000E9971AE0115071F09E0125563F4F44E019
:10E0000050E0BE016B587F4FCE0183569F4F0E9458
:10E0100023ABF0CF83E0CA55DF4F8883C65AD04088
:10E02000C955DF4F8883C75AD040CB57DF4F18827E
:10E0300019821A821B82C558D040C757DF4F1882F9
:10E0400019821A821B82C958D040E9961CAE1DAEB7
:10E050001EAE1FAEE9979E0125563F4F41E050E0AE
:10E06000BE016A557F4FCE0183569F4F0E9423AB5E
:10E070009E0125563F4F41E050E0BE0169557F4F5C
:10E08000CE0183569F4F0E9423AB9E0125563F4FE2
:10E0900044E050E0BE0167577F4FCE0183569F4F4B
:10E0A0000E9423AB9E0125563F4F44E050E0BE0145
:10E0B0006B577F4FCE0183569F4F0E9423AB0AE0E0
:10E0C00010E00150110971F09E0125563F4F44E0C8
:10E0D00050E0BE016B587F4FCE0183569F4F0E9488
:10E0E00023ABEFCFC855DF4F1882C85AD0408FEF0F
:10E0F000C755DF4F8883C95AD0409E0125563F4FF0
:10E1000041E050E0BE0168557F4FCE0183569F4FDE
:10E110000E9423AB9E0125563F4F41E050E0BE01D7
:10E1200067557F4FCE0183569F4F0E9423ABE996E0
:10E130001CAE1DAE1EAE1FAEE9979E0125563F4F89
:10E1400044E050E0BE016B587F4FCE0183569F4F95
:10E150000E9423AB9E0125563F4F44E050E0BE0194
:10E160006B587F4FCE0183569F4F0E9423AB9E0179
:10E1700025563F4F44E050E065EF75E1CE018356F0
:10E180009F4F0E9423AB8091830290918402A091C3
:10E190008502B0918602C357DF4F88839983AA8393
:10E1A000BB83CD58D0408091870290918802A09186
:10E1B0008902B0918A02CF56DF4F88839983AA8360
:10E1C000BB83C159D040CB56DF4F19821882C55945
:10E1D000D040C956DF4F19821882C759D0409E01DE
:10E1E00025563F4F44E050E0BE0163577F4FCE01BC
:10E1F00083569F4F0E9423AB9E0125563F4F44E01C
:10E2000050E0BE016F567F4FCE0183569F4F0E9454
:10E2100023AB9E0125563F4F44E050E0BE016B56B4
:10E220007F4FCE0183569F4F0E9423AB10E0C12C3D
:10E2300080E8D82E8BE3E82E85E4F82E812C912CF3
:10E2400090E8A92E9FE3B92E111138C09E012556E2
:10E250003F4F44E050E064E875E1CE0183569F4FA4
:10E260000E9423AB9E0125563F4F44E050E060E8FA
:10E2700075E1CE0183569F4F0E9423AB9E01255628
:10E280003F4F44E050E068E875E1CE0183569F4F70
:10E290000E9423ABE9968CAE9DAEAEAEBFAEE997C1
:10E2A0009E0125563F4F44E050E0BE016B587F4F22
:10E2B000CE0183569F4F0E9423AB2AC0E996CCAE75
:10E2C000DDAEEEAEFFAEE9979E0125563F4F44E02E
:10E2D00050E0BE016B587F4FCE0183569F4F0E9486
:10E2E00023ABE9961CAE1DAE1EAE1FAEE99704E04F
:10E2F000015071F09E0125563F4F44E050E0BE01B1
:10E300006B587F4FCE0183569F4F0E9423ABF0CFB7
:10E310001F5F153009F098CF84E190E0C156DF4FC0
:10E3200099838883CF59D0409E0125563F4F42E0C4
:10E3300050E0BE0161567F4FCE0183569F4F0E9431
:10E3400023AB9E0125563F4F44E050E06CE775E15A
:10E35000CE0183569F4F0E9423AB9E0125563F4F0F
:10E3600044E050E068E775E1CE0183569F4F0E947C
:10E3700023AB9E0125563F4F44E050E064E775E132
:10E38000CE0183569F4F0E9423AB80E290E0CF5591
:10E39000DF4F99838883C15AD0409E0125563F4F55
:10E3A00042E050E0BE016F557F4FCE0183569F4F34
:10E3B0000E9423ABC655DF4F1882CA5AD04080E274
:10E3C000EBE8F2E0DE019D9601900D928A95E1F76F
:10E3D0009E0125563F4F41E050E0BE0166557F4FFC
:10E3E000CE0183569F4F0E9423AB9E0125563F4F7F
:10E3F00040E250E0BE01635D7F4FCE0183569F4FE8
:10E400000E9423AB9E0125563F4F41E050E061E65C
:10E4100076E1CE0183569F4F0E9423AB10E011118D
:10E420000EC08091661690916716A0916816B09103
:10E430006916E9968CAF9DAFAEAFBFAFE9979E016D
:10E4400025563F4F44E050E0BE016B587F4FCE0150
:10E4500083569F4F0E9423AB1F5F153001F7BE010B
:10E46000635B7F4F86E1FB0111928A95E9F79E017C
:10E4700025563F4F46E150E0CE0183569F4F0E9404
:10E4800023AB8CE2EBEAF2E0DE01119601900D92F3
:10E490008A95E1F79E0125563F4F4CE250E0BE01C0
:10E4A0006F5F7F4FCE0183569F4F0E9423ABBE010B
:10E4B00061597F4F86E0FB0111928A95E9F79E0131
:10E4C00025563F4F46E050E0CE0183569F4F0E94B5
:10E4D00023AB9E0125563F4F44E050E06EE57BE0C4
:10E4E000CE0183569F4F0E9423ABBE016D597F4FD3
:10E4F0008CE0FB0111928A95E9F79E0125563F4F6A
:10E500004CE050E0CE0183569F4F0E9423ABE9962A
:10E510001CAE1DAE1EAE1FAEE9971CE1115071F08E
:10E520009E0125563F4F44E050E0BE016B587F4F9F
:10E53000CE0183569F4F0E9423ABF0CFE9961CAECD
:10E540001DAE1EAE1FAEE99714E0115071F09E0192
:10E5500025563F4F44E050E0BE016B587F4FCE013F
:10E5600083569F4F0E9423ABF0CFE9961CAE1DAEA1
:10E570001EAE1FAEE9971BE0115071F09E012556AB
:10E580003F4F44E050E0BE016B587F4FCE018356B1
:10E590009F4F0E9423ABF0CF8091910B811167C0F8
:10E5A000C356DF4FE880F980CD59D040F4E6EF1A2A
:10E5B000F108C556DF4F88819981CB59D040C756A5
:10E5C000DF4F99838883C959D04084E690E0C356D1
:10E5D000DF4F99838883CD59D0409E0125563F4F08
:10E5E00044E050E067ED72E0CE0183569F4F0E94F9
:10E5F00023AB9E0125563F4F42E050E0BE016756D7
:10E600007F4FCE0183569F4F0E9423ABEEEEF9E180
:10E6100084918F010F5F1F4F882321F00E94D63E07
:10E62000F801F6CFB7018AE597E10E94474DC7563A
:10E63000DF4F48815981C959D04060E070E08DE4D6
:10E6400097E10E940D4DEAE4F7E184918F010F5F9D
:10E650001F4F882321F00E94D63EF801F6CFC70154
:10E660000E9446689091910B892B8093910B909119
:10E67000910B81E08927C655DF4F0FB6F894DEBFB6
:10E680000FBECDBFDF91CF911F910F91FF90EF9003
:10E69000DF90CF90BF90AF909F908F900895CF92D2
:10E6A000DF92EF92FF920F931F93CF93DF936C0152
:10E6B0007A018B01C0E0D0E0CE15DF0581F0D801F2
:10E6C0006D918D01D601ED91FC910190F081E02DCD
:10E6D000C6011995892B11F02196EECF7E01C70155
:10E6E000DF91CF911F910F91FF90EF90DF90CF902E
:10E6F00008950E9413CE1F920F920FB60F9211240D
:10E700000BB60F922F933F934F935F936F937F932B
:10E710008F939F93AF93BF93EF93FF938091960B4B
:10E720009091970BA091980BB091990B892B8A2B04
:10E730008B2B59F19091950BE091930BF091940BE9
:10E740008081892780838091960B9091970BA0916F
:10E75000980BB091990B181619061A061B060CF0A7
:10E7600056C08091960B9091970BA091980BB09109
:10E77000990B0197A109B1098093960B9093970B80
:10E78000A093980BB093990B42C080913902EEE0B0
:10E79000F8E1E4919FEF90933902E230C9F050F430
:10E7A000EE2399F0E13081F590916F009D7F909379
:10E7B0006F002AC0E43019F1E0F0E53029F59091BE
:10E7C00073009D7F909373001FC010926E001CC059
:10E7D000909170009D7F9093700091E09093B000B5
:10E7E0009091B100987F94609093B1001092B30023
:10E7F0000BC0909171009D7F9093710005C0909126
:10E8000072009D7F9093720060E00E94E2B2FF91DF
:10E81000EF91BF91AF919F918F917F916F915F9198
:10E820004F913F912F910F900BBE0F900FBE0F9005
:10E830001F9018959093100480930F0480E00C941F
:10E84000407C8F929F92AF92BF92CF92DF92EF92D5
:10E85000FF921F93CF93DF93C82F85E691E19093AA
:10E86000410F8093400F1092811182E090E0A0E070
:10E87000B0E080936A1190936B11A0936C11B093E8
:10E880006D1110923F0F10923B0F10923C0F10929F
:10E890003D0F10923E0F8FEF9FEFDC018093370FFB
:10E8A0009093380FA093390FB0933A0FCC2379F19E
:10E8B000C53008F0F8C040E060E070E0CB010E9495
:10E8C0007DAC882309F4EFC020E1C29FC001112470
:10E8D000895D924FFC01E254FE4F20812F7709F0B1
:10E8E000E2C03C964081518162817381443651057A
:10E8F0006105710508F4D7C03497C080D180E280EB
:10E90000F380C114D104E104F10421F4CCC0C12C82
:10E91000D12C760140E0C701B6010E947DAC182FD2
:10E92000882309F4C0C08091420D9091430D811558
:10E93000924009F0B8C0A091470DAA2309F4B3C0D2
:10E940006091450D7091460D6115710509F4ABC0DC
:10E950002091440D222309F4A6C0A0937C1120939A
:10E960006E1180E030E041E050E0C82FFA01082E3F
:10E9700002C0EE0FFF1F0A94E2F72E173F0739F08F
:10E980008F5FC83091F789E0809377118CC08093B6
:10E99000771120914D0D30914E0D2115310519F053
:10E9A00040E050E008C020915B0D30915C0D40913B
:10E9B0005D0D50915E0D20936F1130937011409357
:10E9C00071115093721146015701860E971EA11CBA
:10E9D000B11C80927D1190927E11A0927F11B09215
:10E9E0008011E091480DF091490DF0938311E0936F
:10E9F0008211B0E00E94CDCA860E971EA81EB91ED5
:10EA00008092841190928511A0928611B092871104
:10EA100085E0EE0FFF1F8A95E1F7E150FE4FEF2FE3
:10EA2000FF27E6958E0E9F1EA11CB11C80927811C7
:10EA300090927911A0927A11B0927B1120914A0D97
:10EA400030914B0D2115310521F0A90160E070E0F6
:10EA500008C04091570D5091580D6091590D70911B
:10EA60005A0DD701C60188199909AA09BB09840F53
:10EA7000951FA61FB71F04C0B695A79597958795B4
:10EA8000CA95D2F78093731190937411A093751166
:10EA9000B0937611853F2FE09207A105B10528F4C8
:10EAA0008CE08093811110E01AC0853F9F4FA10533
:10EAB000B10510F480E111C08091630D9091640D57
:10EAC000A091650DB091660D80938411909385118E
:10EAD000A0938611B093871180E280938111812FDA
:10EAE000DF91CF911F91FF90EF90DF90CF90BF907B
:10EAF000AF909F908F900895682F8CE295E10C94D1
:10EB00005A39CF92DF92EF92FF921F93CF93DF9308
:10EB10001092C40F8091F70F882321F084EF9FE0BB
:10EB20000E941E90109269111092661185E38093E5
:10EB300065110E944BB4EB01A89561E080916511CD
:10EB40000E9410B385E691E10E947F912398229A5A
:10EB5000219A209A289A85E08093671182E58CBDDE
:10EB60001DBC1AE08FEF0E9484911150D9F720E06C
:10EB700030E0A90160E085E691E10E948991182FBB
:10EB800080936811813049F00E944BB46C1B7D0B5F
:10EB9000613D774060F381E054C02AEA31E040E013
:10EBA00050E068E085E691E10E94899182FF03C010
:10EBB000109369110EC014E00E94DB4D8093681120
:10EBC0001150D1F78A3A11F082E03BC082E0809385
:10EBD000691180916911823021F0C12CD12C76010C
:10EBE00005C0C12CD12CE12C80E4F82E20E030E0CF
:10EBF000A90167E385E691E10E948991A701960149
:10EC000069E285E691E10E948991809368118823E9
:10EC100049F00E944BB46C1B7D0B613D774030F393
:10EC20008AE00FC080916911823011F520E030E058
:10EC3000A9016AE385E691E10E948991882351F058
:10EC400088E08093661185E691E10E947F91EEEE67
:10EC5000F9E119C00E94DB4D807C803C19F483E00F
:10EC6000809369110E94DB4D0E94DB4D0E94DB4DB9
:10EC700085E691E10E947F911092671181E0E1DDCC
:10EC8000811131C015C08491EF012196882321F0B4
:10EC90000E94D63EFE01F7CFE0EEF9E18491EF014C
:10ECA0002196882309F456C00E94D63EFE01F6CF75
:10ECB00080E0C7DD811117C0E9EDF9E18491EF0132
:10ECC0002196882321F00E94D63EFE01F7CFE5EC85
:10ECD000F9E18491EF012196882309F43BC00E9459
:10ECE000D63EFE01F6CF6AE671E184EF9FE00E9416
:10ECF000CB8F811116C0E9EDF9E18491EF012196E6
:10ED0000882321F00E94D63EFE01F7CFE4EBF9E123
:10ED10008491EF0121968823E9F00E94D63EFE01FE
:10ED2000F7CF81E08093C40FEEEEF9E18491EF011B
:10ED30002196882321F00E94D63EFE01F7CFE8EA13
:10ED4000F9E18491EF012196882321F00E94D63EBB
:10ED5000FE01F7CF8BE1E4EFFFE0A3E1B0E101902A
:10ED60000D928A95E1F78091F20F9091F30F9093B5
:10ED7000121080931110DF91CF911F91FF90EF90AF
:10ED8000DF90CF9008958091D113823041F483E9D0
:10ED900099E19093360D8093350D0E94023F0E94B9
:10EDA0004BB46093D5137093D6138093D71390937D
:10EDB000D8138091C40F882319F081E08093C30F8A
:10EDC00081E08093D1130895CF93DF931092C30F06
:10EDD00083E08093D11380911E148823B1F0EBE877
:10EDE000F9E18491EF01882341F0082E000C990B82
:10EDF00083DE2196FE018491F6CF8DE090E07CDEEB
:10EE00008AE090E0DF91CF9177CEEFE8F9E184914D
:10EE1000EF01882391F3082E000C990B6DDE2196EB
:10EE2000FE018491F6CF8F929F92AF92BF92CF92C4
:10EE3000DF92EF92FF920F931F93CF93DF9300D057
:10EE40001F92CDB7DEB7FC018381813079F58181D6
:10EE500081FF2CC081899289A389B489892B8A2B4F
:10EE60008B2B09F448C07F0140E050E0BA01CF018C
:10EE70000E94348F8823D1F0F70185889688A7886F
:10EE8000B08CC18CD28C82E090E0A0E0B0E0F601C2
:10EE900080839183A283B3839E012F5F3F4FB5018F
:10EEA000A401C6010E9446AD811102C080E03CC0B1
:10EEB00000E010E09801B501A401C6010E94B5ACC4
:10EEC0008823A1F389809A80AB80BC80F601878972
:10EED000803141F4F8EF8F16FFEF9F06A104B104D3
:10EEE00060F4DACF88EF88168FEF9806A8068FE0D7
:10EEF000B80618F4D1CF81E017C0F701158A168A39
:10EF0000178A108E118A128A138A148A8181806866
:10EF10008183C7010E9494AE882341F240E050E013
:10EF2000BA01C7010E94348F0F900F900F900F907D
:10EF3000DF91CF911F910F91FF90EF90DF90CF90D5
:10EF4000BF90AF909F908F9008951092C60F10922F
:10EF5000C30F80918F11882321F08CE891E10C94EC
:10EF60001E9008952F923F924F925F926F927F92E0
:10EF70008F929F92AF92BF92CF92DF92EF92FF92C9
:10EF80000F931F93CF93DF93CDB7DEB7C257D1094D
:10EF90000FB6F894DEBF0FBECDBF8C013B014A0116
:10EFA0004DB75EB7E1965FAF4EAFE197AD961FAE3E
:10EFB000AD971B0154E0250E311C7E018FE5E80E54
:10EFC000F11C95EE492E92E0592EE0E4F0E0EC0FB2
:10EFD000FD1F3496E396FFAFEEAFE397F301878111
:10EFE000823008F462C184859585A685B7858F71C6
:10EFF0009927AA27BB27892B8A2B8B2B09F055C170
:10F000001092D40F44ED5FE0BE016F5F7F4FC101EE
:10F010000E942CAE18160CF048C18C85982F987160
:10F02000903129F4209141122150223078F4298125
:10F03000222309F43AC1253E89F22E3279F2209139
:10F04000D40F2E3259F28A7049F6B8C04DB75EB768
:10F05000AF965FAF4EAFAF97BE016F5F7F4FC701F7
:10F060000E9427AC0115110521F0F8018081811162
:10F070009BC021E081E090E0F70101900020E9F7DA
:10F080003197EE19FF098E0F9F1F02964DB75EB79D
:10F09000481B590B0FB6F8945EBF0FBE4DBF8DB71E
:10F0A0009EB701965C01211102C0B80102C06AE15D
:10F0B00073E0C5010E9467CEB701C5010E9448CE2A
:10F0C0006AE173E0C5010E9448CE25961FAE2597E0
:10F0D00028961FAE289724961FAE1EAE2497229620
:10F0E0005FAE4EAE229721E0A701B101E3968EAD4F
:10F0F0009FADE3970E94B19581112AC08091411282
:10F10000811126C0EEEEF9E184916F019FEFC91ADB
:10F11000D90A882321F00E94D63EF601F5CFE7E711
:10F12000F9E184916F012FEFC21AD20A882321F0EE
:10F130000E94D63EF601F5CF6701F60181916F017D
:10F14000882319F00E94D63EF8CF8AE00E94D63E6E
:10F150008BE1FE01EC5BFF4FDE01959601900D9275
:10F160008A95E1F724968EAD9FAD24979CA38BA33F
:10F170005AA249A240E050E0BE016F5D7F4FC50139
:10F18000F1DECE0181960E94AD4FCE01805C9F4F93
:10F190000E94AD4FAF964EAD5FADAF970FB6F894EE
:10F1A0005EBF0FBE4DBF1ACFF80101900020E9F7F6
:10F1B0003197CF01801B910B20E05ECF81E0903131
:10F1C00009F080E08093C50F903141F08985873444
:10F1D00009F004CF8A858E3709F400CF809141125F
:10F1E000813029F08230D9F18111F8CE0AC08091A6
:10F1F00042129091431201969093431280934212CF
:10F20000EDCEBE016F5F7F4F87EC9FE00E9427AC81
:10F210000115110529F487ECC82E8FE0D82E09C0FE
:10F220006801F60181916F018823A9F30E94D63EFF
:10F23000F8CFF60181916F01882319F00E94D63E24
:10F24000F8CF80E20E94D63E6D8D7E8D8F8D98A185
:10F250004AE00E94F2418AE00E94D63EBFCEBE0143
:10F260006F5F7F4F87EC9FE00E9427AC8114910471
:10F2700041F067EC7FE0C4010E9435CE892B69F430
:10F2800014C0AD96FFADAD978F2F90E020914E1535
:10F2900030914F158217930741F0AD962FADAD9782
:10F2A0002F5FAD962FAFAD9799CEE1968EAD9FAD06
:10F2B000E1970FB6F8949EBF0FBE8DBFCE58DF4FBB
:10F2C0000FB6F894DEBF0FBECDBFDF91CF911F9177
:10F2D0000F91FF90EF90DF90CF90BF90AF909F90F5
:10F2E0008F907F906F905F904F903F902F900895F8
:10F2F0000F931F93CF93DF93CDB7DEB76F970FB602
:10F30000F894DEBF0FBECDBF8B0122E020934112E7
:10F3100090934F1580934E1583E190E10E947B916D
:10F320008BE1E3E1F0E1DE01159601900D928A9503
:10F33000E1F780911110909112109C838B8385EEE0
:10F3400092E09A838983A801BE016F5F7F4F80E0BE
:10F3500090E008DECE0101960E94AD4F6F960FB689
:10F36000F894DEBF0FBECDBFDF91CF911F910F91FB
:10F3700008952F923F924F925F926F927F928F9259
:10F380009F92AF92BF92CF92DF92EF92FF920F9334
:10F390001F93CF93DF93CDB7DEB76F970FB6F89477
:10F3A000DEBF0FBECDBF6C012DB63EB61D821886E6
:10F3B0001C821B8285EE92E09A838983FB01808107
:10F3C0009E012F5F3F4F39018F3241F08FE090E176
:10F3D000F60191838083F62E172F64C080EF9FE0A3
:10F3E000F601918380838B010F5F1F4F011511057B
:10F3F00009F456C04DB65EB66FE270E0C8010E94D7
:10F4000053CE4C010817190708F048C07C01E01AD8
:10F41000F10AFF24C70101962DB73EB7281B390B0F
:10F420000FB6F8943EBF0FBE2DBF8DB79EB70196A5
:10F430005C01A701B8010E947CCEF501EE0DFF1D15
:10F440001082F601608171816115710511F06C5FA8
:10F450007F4F21E0A501CE0105960E94B195811153
:10F4600011C0B50183E699E10E94604D8EE20E94D1
:10F47000D63E8AE00E94D63E0FB6F8945EBE0FBE1E
:10F480004DBE0EC0F6017182608284010F5F1F4F76
:10F490000FB6F8945EBE0FBE4DBEA8CFF02E02C0D0
:10F4A000F12C10E0C3010E94AD4F8F2D912F0FB6AC
:10F4B000F8943EBE0FBE2DBE6F960FB6F894DEBF19
:10F4C0000FBECDBFDF91CF911F910F91FF90EF90B5
:10F4D000DF90CF90BF90AF909F908F907F906F9074
:10F4E0005F904F903F902F900895FF920F931F933E
:10F4F000CF93DF938C01EB01F42E80E20E94D63E85
:10F500008FEFF81611F084E501C082E40E94D63E28
:10F510008AE30E94D63EF8016081718182819381E5
:10F5200042E00E947742488159816A817B818FE85D
:10F530009CE10E942A4D62E070E080E090E0DF9163
:10F54000CF911F910F91FF900C9413B48F929F92C3
:10F55000AF92BF92CF92DF92EF92FF920F931F93E1
:10F56000CF93DF93F0E2FF2EE12CAE2DB0E0BD0192
:10F570006F0D711D759567956E1511F0F6120BC024
:10F58000E2E7FAE165917491072E000C880B990B64
:10F590000E94C3C662C09B0121503109220F331F54
:10F5A000220F331FF901EC50F64E05911491AB0177
:10F5B000440F551F440F551FFA01EC50F64EC591EC
:10F5C000D4918017910714F4F62ED1CFC817D9071C
:10F5D00014F4E62ECACFF901EA50F64EE590F49005
:10F5E000FA01EA50F64EC590D490BC01601B710B35
:10F5F000072E000C880B990B0E94C3C64B015C01BF
:10F60000B6016E197F09072E000C880B990B0E941A
:10F61000C3C69B01AC01C501B4010E9422C74B01C6
:10F620005C01C01BD10BBE01DD0F880B990B0E9442
:10F63000C3C69B01AC01C501B4010E94C3CB4B0101
:10F640005C01B701FF0C880B990B0E94C3C69B019C
:10F65000AC01C501B4010E94E7CADF91CF911F91AF
:10F660000F91FF90EF90DF90CF90BF90AF909F9061
:10F670008F9008950F931F93CF93DF93CDB7DEB78D
:10F6800028970FB6F894DEBF0FBECDBF60910F0470
:10F6900070911004072E000C880B990B0E94C3C6B2
:10F6A0006D837E838F8398878091110490911204DB
:10F6B000A0911304B091140489839A83AB83BC8313
:10F6C0004DEFBE016B5F7F4FCE0101960EDF609163
:10F6D000090470910A04072E000C880B990B0E94F4
:10F6E000C3C66D837E838F83988780910B0490912E
:10F6F0000C04A0910D04B0910E0489839A83AB830E
:10F70000BC834FEFBE016B5F7F4FCE010196EDDEF4
:10F71000E7E9FCE184918F010F5F1F4F882321F0FF
:10F720000E94D63EF801F6CFE0919615F0E0EC5637
:10F73000FA4E608170E080E090E00E945D42E2E974
:10F74000FCE184918F010F5F1F4F882321F00E94FD
:10F75000D63EF801F6CF6091951570E080E090E01C
:10F760000E945D4228960FB6F894DEBF0FBECDBF53
:10F77000DF91CF911F910F9108950F930FB70F93C2
:10F7800000916E000B7F00936E0078940F930BB77F
:10F790000F930CB70F921F922F933F934F935F934A
:10F7A0006F937F938F939F93AF93BF93EF93FF9349
:10F7B0001124DAD2FF91EF91BF91AF919F918F9178
:10F7C0007F916F915F914F913F912F911F900F907B
:10F7D0000CBF0F910BBF0F910460F89400936E0063
:10F7E0000F910FBF0F911895CF92DF92EF92FF927A
:10F7F000C0900B04D0900C04E0900D04F0900E0427
:10F800006091090470910A0466507109072E000C7A
:10F81000880B990B0E94C3C69B01AC01C701B601BE
:10F820000E94BDC687FF1FC020E030E040E050E4EA
:10F83000C701B6010E94E7CA0E9430CC7093CE1572
:10F840006093CD150E944BB4DC01CB01805A9541E9
:10F85000AF4FBF4F8093C9159093CA15A093CB1596
:10F86000B093CC1508C01092C9151092CA15109209
:10F87000CB151092CC15FF90EF90DF90CF900895AC
:10F88000CF92DF92EF92FF92C0901104D0901204B9
:10F89000E0901304F090140460910F047091100430
:10F8A00066507109072E000C880B990B0E94C3C685
:10F8B0009B01AC01C701B6010E94BDC687FF1FC0F6
:10F8C00020E030E040E050E4C701B6010E94E7CA02
:10F8D0000E9430CC7093C8156093C7150E944BB43A
:10F8E000DC01CB01805E914BAF4FBF4F8093C315BE
:10F8F0009093C415A093C515B093C61508C0109277
:10F90000C3151092C4151092C5151092C615FF901C
:10F91000EF90DF90CF9008958F929F92AF92BF9219
:10F92000CF92DF92EF92FF920F931F93CF93DF93CB
:10F93000F0E4FF2EE12CAE2DB0E0BD016F0D711D86
:10F94000759567956E1511F0F6120BC0E4EEFBE1AC
:10F9500065917491072E000C880B990B0E94C3C609
:10F9600062C09B0121503109220F331F220F331F28
:10F97000F901EA51F54E05911491AB01440F551F61
:10F98000440F551FFA01EA51F54EC591D4918017E5
:10F99000910714F4F62ED1CFC817D90714F4E62E28
:10F9A000CACFF901E851F54EE590F490FA01E8511B
:10F9B000F54EC590D490BC01601B710B072E000C56
:10F9C000880B990B0E94C3C64B015C01B6016E19EE
:10F9D0007F09072E000C880B990B0E94C3C69B0160
:10F9E000AC01C501B4010E9422C74B015C01C01BE0
:10F9F000D10BBE01DD0F880B990B0E94C3C69B0182
:10FA0000AC01C501B4010E94C3CB4B015C01B7013D
:10FA1000FF0C880B990B0E94C3C69B01AC01C5016A
:10FA2000B4010E94E7CADF91CF911F910F91FF901F
:10FA3000EF90DF90CF90BF90AF909F908F90089500
:10FA400060E08091D9159091DA1580DD6093110402
:10FA50007093120480931304909314048091D7152B
:10FA60009091D81559DF60930B0470930C04809328
:10FA70000D0490930E04A8951092911508957F920D
:10FA80008F929F92AF92BF92CF92DF92EF92FF92AE
:10FA90000F931F93CF93DF9320E030E048E452E4CC
:10FAA00060911104709112048091130490911404D8
:10FAB0000E940DCD18164CF4EAE7FAE1E491C1E09A
:10FAC00001C0CC0FEA95EAF701C0C0E084E7E82E58
:10FAD0008AE1F82E0AE71AE196E0A92E912CD0E0EF
:10FAE000CC24C394D12CF7017490F801849077FC56
:10FAF00023C0892D90E0082C02C0959587950A9423
:10FB0000E2F780FD19C0BE01082C02C0759567950B
:10FB10000A94E2F76170B62EB1946B2D872D0E9486
:10FB2000E2B26B2D70E0872D0E944CB3C60101C07C
:10FB3000880F8A94EAF7982AAA94FFEFEF1AFF0A2F
:10FB40000F5F1F4FA110CFCFDF91CF911F910F916A
:10FB5000FF90EF90DF90CF90BF90AF909F908F90ED
:10FB60007F9008950F931F9380917315813019F43E
:10FB70000E944BB408C060916F1570917015809110
:10FB800071159091721500919B1510919C15209103
:10FB90009D1530919E15601B710B820B930B28EE07
:10FBA00033E040E050E00E94ABCA809197159091FD
:10FBB0009815A0919915B0919A15BC01CD01620FCD
:10FBC000731F841F951F1F910F9108951092731535
:10FBD00010929B1510929C1510929D1510929E15D7
:10FBE00010926F1510927015109271151092721577
:10FBF00010929715109298151092991510929A15C7
:10FC00000895809173158130E1F0823051F4AADFBC
:10FC100060939715709398158093991590939A1502
:10FC200001C0D4DF81E0809373150E944BB46093D0
:10FC30009B1570939C1580939D1590939E1581E064
:10FC4000089580E00895809173158150823010F0FE
:10FC500080E00895109273150E944BB460936F1565
:10FC600070937015809371159093721581E00895CB
:10FC70001092901580E090E00E941A7410920A048D
:10FC800010920904B1DDDFDF80E090E00E941A7479
:10FC9000109294152C9810920A0410920904109254
:10FCA0009515809102018072809300010895DF9282
:10FCB000EF92FF920F931F93CF93DF93F82ED62EE0
:10FCC000E72E8A0180914102882309F439C0E9EDC9
:10FCD000F9E18491EF012196882321F00E94D63E1C
:10FCE000FE01F7CFED2DFE2D8491EF0121968823A3
:10FCF00021F00E94D63EFE01F7CFE5E8FAE18491BB
:10FD0000EF012196882321F00E94D63EFE01F7CF15
:10FD1000F7FC0BC06F2DFF0C770B880B990B0E9423
:10FD20005D428AE00E94D63E0BC0E0E8FAE1849191
:10FD3000EF012196882321F00E94D63EFE01F7CFE5
:10FD400080919F15811108C01092410281E080933B
:10FD50009F15C8010E94D04FDF91CF911F910F9145
:10FD6000FF90EF90DF9084CFEF92FF920F931F935D
:10FD7000CF93DF93809144028F37A0F08F579091FB
:10FD800094159093EA15992311F02C9A01C02C98A0
:10FD9000209195152093E91590910201222369F095
:10FDA00090950BC09091EA15891708F02C989091C6
:10FDB000E915891728F09091020190729093000143
:10FDC0008F5F809344029091E81581E089278093AA
:10FDD000E8158091430285301CF4C1E0C80F01C0D2
:10FDE000C0E0823009F4B4C054F4882301F18130BA
:10FDF00009F0E3C088E080937B0085E4C0C08430D4
:10FE000009F4C5C00CF4B7C0853009F0D6C0909194
:10FE1000E715911102C08093E7158091E715815095
:10FE20008093E715882309F4C8C0C5E0C6C0809157
:10FE300042028F5F80311CF480934202BEC0109258
:10FE4000420280919115811113C08091DD1590912E
:10FE5000DE159093DA158093D9158091DB1590917A
:10FE6000DC159093D8158093D71581E08093911578
:10FE70008AE0EDEDF5E1DF011D928A95E9F7109238
:10FE8000DC151092DB150091D9151091DA1511953A
:10FE90000195110980910F0490911004D1E018167A
:10FEA00019062CF080919415811101C0D0E0809149
:10FEB0009D0B90919E0B91958195910980179107CB
:10FEC00034F44DE15CE16EE37CE180E0F0DE8091B2
:10FED0003C0290913D02919581959109081719076F
:10FEE00044F4DD2331F040E55CE161E77CE180E052
:10FEF000DEDE8091090490910A0411E018161906BB
:10FF00002CF080919515811101C010E0E090D7157B
:10FF1000F090D81580919B0B90919C0B8E159F05AE
:10FF200034F04DE25CE16EE37CE18FEFC0DE809166
:10FF30003A0290913B02E816F9060CF43EC01123F8
:10FF4000E1F140E65CE161E77CE18FEFB0DE35C0D6
:10FF500080917A0086FD2EC0809178009091790082
:10FF60002091DD153091DE15820F931F9093DE15E1
:10FF70008093DD1522C088E080937B0086E4809327
:10FF80007C0080917A00806480937A0016C0809112
:10FF90007A0086FD11C080917800909179002091BF
:10FFA000DB153091DC15820F931F9093DC15809345
:10FFB000DB1503C0C2E001C0C4E0C09343028091DE
:10FFC000A20B81110E941AAA80919215909193150B
:10FFD0000097A9F001979093931580939215892B20
:10FFE00071F483E89CE19093360D8093350DDF9199
:10FFF000CF911F910F91FF90EF900C94023FDF91F2
:020000021000EC
:10000000CF911F910F91FF90EF9008952F923F9203
:100010004F925F926F927F928F929F92AF92BF9218
:10002000CF92DF92EF92FF920F931F93CF93DF93C4
:1000300000D01F92CDB7DEB75C017A8369834A0195
:10004000170107FD07C0802F002E000C990B9C8321
:100050008B8304C0E1E0F0E0FC83EB83F901408096
:100060005180628073808B819C81880F991F880FDB
:10007000991F9C838B8381539A4E7C01A30192012B
:10008000FC0160817181828193810E94BDC68823B9
:1000900091F0F701408251826282738211E020E088
:1000A00030E0A901C301B2010E940DCD18160CF079
:1000B00010E0F5011083F50180818230D1F08330AA
:1000C00009F45EC0813009F07CC0EB81FC81E15312
:1000D000FA4E2081318142815381F4016081718126
:1000E000828193810E94BDC687FD6BC082E0F501CD
:1000F00080838B819C8181539A4E9C838B83B60134
:1001000080E090E00E94C1C69B01AC01EB81FC81C4
:1001100060817181828193810E94E6CA9B01AC015A
:10012000F40160817181828193810E940DCD87FDF0
:1001300014C00E944BB46B017C019101A8EEB3E0A6
:100140000E94D7CAC60ED71EE81EF91EE981FA81A1
:10015000C082D182E282F38234C00E944BB4E98132
:10016000FA81C080D180E280F380DC01CB018C1960
:100170009D09AE09BF09B7FD24C083E0F501808366
:100180000F3F19F046EE5BE102C049EF5BE16DE025
:100190007CE1802F0F900F900F900F90DF91CF9107
:1001A0001F910F91FF90EF90DF90CF90BF90AF9095
:1001B0009F908F907F906F905F904F903F902F9087
:1001C00076CD0F900F900F900F90DF91CF911F91F0
:1001D0000F91FF90EF90DF90CF90BF90AF909F90E6
:1001E0008F907F906F905F904F903F902F900895E9
:1001F0004F925F926F927F928F929F92AF92BF9237
:10020000CF92DF92EF92FF920F931F93CF93DF93E2
:10021000CDB7DEB760970FB6F894DEBF0FBECDBF87
:1002200080919115811117C060960FB6F894DEBFCA
:100230000FBECDBFDF91CF911F910F91FF90EF9037
:10024000DF90CF90BF90AF909F908F907F906F90F6
:100250005F904F900895F4DB0E944BB44B015C011A
:1002600060910F0470911004072E000C880B990BFD
:100270000E94C3C669837A838B839C8348E0C42E23
:10028000D12C5CE3E52EF12C00E09E012F5F3F4F67
:1002900041E154E06FEB75E18EEB95E1B7DEC09084
:1002A0001104D0901204E0901304F09014046091B3
:1002B0009F0B7091A00B072E000C880B990B0E94CE
:1002C000C3C69B01AC01C701B6010E940DCD181633
:1002D0000CF009C160913E0270913F02072E000CA4
:1002E000880B990B0E94C3C69B01AC01C701B601E4
:1002F0000E94BDC687FFF7C000910F041091100443
:10030000B801012E000C880B990B0E94C3C6A701EF
:1003100096010E94E6CA2B013C0120ED3CEC4CE426
:100320005DE3609188157091891580918A1590918F
:100330008B150E9422C76D837E838F8398872091BF
:10034000B5153091B6154091B7155091B815C70144
:10035000B6010E94E6CA9B01AC016D817E818F814E
:1003600098850E9422C76D837E838F83988723E3BD
:1003700033E343E75FE36091B1157091B21580916B
:10038000B3159091B4150E9422C79B01AC016D81F9
:100390007E818F8198850E94E7CA6D837E838F83DB
:1003A00098876093B1157093B2158093B3159093AD
:1003B000B415C092B515D092B615E092B715F0926B
:1003C000B81520E030E040E251E4C301B2010E94E0
:1003D0000DCD18160CF431C220E030E040E251ECB3
:1003E000C301B2010E94BDC687FD2FC2012B09F4D3
:1003F0002CC28091B01581112CC22091AC15309186
:10040000AD154091AE155091AF1529873A874B87AE
:100410005C87209184153091851540918615509107
:100420008715C301B2010E9422C76B017C01A301A1
:10043000920169857A858B859C850E94E7CA6987C8
:100440007A878B879C876093AC157093AD158093EA
:10045000AE159093AF152091801530918115409184
:100460008215509183150E9422C7A70196010E9410
:10047000E7CA2D813E814F8158850E94E6CA6B01F3
:100480007C0120E030E04FE753E40E940DCD20E0F6
:1004900030E0A90118160CF4E3C1C701B6010E94AF
:1004A000BDC687FD07C0C701B6010E942BCC75955C
:1004B00067951AC020E030E0A901C301B2010E9493
:1004C000BDC687FF10C0A301920169857A858B851F
:1004D0009C850E94E6CA6093AC157093AD1580931D
:1004E000AE159093AF1560E0609394158091C3159D
:1004F0009091C415A091C515B091C6150097A1059E
:10050000B10521F1A5019401281B390B4A0B5B0BA6
:1005100057FD1CC06091C7157091C81580E090E030
:100520000E94C1C69B01AC0160911104709112043C
:1005300080911304909114040E94BDC687FF82C16C
:1005400045EC5AE167ED7AE180E0B1DB80918C15F2
:1005500090918D15A0918E15B0918F15A5019401E4
:10056000281B390B4A0B5B0B57FD0FC088DAD501EE
:10057000C4018C53964FAF4FBF4F80938C1590930F
:100580008D15A0938E15B0938F158091C9159091FC
:10059000CA15A091CB15B091CC150097A105B10556
:1005A00011F1881A990AAA0ABB0AB7FC1CC060910B
:1005B000CD157091CE1580E090E00E94C1C69B01E0
:1005C000AC0160910B0470910C0480910D0490912A
:1005D0000E040E94BDC687FF20C143EA5AE166EBC4
:1005E0007AE18FEF64DB6091090470910A04072EB1
:1005F000000C880B990B0E94C3C669837A838B8396
:100600009C8392E0C92ED12C24E1E22EF12C0FEF35
:100610009E012F5F3F4F4BE054E069EB75E18DEB9E
:1006200095E1F4DCC0900B04D0900C04E0900D0434
:10063000F0900E0420E030E040EA50E4C701B6013B
:100640000E940DCD87FDE5C020E030E04CED52E486
:10065000C701B6010E94BDC618160CF4DAC060913D
:10066000090470910A04072E000C880B990B0E9454
:10067000C3C6A70196010E94E6CA4B015C01209106
:100680007C1530917D1540917E1550917F150E940B
:1006900022C769877A878B879C872091A81530911C
:1006A000A9154091AA155091AB15C501B4010E943E
:1006B000E7CA6D837E838F8398876093A8157093B4
:1006C000A9158093AA159093AB15209178153091B8
:1006D000791540917A1550917B150E9422C76D873C
:1006E0007E878F87988B20ED3CEC4CE45DE3609136
:1006F00074157091751580917615909177150E94FB
:1007000022C72B013C012091A4153091A5154091E1
:10071000A6155091A715C701B6010E94E6CA9B0114
:10072000AC01C301B2010E9422C72B013C0123E3AB
:1007300033E343E75FE36091A0157091A1158091C9
:10074000A2159091A3150E9422C79B01AC01C30181
:10075000B2010E94E7CA2B013C016093A01570937F
:10076000A1158093A2159093A315C092A415D092C1
:10077000A515E092A615F092A7152D853E854F850B
:10078000588969857A858B859C850E94E7CAA30173
:1007900092010E94E6CA6B017C0120E030E04FE745
:1007A00053E40E940DCD20E030E0A9011816C4F5F5
:1007B000C501B4010E940DCD181684F4A501940161
:1007C0006D817E818F8198850E94E6CA6093A8150D
:1007D0007093A9158093AA159093AB156FE71AC073
:1007E00020E030E0A901C501B4010E94BDC687FF29
:1007F00010C0A50194016D817E818F8198850E9432
:10080000E6CA6093A8157093A9158093AA159093D2
:10081000AB1560E06093951507CD0E94F47BE3CEA5
:10082000C701B6010E94BDC687FDDACFC701B60178
:100830000E942BCC75956795EDCF81E08093B01524
:100840006FE752CE80E01CD881CE81E08093B01556
:100850004ACE1092B01519861A861B861C86D9CDF1
:10086000C301B2010E940DCD181654F7A3019201E5
:1008700069857A858B859C850E94E6CA6093AC1554
:100880007093AD158093AE159093AF156FE72CCE96
:1008900090916F00292F227091FF05C090916F00F9
:1008A0009D7F90936F0034E0839FC0011124FC0171
:1008B000E15AFA4E4081518162817381FC01ED5A07
:1008C000FA4E408351836283738381E08093521593
:1008D000222329F080916F00826080936F00089539
:1008E000BC012091501530915115409150155091F7
:1008F00051152417350711F09A01F7CF81E026171B
:10090000370709F080E008952F923F924F925F924F
:100910006F927F928F929F92AF92BF92CF92DF920F
:10092000EF92FF920F931F93CF93DF93CDB7DEB774
:1009300062970FB6F894DEBF0FBECDBF8091130B48
:10094000982F9270E92EE82FE470FE2EF82FF170A8
:10095000DF2E80FF04C0992311F0E11152C0EEEEAA
:10096000F9E184918F010F5F1F4F811103C0E3E50F
:10097000FFE104C00E94D63EF801F3CF84918F01BD
:100980000F5F1F4F882321F00E94D63EF801F6CF5B
:10099000D1100CC0E1E5FFE184918F010F5F1F4F83
:1009A000882321F00E94D63EF801F6CFE1100CC05A
:1009B000EFE4FFE184918F010F5F1F4F882321F047
:1009C0000E94D63EF801F6CFF11003C0EDE4FFE13E
:1009D00003C0E5E4FFE10AC084918F010F5F1F4F60
:1009E0008823B9F30E94D63EF801F6CF84918F0197
:1009F0000F5F1F4F882309F4C7C00E94D63EF8013D
:100A0000F5CF0CEA16E187EF93E09A8B898BFE0114
:100A100031965F0195EF892E96E1992E1F01F8011D
:100A20006591759185919491E989FA89C190D190E8
:100A3000E190F190FA8BE98BA70196010E94E6CA3A
:100A40002B013C01F101608371838283938320E059
:100A500030E040EA51EC0E940DCD87FD0AC020E055
:100A600030E040EA51E4C301B2010E94BDC618164D
:100A70002CF4F401849118160CF47CC0F101C1909F
:100A8000D190E190F1901F0120E030E040EA51EC7C
:100A9000C701B6010E940DCD87FD0AC020E030E0FD
:100AA00040EA51E4C701B6010E94BDC6181614F50C
:100AB000E9EDF9E184918F010F5F1F4F811103C0B0
:100AC000E9E5FFE104C00E94D63EF801F3CF84912E
:100AD0008F010F5F1F4F882321F00E94D63EF8013F
:100AE000F6CF88E290E0988B8F8788EC90E09E8725
:100AF0008D8738C00C5F1F4FFFEF8F1A9F0A86E16A
:100B0000083B180709F08BCF83EAE82E8BE0F82E1C
:100B100010E0F50181919191A191B1915F01F701EF
:100B200081939193A193B1937F01812F0E94279C80
:100B30001F5F133071F70E949E9683E992E0988BB5
:100B40008F8704E610E01E870D87BE01615F7F4F2F
:100B5000CE010D960E9469B28AEB92E0988B8F8746
:100B60001E870D87BE01615F7F4FCE010D960E94EB
:100B700069B20AC0F7FAF094F7F8F094F101C08274
:100B8000D182E282F3827ACF62960FB6F894DEBF0A
:100B90000FBECDBFDF91CF911F910F91FF90EF90CE
:100BA000DF90CF90BF90AF909F908F907F906F908D
:100BB0005F904F903F902F900895CF92DF92EF92E9
:100BC000FF920F931F93CF93DF9388E50E94713EAE
:100BD000D82E89E40E94713EC82E882319F00E9405
:100BE0000A3E1CC0DD20C1F00E943A3E20E030E009
:100BF00040E251E40E94E6CA20E030E04CEB51E4D0
:100C00000E94E7CA21E43CE44EEA5CE30E9422C76A
:100C10000E942BCC653010F01FEF01C0162F89E524
:100C20000E94713E082F8AE40E94713EC82F8823DB
:100C300019F00E940A3E1CC00023C1F00E943A3EF7
:100C400020E030E040E251E40E94E6CA20E030E0DB
:100C50004CEB51E40E94E7CA21E43CE44EEA5CE339
:100C60000E9422C70E942BCC653010F0DFEF01C03C
:100C7000D62F8AE50E94713EE82E811105C081E5DC
:100C80000E94713EF82E01C0F12CC11001C0C0E0DD
:100C90002C2F30E0D11001C000E0200F311D213099
:100CA000310521F4E1101AC0F11018C0E9EDF9E1A5
:100CB0008491EF012196811103C0E5E2FFE104C0B8
:100CC0000E94D63EFE01F4CF8491EF012196882345
:100CD00009F455C00E94D63EFE01F6CF17FD02C0B2
:100CE000D7FF17C0E9EDF9E18491EF012196811159
:100CF00003C0E6E0FFE104C00E94D63EFE01F4CF4F
:100D00008491EF0121968823D1F10E94D63EFE0105
:100D1000F7CF0E943A3E9B01AC01012F110F110B3E
:100D2000AD2FDD0FBB0BFF2099F085E0809FF00118
:100D3000819FF00D1124EA0FFB1FEE0FFF1FEE0F36
:100D4000FF1FE350FA4E608171818281938103C05D
:100D500060E070E0CB01E5E0E09FE001E19FD00DB5
:100D60001124CA0FDB1FCC0FDD1FCC0FDD1FC350BA
:100D7000DA4E0E94E7CA688379838A839B83DF9176
:100D8000CF911F910F91FF90EF90DF90CF9008953A
:100D90002F923F924F925F926F927F928F929F928B
:100DA000AF92BF92CF92DF92EF92FF920F931F9379
:100DB000CF93DF93CDB7DEB761970FB6F894DEBF60
:100DC0000FBECDBF83E50E94713E882349F00E948B
:100DD0002B3E182F811106C080E00E94C39A02C0EA
:100DE000109175168091F7039091F803A091F90383
:100DF000B091FA0389839A83AB83BC838091FB0310
:100E00009091FC03A091FD03B091FE038D839E831E
:100E1000AF83B8878091FF0390910004A0910104F3
:100E2000B091020489879A87AB87BC870E94969A03
:100E3000882309F49AC083E40E94713E882309F450
:100E400094C00E943A3E1B012C0105E0612C712CDC
:100E500038EC388B82EC898BA12CB12C98EC9E87D6
:100E6000E2E4EF87015080F125E02D87209F4001CB
:100E700011243D8531503D873F3FA1F3F401E30F3D
:100E8000F11DEE0FFF1FEE0FFF1FE350FA4EC08063
:100E9000D180E280F3809601A701B5018E859F8500
:100EA0000E940DCD18161CF45601EE86FF869601A1
:100EB000A701B301888999890E94BDC687FFD9CF50
:100EC0003601E88AF98AD5CF930148895989B50155
:100ED0008E859F850E94E7CA20E030E040E05FE316
:100EE0000E9422C7A20191010E94E7CA2B013C0186
:100EF0002DEB37E346E855EB0E940DCD87FD0AC088
:100F00002DEB37E346E855E3C301B2010E94BDC6AD
:100F100018165CF580E00E94C39A35E0D32E45E0B8
:100F2000C42EDA949FEFD91601F105E0CD9C500153
:100F300011240150B0F37501E00EF11CC701880FB8
:100F4000991F880F991FFC01E350FA4E7F01A301FE
:100F5000920160817181828193810E94E6CAF701CA
:100F60006083718382839383E4CF86E50E94713E20
:100F7000882399F00E94969A882379F0E0EFFEE1A9
:100F800084917F012FEFE21AF20A882321F00E9458
:100F9000D63EF701F5CF0E9457A98AE50E94713E1F
:100FA000882321F00E943A3E0E94D4B1812F0E94F2
:100FB000C39A111103C0EEEEF9E11CC080917516C1
:100FC0008111F9CFE9EDF9E184918F010F5F1F4F96
:100FD000882321F00E94D63EF801F6CFE1EDFEE134
:100FE00084918F010F5F1F4F882329F30E94D63E03
:100FF000F801F6CF84918F010F5F1F4F882321F0F6
:101000000E94D63EF801F6CF80917516811103C07B
:101010006FE073E002C06BE073E083EC9EE10E943E
:10102000604D8AE00E94D63EEEEEF9E184918F0198
:101030000F5F1F4F882321F00E94D63EF801F6CFA4
:10104000E6EBFEE184918F010F5F1F4F882321F0B3
:101050000E94D63EF801F6CFC0907616D090771653
:10106000E0907816F090791620E030E0A901C701F1
:10107000B6010E940DCD18164CF442E0C701B6012E
:101080000E9477428AE00E94D63E0CC0E1EBFEE16E
:1010900084918F010F5F1F4F882321F00E94D63E5D
:1010A000F801F6CF4CE050E067EF73E0CE01019617
:1010B0000E941FCE892BD1F061960FB6F894DEBF47
:1010C0000FBECDBFDF91CF911F910F91FF90EF9099
:1010D000DF90CF90BF90AF909F908F907F906F9058
:1010E0005F904F903F902F900C949E9661960FB614
:1010F000F894DEBF0FBECDBFDF91CF911F910F914E
:10110000FF90EF90DF90CF90BF90AF909F908F9027
:101110007F906F905F904F903F902F9008958091B7
:101120006F00982F927081FF05C080916F008D7FB6
:1011300080936F008091460F8093450F8093440FFA
:101140008093430F84E68093420F28EE33E0309380
:10115000931520939215992329F080916F00826056
:1011600080936F0081E0809352150E9436680E9440
:10117000B35780917516882321F08CEE9AE00E9477
:101180007B4D8CE0ECEEFAE0A7EFB3E001900D921E
:101190008A95E1F70C94C33D2F923F924F925F9254
:1011A0006F927F928F929F92AF92BF92CF92DF9277
:1011B000EF92FF920F931F93CF93DF93CDB7DEB7DC
:1011C000C554D1090FB6F894DEBF0FBECDBF85E47C
:1011D0000E94BA3E882321F00E940A3E7B0102C091
:1011E000E12CF12C83E40E94BA3E882321F00E9476
:1011F0000A3E6AA302C005E00AA385E50E94BA3E42
:10120000882319F00E942B3E03C085E50E94713EA1
:101210008CA7F7FC07C0812C912C16E1A12E13E4BA
:10122000B12E06C0812C912CBCE8AB2EB2E4BB2EB3
:1012300083E50E94BA3E882321F00E943A3E4B018A
:101240005C01E114F10411F4109296151092F90A60
:10125000ED820E944BB42B013C011D8117FD03C0A0
:1012600004E110E002C00CE310E0D301C2018C5392
:10127000964FAF4FBF4F80938C1590938D15A093D1
:101280008E15B0938F1561E06E0D623080F0E3E74C
:10129000FEE184918F010F5F1F4F1A83098388231A
:1012A00009F43AC30E94D63EE981FA81F2CFEDE912
:1012B000FEE184917F012FEFE21AF20A882321F0E8
:1012C0000E94D63EF701F5CF0E94387E3D8137FF60
:1012D00004C08FE78093951508C04D81E42F440F1B
:1012E000FF0BEC56FA4E8FE78083C501B4010E94D4
:1012F0002BCC072E000C880B990B0E94C3C66A8763
:101300007B878C879D879801A8EEB3E00E94D7CA9F
:101310006DA77EA78FA798ABDC01CB01840D951D2F
:10132000A61DB71D8AAF9BAFACAFBDAF81E0809368
:1013300040020D810F3F39F40DED1DE11FAF0EAFDF
:1013400007EA1DE106C00BEC1DE11FAF0EAF04E97B
:101350001DE122961FAF0EAF22974CA25DA26EA296
:101360007FA249AA5AAA6BAA7CAA1DAA1EAA1FAAD2
:1013700018AE19AE188E10E4198F0CE10A8F16E41E
:101380001B8F1C8E1D8E1E8E1F8E1C8A1D8A1E8A10
:101390001F8A188A198A1A8A1B8A19821A821B8242
:1013A0001C822FE730E040E050E02E833F834887E7
:1013B0005987FFE7CF2ED12CE12CF12C18A619A6C6
:1013C0001AA61BA611E01F861E8625961FAE25971E
:1013D000212C312C26961FAE26970D81802F000FD1
:1013E000990B9C012C563A4E24963FAF2EAF249772
:1013F000880F991F880F991FAC014F5E5B4F59A34F
:1014000048A38AA1082E000C990B9BA38AA3809164
:101410004002882309F47EC20E944BB44B015C0158
:1014200080919115882309F4D4C00E94207D0D81FC
:1014300007FD0CC0A8A1B9A1BC912596BFAF259707
:10144000E8A1F9A12180328003810BC000910B0437
:1014500025960FAF259720900C0430900D04009135
:101460000E0426960FAF269725962FAD2597322D81
:10147000432D26965FAD26976C8D7D8D8E8D9F8D2D
:101480000E94BDC687FF0AC025960FAD25970C8F19
:101490002D8E3E8E26960FAD26970F8F288D398D77
:1014A0004A8D5B8D25966FAD2597722D832D2696DF
:1014B0009FAD26970E94BDC687FF0AC025960FAD37
:1014C0002597088F298E3A8E26960FAD26970B8F7B
:1014D00080918C1590918D15A0918E15B0918F15DE
:1014E000A5019401281B390B4A0B5B0B57FD10C05B
:1014F0000E943F7DD501C4018C53964FAF4FBF4F23
:1015000080938C1590938D15A0938E15B0938F15A5
:1015100025962FAD2597322D432D26965FAD269724
:101520006A857B858C859D851123E9F10E94BDC666
:1015300087FF4FC0B501A401441955096609770911
:10154000DB01CA0188589341A109B109B7FD41C027
:10155000D701C6010E811F8128853985801B910B1B
:10156000A20BB30B1D81B595A7959795879517FF8E
:1015700003C08093951505C02496EEADFFAD24976A
:10158000808348A759A76AA77BA70A850C8F1B856C
:101590001D8F0C850E8F1D851F8F8CA29DA2AEA264
:1015A000BFA210E016C00E940DCD181694F4D5010C
:1015B000C4012CA13DA14EA15FA1821B930BA40BE2
:1015C000B50BAC01BD01485853416109710977FF62
:1015D000C0C120E030E040EA51E46A857B858C851B
:1015E0009D850E94E7CA25962FAD2597322D432D64
:1015F00026965FAD26970E94BDC687FF10C0EFEF0D
:10160000FDE184918F010F5F1F4F1A8309838823A7
:1016100009F480C10E94D63EE981FA81F2CFD5015A
:10162000C40129A93AA94BA95CA9821B930BA40B5D
:10163000B50BB7FD8BC00E943A7B8AE00E94D63E74
:10164000D501C4018053984FAF4FBF4F89AB9AABC0
:10165000ABABBCAB0DA9011158C02EA93FA948AD39
:1016600059AD25966FAD2597722D832D26969FAD8A
:1016700026970E940DCD1816BCF520E030E040E022
:1016800050E425966FAD2597722D832D26969FAD3C
:1016900026970E94E7CA6EAB7FAB88AF99AF2DA5A6
:1016A0003EA54FA558A9280D391D4A1D5B1D2AAF1F
:1016B0003BAF4CAF5DAF20E030E040EC50E46A85DA
:1016C0007B858C859D850E94E6CA25962FAD259742
:1016D000322D432D26965FAD26970E94BDC6881FEA
:1016E0008827881F8DAB32C0D501C4012AAD3BAD20
:1016F0004CAD5DAD821B930BA40BB50BB7FD26C0A3
:101700004EAD5FAD60EF7DE11EC020E030E040EA0D
:1017100051E46A857B858C859D850E94E6CA9B0184
:10172000AC0125966FAD2597722D832D26969FAD22
:1017300026970E94BDC687FF09C022964EAD5FADB9
:1017400022976BEB7DE18D810E94577ED501C4010C
:10175000880F991FAA1FBB1F2CA13DA14EA15FA1FD
:10176000821B930BA40BB50B84199509A609B70925
:1017700081389F44A241B10580F0E6E7FDE1849104
:101780008F010F5F1F4F1A830983882309F4C2C09A
:101790000E94D63EE981FA81F2CF2AA13BA14E8573
:1017A0005F85241735070CF032CEE9E1FDE1849125
:1017B0008F010F5F1F4F1F830E83882329F00E9424
:1017C000D63EEE81FF81F3CF1D8117FD03C00EE0F1
:1017D00013E002C009EC13E01F830E836E817F814A
:1017E00088E09DE10E94604D49815A816B817C8136
:1017F00084E09DE10E942A4D8AE00E94D63E6E81DF
:101800007F8183EF9CE10E94604D488959896A89F4
:101810007B898FEE9CE10E942A4D8AE00E94D63E91
:101820006E817F818EED9CE10E94604D4C895D89C7
:101830006E897F898AED9CE10E942A4D8AE00E9490
:10184000D63E1CA5112309F467C00D8107FF31C0E6
:1018500029813A814B815C8120937C1530937D15E1
:1018600040937E1550937F152CEA35EC47E25EE3FA
:10187000688979898A899B890E9422C76093781533
:101880007093791580937A1590937B152CEA35EC3B
:1018900047E25EE36C897D898E899F890E94C3CB74
:1018A00060937415709375158093761590937715E2
:1018B00033C089819A81AB81BC81809384159093D8
:1018C0008515A0938615B09387152CEA35EC47E271
:1018D0005EE3688979898A899B890E9422C760931F
:1018E00080157093811580938215909383152CEA4F
:1018F00035EC47E25EE36C897D898E899F890E9481
:10190000C3CB609388157093891580938A15909343
:101910008B1502C00E94387E81E08093F90ACB5B70
:10192000DF4F0FB6F894DEBF0FBECDBFDF91CF9172
:101930001F910F91FF90EF90DF90CF90BF90AF90ED
:101940009F908F907F906F905F904F903F902F90DF
:1019500008950E851F85012B09F42DC148A459A4B3
:101960006AA47BA4480E591E6A1E7B1E28A539A5B1
:101970004AA55BA5281B390B4A0B5B0B6E817F8147
:10198000888599850E949CCAA30192010E94E3CD9B
:10199000DA01C9018C0D9D1DAE1DBF1D843191055D
:1019A000A105B105FCF06C017D018C3E9105A105FE
:1019B000B1052CF05BEEC52ED12CE12CF12C20E8EA
:1019C000C216D104E104F104DCF08EEF90E0A0E057
:1019D000B0E08C199D09AE09BF098E839F83A8874B
:1019E000B98712C044E1C42ED12CE12CF12C04E1C2
:1019F00010E020E030E00E831F832887398704C081
:101A0000CE82DF82E886F986EBE6FEE184918F01E3
:101A10000F5F1F4F882321F00E94D63EF801F6CFBA
:101A2000C701B6010E945D42E6E6FEE184918F01A6
:101A30000F5F1F4F882321F00E94D63EF801F6CF9A
:101A40006E817F81888599850E945D42488D598D80
:101A50006A8D7B8D8FE59EE10E942A4D4C8D5D8DB8
:101A60006E8D7F8D88E59EE10E942A4D0E851F8533
:101A7000033011050CF49FC06E817F8188859985A4
:101A80000E94C3C620E030E040E850E40E9422C734
:101A900069837A838B839C83288D398D4A8D5B8DF6
:101AA0006C8D7D8D8E8D9F8D0E94E6CA2BED3FE063
:101AB00049E450E40E9422C720E030E040E05FE3C8
:101AC0000E9422C79B01AC0169817A818B819C8134
:101AD0000E94C3CB69837A838B839C83C301B20149
:101AE0000E94C3C62FE632E143E85AE30E9422C7B0
:101AF0002B013C0149815A816B817C8182E59EE109
:101B00000E942A4DB301A2018CE49EE10E942A4D5D
:101B10002AE939E949E15FE369817A818B819C8116
:101B20000E9422C769837A838B839C839B01AC01CB
:101B30000E94E7CAA30192010E94C3CB688B798BF4
:101B40008A8B9B8B29813A814B815C81C301B201D5
:101B50000E9422C720E030E040E05EE30E9422C7FE
:101B60006C8B7D8B8E8B9F8BECE3FEE184918F01E0
:101B70000F5F1F4F882321F00E94D63EF801F6CF59
:101B800049815A816B817C8186E39EE10E942A4DC6
:101B9000488959896A897B8980E39EE10E942A4DA0
:101BA0004C895D896E897F898AE29EE10E942A4D77
:101BB0008AE00E94D63E8E819F81A885B9858C0DD2
:101BC0009D1DAE1DBF1D1D81B595A7959795879548
:101BD00017FF03C08093951505C02496EEADFFADA9
:101BE000249780830E851F850F5F1F4F1F870E87E9
:101BF0001A85188F0B85098F1C851A8F0D850B8F01
:101C00002401350111E0E5CCCF93DF93EEEEF9E14D
